:100000000C949C100C94393A0C940E3A0C94E339ED
:100010000C94B8390C948D390C9462390C9437399E
:100020000C940C390C94CD100C94CD100C94CD1074
:100030000C94CD100C94BD3A0C94CD100C94CD10B2
:100040000C94CD100C94A7860C94CD100C94CD106C
:100050000C94CD100C94CD100C94C74B0C94073D10
:100060000C94CD100C94A0980C9475990C94CD1010
:100070000C94CD100C94CD100C94CD100C94CD108C
:100080000C94CD100C94CD100C94CD100C94CD107C
:100090000C94CD100C94CD100C94CD100C94CD106C
:1000A0000C94CD100C94CD100C94CD100C94CD105C
:1000B0000C94CD100C94CD100C94CD100C94CD104C
:1000C0000C94CD100C94CD100C94CD100C94CD103C
:1000D0000C94CD100C94CD100C94CD100C94CD102C
:1000E0000C94CD109B2F9E2F8D2F912F972FD52FB6
:1000F000A22FA62FAC2FB02FB42FBA2FBE2FC22FF6
:10010000D52FC82FCC2FD02F823B873B8C3B963BE3
:10011000A03B193CAA3BB23BBA3BC43BCE3BD83BCD
:10012000E73BF13B193CFB3B053C0F3CCF98D59896
:10013000E698F198F9980F99FD980F99019905990A
:100140000F990B99ECA8ECA8F3A8F3A8F3A8FAA8C8
:10015000FAA8FAA807A901A901A901A9084AD73B49
:100160003BCE016E84BCBFFDC12F3D6C74319ABD86
:1001700056833DDA3D00C77F11BED9E4BB4C3E91AA
:100180006BAAAABE000000803F05A84CCDB2D44E99
:10019000B93836A9020C50B9918688083CA6AAAA9B
:1001A0002ABE000000803F004E414E494E4954593E
:1001B000494E46CDCCCC3D0AD7233C17B7D1387732
:1001C000CC2B329595E6241FB14F0A000020410048
:1001D00000C84200401C4620BCBE4CCA1B0E5AAE92
:1001E000C59D7420746F6F206C6F6E672065787486
:1001F000727573696F6E2070726576656E74656472
:100200000A0020636F6C6420657874727573696F7F
:100210006E2070726576656E7465640A0047322FD1
:1002200047332062616420706172616D657465722C
:10023000730A0050726F62696E67206661696C654F
:1002400064004D31313720426564206C6576656C01
:10025000696E67206661696C65642E0A4730205AB2
:1002600031300A47302045300A4D3330302050328B
:100270003520533838300A4D333030205035302057
:1002800053300A4D33303020503235205338383017
:100290000A4D333030205035302053300A4D333042
:1002A000302050323520533838300A47342053310B
:1002B000004D3131372050726F6265207375636372
:1002C00065737366756C0A0050524F424520464173
:1002D000494C20434C45414E204E4F5A5A4C450AFA
:1002E000004D31303420533137300A4D3131372011
:1002F0005265776970696E67206E6F7A7A6C650AED
:100300004D3132310A4730205A31300A47323820D5
:1003100058302059300A4D31303920523137300AA7
:100320004D313137205265776970696E67206E6F85
:100330007A7A6C650A4731322050302053313220AE
:1003400054300A4D31303420533136300A4D313279
:10035000300A4D3131372050726F62696E6720620A
:1003600065640020573A0020573A00544845524DE2
:10037000414C5F50524F54454354494F4E004155F4
:10038000544F5245504F52545F53445F535441545D
:10039000555300454D455247454E43595F504152D4
:1003A00053455200434153455F4C494748545F42CF
:1003B00052494748544E45535300544F47474C45C4
:1003C0005F4C494748545300534F46545741524598
:1003D0005F504F574552004255494C445F5045527B
:1003E00043454E54004C4556454C494E475F4441A9
:1003F0005441005A5F50524F4245004155544F4CB2
:100400004556454C005052494E545F4A4F420050A9
:10041000524F4752455353004155544F5245504F48
:1004200052545F54454D5000564F4C554D45545213
:10043000494300454550524F4D0053455249414CA8
:100440005F584F4E5F584F4646004649524D574100
:1004500052455F4E414D453A4D61726C696E2020A8
:100460004649524D574152455F56455253494F4EAA
:100470003A312E312E392E333420455854525544BA
:1004800045525F545950453A536D616C6C4C6179DB
:10049000657220534F555243455F434F44455F5566
:1004A000524C3A68747470733A2F2F636F64652EE0
:1004B000616C6570686F626A656374732E636F6DDB
:1004C0002F646966667573696F6E2F4D41524C4992
:1004D0004E2050524F544F434F4C5F564552534954
:1004E0004F4E3A312E30204D414348494E455F54DE
:1004F0005950453A4C756C7A426F74204D696E695B
:100500002045585452554445525F434F554E543A36
:100510003120555549443A33353134383762362D18
:10052000636139612D346331612D383736352D647F
:1005300036363862316461363538350A002F2F205F
:10054000007A5F6D61783A20007A5F6D696E3A20BB
:1005500000795F6D61783A2000795F6D696E3A20AD
:1005600000785F6D61783A2000785F6D696E3A209F
:10057000005265706F7274696E6720656E64737483
:100580006F70207374617475730A004B64200023CC
:10059000646566696E652044454641554C545F006C
:1005A0004B69200023646566696E652044454641B9
:1005B000554C545F004B70200023646566696E657E
:1005C0002044454641554C545F00504944204175F4
:1005D000746F74756E652066696E697368656421F1
:1005E0002050757420746865206C617374204B70A2
:1005F0002C204B6920616E64204B6420636F6E7306
:1006000074616E74732066726F6D2062656C6F77B3
:1006100020696E746F20436F6E66696775726174CE
:10062000696F6E2E680A00504944204175746F74DA
:10063000756E65206661696C6564212074696D65FD
:100640006F75740A00453120544845524D414C2085
:1006500052554E4157415900424544205448455255
:100660004D414C2052554E415741590054686572D6
:100670006D616C2052756E6177617900453120485B
:10068000656174696E67206661696C6564004265C6
:10069000642068656174696E67206661696C656471
:1006A0000048656174696E67206661696C65640005
:1006B000504944204175746F74756E652066616998
:1006C0006C6564212054656D706572617475726526
:1006D00020746F6F20686967680A00204B643A20B5
:1006E00000204B693A2000204B703A20000A20433A
:1006F0006C617373696320504944200A002054756B
:100700003A2000204B753A2000206D61783A200095
:10071000206D696E3A200020643A200020626961F1
:10072000733A2000504944204175746F74756E65AA
:10073000206661696C65642120426164206578747B
:100740007275646572206E756D6265720A0050493B
:1007500044204175746F74756E6520737461727492
:100760000A0020643A0020693A0020703A004E6F77
:100770002063617365206C696768740A0042656470
:10078000204C6576656C696E6720004661696C6512
:100790006420746F20656E61626C65204265642020
:1007A0004C6576656C696E670A00426564204C652D
:1007B00076656C20436F7272656374696F6E204D4D
:1007C00061747269783A0020202020202846312E5A
:1007D00030203D2066756C6C20636F7272656374A7
:1007E000696F6E2C2046302E30203D206E6F2063C6
:1007F0006F7272656374696F6E290A00202046610A
:1008000064653A2020202020202020202020202045
:100810002020202046002020536D6F6F7468696E81
:100820006720286D6D293A202020202020205300A9
:10083000202044697374616E636520286D6D293AC8
:1008400020202020202020205A004261636B6C6110
:10085000736820636F7272656374696F6E20697369
:10086000206163746976653A0A004261636B6C616A
:10087000736820636F7272656374696F6E20697349
:1008800020696E6163746976653A0A004261636B40
:100890006C617368206D6561737572656D656E74EA
:1008A00020286D6D293A202000454550524F4D209B
:1008B0004F4B0A003A200050726F6265205A204F59
:1008C0006666736574003F5A206F7574206F6620EA
:1008D00072616E676520282D3220746F2035290AD9
:1008E000003F4B2076616C7565206F7574206F66D4
:1008F0002072616E67652028302D3130292E0A0064
:10090000416476616E6365204B3D00416374697696
:10091000652045787472756465723A2000496E7678
:10092000616C69642065787472756465720A000090
:100930000020002300260029002C002F0032000098
:100940000100000301060109010225697300256900
:100950006D20256973002569682025696D2025694A
:100960007300256964202569682025696D20256943
:100970007300256979202569642025696820256927
:100980006D2025697300486F6D696E672066616927
:100990006C656400656E7175657565696E672022AA
:1009A000004C696E65204E756D626572206973201A
:1009B0006E6F74204C617374204C696E65204E75A7
:1009C0006D6265722B312C204C617374204C696E02
:1009D000653A20005072696E7465722073746F708E
:1009E0007065642064756520746F206572726F7223
:1009F000732E2046697820746865206572726F7264
:100A000020616E6420757365204D39393920746F0B
:100A100020726573746172742E202854656D706540
:100A20007261747572652069732072657365742EC6
:100A30002053657420697420616674657220726544
:100A40007374617274696E67290A004E6F2043687F
:100A500065636B73756D2077697468206C696E656A
:100A6000206E756D6265722C204C617374204C6928
:100A70006E653A2000636865636B73756D206D6900
:100A8000736D617463682C204C617374204C696EC3
:100A9000653A20004D3131300020496E76616C6935
:100AA000642065787472756465722000000040C02F
:100AB0000000E0C0000000C000002243CDCC36435F
:100AC00000001F432066697273740A005A005900BF
:100AD0005800486F6D652000434F4D4D554E4943BA
:100AE0004154494F4E0044525952554E00455252BE
:100AF0004F525300494E464F004543484F005072F5
:100B0000696E742074696D653A2000000125301DFE
:100B10000C1E2829FF24311C0B184527FF232F1BEF
:100B20000A174443FFFFFFFF040806FF06222B1AA3
:100B30004142FF043803FF3650726F746563746579
:100B4000642050696E0A0046696C616D656E7420A0
:100B5000757365643A200053746174733A20002CF5
:100B6000204C6F6E67657374206A6F623A20005480
:100B70006F74616C2074696D653A20005374617400
:100B8000733A20002C204661696C65643A20002C81
:100B90002046696E69736865643A20005072696E18
:100BA00074733A200053746174733A20006F6B00C1
:100BB000F90AF40AED0AE60AD80A6F6666004445A7
:100BC0004255473A004D313133205300205A3A0004
:100BD00020593A0020436F756E7420583A00204522
:100BE0003A00205A3A0020593A00583A003A004355
:100BF00061703A00205400205200416363656C65C7
:100C0000726174696F6E3A205000205A00205900BA
:100C1000580020204D61783A2000205A00205900C9
:100C2000580020204D696E3A20004F6E20004F661C
:100C30006600536F667420656E6473746F70733AE8
:100C4000200020466C6F773A200020643A0020692B
:100C50003A0020703A00496E76616C6964206578CC
:100C60007472756465720A0043290A0061626C65DA
:100C70006420286D696E2074656D702000436F6C70
:100C800064206578747275646573206172652000F4
:100C9000546F6F206661722066726F6D2072656698
:100CA0006572656E636520706F696E740A0010006E
:100CB000C90210012C014001220170011801B0018C
:100CC0000E01F00104015002FA00B002F0003003FE
:100CD000E600D003DC009004D2007005C800A00636
:100CE000BE000008B400B009AA00D00BA000600E3E
:100CF000960060118C000015820020197800C01D3C
:100D00006E00A0226400B0275A00902C50000031E1
:100D10004600E0343C0010383200903A2800603C35
:100D20001E00A03D1400803E0A00203F00006265C6
:100D3000640A002C2073797374656D2073746F706E
:100D400070656421204865617465725F49443A208A
:100D5000004265642068656174696E672066616938
:100D60006C65640048656174696E67206661696CD2
:100D700065640045312048656174696E672066616D
:100D8000696C65640048656174696E6720666169B5
:100D90006C6564004B494C4C45442E20001000AD5E
:100DA0000330016A0150022B0170030A019004F51F
:100DB00000B005E500D006D800F007CE001009C548
:100DC00000300ABE00500BB700700CB100900DABA4
:100DD00000B00EA600D00FA200F0109D00101299D6
:100DE00000301395005014920070158E0090168BF1
:100DF00000B0178700D0188400F0198100101B7E06
:100E000000301C7B00501D7900701E7600901F730F
:100E100000B0207000D0216E00F0226B0010246919
:100E20000030256600502663007027610090285E20
:100E300000B0295C00D02A5900F02B5600102D5428
:100E400000302E5100502F4E0070304B0090314832
:100E500000B0324500D0334200F0343E0010363B43
:100E600000303737005038330070392E00903A295F
:100E700000B03B2300D03C1B00F03D1100103F01AF
:100E800000F03F00004531204572723A204D415834
:100E900054454D50004572723A204D415854454DCD
:100EA0005020424544004D415854454D50207472E5
:100EB00069676765726564004531204572723A2042
:100EC0004D494E54454D50004572723A204D494EA1
:100ED00054454D5020424544004D494E54454D50D7
:100EE0002074726967676572656400202F00204274
:100EF000403A0020403A0020746F6F206C6F6E679C
:100F000020657874727573696F6E2070726576658E
:100F10006E7465640A0020636F6C64206578747277
:100F20007573696F6E2070726576656E7465640A9C
:100F3000000A0A426564204C6576656C20436F7236
:100F400072656374696F6E204D61747269783A00DE
:100F5000202B000A436F72726563746564204265DA
:100F600064204865696768742076732E2042656442
:100F700020546F706F6C6F67793A0A00202B000A5B
:100F80004265642048656967687420546F706F67B4
:100F900072617068793A0A2020202B2D2D2D204275
:100FA00041434B202D2D2B0A2020207C2020202067
:100FB000202020202020207C0A204C207C20202063
:100FC00020282B29202020207C20520A2045207C0C
:100FD00020202020202020202020207C20490A20A2
:100FE00046207C20282D29204E20282B29207C20BB
:100FF000470A2054207C2020202020202020202050
:10100000207C20480A2020207C20202020282D29F8
:10101000202020207C20540A2020207C20202020FA
:10102000202020202020207C0A2020204F2D2D2031
:1010300046524F4E54202D2D2B0A2028302C30297B
:101040000A004D65616E206F662073616D706C657E
:101050006420706F696E74733A200020643A200037
:1010600020623A200045716E20636F656666696391
:1010700069656E74733A20613A2000347468207098
:10108000726F626520706F696E742C20646973746E
:10109000616E63652066726F6D20706C616E653A7B
:1010A0002000202844525952554E290047323920F9
:1010B0004175746F20426564204C6576656C696E7D
:1010C00067003F20284C2C522C462C4229206F755B
:1010D00074206F6620626F756E64732E0A003F5035
:1010E000726F626520706F696E74732028592920B1
:1010F000697320696D706C61757369626C65202815
:10110000322D32292E0A003F50726F626520706FB7
:10111000696E74732028582920697320696D706C7A
:1011200061757369626C652028322D32292E0A00A0
:101130003F2856296572626F7365206C6576656C11
:1011400020697320696D706C61757369626C6520CC
:1011500028302D34292E0A00205A3A200020593AEE
:10116000200042656420583A20002020506C616EB7
:101170006E657242756666657242797465733A206F
:10118000002046726565204D656D6F72793A2000CA
:10119000436F6D70696C65643A204A616E2031302E
:1011A00020323031390A00207C20417574686F721A
:1011B0003A2028416C657068204F626A65637473D9
:1011C00020496E632E2C204C756C7A426F74204738
:1011D0006974205265706F7369746F7279290A009F
:1011E0004A616E203130203230313931333A333870
:1011F0003A323400204C6173742055706461746518
:10120000643A2000312E312E390A004D61726C692A
:101210006E0020536F667477617265205265736546
:10122000740A00205761746368646F6720526573A5
:1012300065740A002042726F776E206F75742052B9
:10124000657365740A002045787465726E616C2060
:1012500052657365740A00506F77657255700A00A5
:1012600073746172740A00205A3A0020593A0020BF
:10127000583A00656E6473746F7073206869743ACD
:101280002000454550524F4D206461746173697A66
:1012900065206572726F722E0A00290A0020627939
:1012A0007465733B20637263200053657474696EC8
:1012B00067732053746F726564202800290A002028
:1012C00062797465733B2063726320002073746FCE
:1012D0007265642073657474696E677320726574D7
:1012E000726965766564202800202863616C6375E7
:1012F0006C6174656429210A0020213D2000454568
:1013000050524F4D20435243206D69736D61746399
:1013100068202D202873746F726564292000205383
:10132000697A653A2000496E6465783A2000204D5C
:1013300061726C696E3D563535290A002845455065
:10134000524F4D3D00454550524F4D2076657273CA
:10135000696F6E206D69736D61746368200024F499
:10136000D43050C38E20C2A24017828B7011127AE3
:10137000910D816CD90AA861E108C75866076151CF
:1013800043061E4B5D05C145A7041A411104093DE2
:101390009803713931034036DB0265339102D43052
:1013A0005402802E1D02632CEE01752AC501B0285F
:1013B000A001102781018F2564012B244B01E0221D
:1013C0003401AC211F018D200D01801FFC00841E03
:1013D000ED00971DDF00B81CD200E61BC600201BE5
:1013E000BC00641AB200B219A8000A19A0006A1859
:1013F0009900D117910040178B00B5168400311663
:101400007E00B31579003A157300C7146F005814A5
:101410006A00EE1366008813630025135E00C7128E
:101420005B006C12570015125400C111510070116D
:101430004F0021114B00D61049008D104700461077
:10144000440002104200C00F4000800F3E00420FD7
:101450003C00060F3B00CB0E3800930E37005C0EAD
:101460003500270E3400F30D3200C10D3100900D10
:101470003000600D2E00320D2D00050D2C00D90C12
:101480002B00AE0C2900850C29005C0C2700350CC4
:1014900027000E0C2600E80B2400C40B2400A00B30
:1014A00023007D0B23005A0B2100390B2100180B60
:1014B0002000F80A1F00D90A1E00BB0A1E009D0A60
:1014C0001D00800A1D00630A1C00470A1B002C0A2D
:1014D0001B00110A1A00F7091A00DD091900C409D6
:1014E0001900AB091900920917007B09180063095C
:1014F00017004C09160036091600200916000A09C3
:101500001500F5081500E0081400CC081400B80810
:101510001400A4081400900813007D0812006B0842
:10152000130058081200460812003408110023085E
:1015300011001208110001081100F0071000E00767
:101540001000D0071000C0071000B0070F00A1075F
:10155000100091070E0083070F0074070F00650746
:101560000E0057070E0049070E003B070D002E071F
:101570000E0020070D0013070D0006070D00F906E9
:101580000C00ED060D00E0060C00D4060C00C806A9
:101590000C00BC060C00B0060C00A4060B0099065B
:1015A0000C008D060B0082060B0077060B006C0604
:1015B0000B0061060A0057060B004C060A004206A3
:1015C0000A0038060A002E060A0024060A001A0637
:1015D0000A001006090007060A00FD050900F405C7
:1015E0000900EB050900E2050900D9050900D0054D
:1015F0000900C7050900BE050900B5050800AD05CD
:101600000800A50509009C050800940508008C0544
:101610000800840508007C050800740508006C05B6
:101620000700650508005D050700560508004E0522
:101630000700470507004005080038050700310589
:1016400007002A050700230507001C0506001605EC
:1016500007000F0507000805060002050700FB0448
:101660000600F5040700EE040600E8040600E204A4
:101670000700DB040600D5040600CF040600C904F9
:101680000600C3040600BD040600B7040600B1044A
:101690000500AC040600A6040600A00405009B0497
:1016A000060095040500900406008A0405008504E0
:1016B0000500800406007A04050075040500700426
:1016C00005006B04050066040500610405005C0468
:1016D000050057040500520405004D0405004804A8
:1016E0000500430405003E0404003A0405003504E7
:1016F0000500300404002C04050027040400230422
:1017000005001E0404001A04040016040500110458
:1017100004000D040400090405000404040000048E
:101720000400FC030400F8030400F4030400F003C5
:101730000400EC030400E8030400E4030400E003F5
:101740000400DC030400D8030400D4030400D00325
:101750000400CC030400C8030300C503030024F401
:1017600004D9201BC40C5C0E9804C4095F026507F1
:101770007101F405F900FB04B30048048700C103BC
:1017800069005803550003034500BE023A00840275
:10179000310053022A002902250004022000E4013E
:1017A0001C00C8011900AF01170098011400840142
:1017B0001300710110006101100051010E0043017E
:1017C0000D0036010B002B010B0020010B00150151
:1017D00009000C01090003010800FB000800F300E8
:1017E0000800EB000700E4000600DE000600D80059
:1017F0000600D2000600CC000500C7000500C200AC
:101800000500BD000400B9000400B5000400B100EB
:101810000400AD000400A9000400A5000300A2001C
:1018200003009F0004009B00030098000300950044
:10183000020093000300900003008D0002008B0063
:10184000030088000200860002008400030081007B
:1018500002007F0002007D0002007B000200790090
:10186000020077000100760002007400020072009E
:101870000100710002006F0002006D0001006C00A9
:1018800002006A00010069000200670001006600B2
:1018900001006500010064000200620001006100B7
:1018A0000100600001005F0002005D0001005C00BB
:1018B00001005B0001005A000100590001005800BE
:1018C00001005700010056000100550001005400BE
:1018D00001005300000053000100520001005100BC
:1018E0000100500001004F0001004E0000004E00BA
:1018F00001004D0001004C0001004B0000004B00B6
:1019000001004A00010049000100480000004800B1
:1019100001004700010046000000460001004500AC
:1019200000004500010044000100430000004300A6
:10193000010042000000420001004100000041009F
:101940000100400001003F0000003F0001003E0098
:1019500000003E0001003D0000003D0001003C0091
:1019600000003C0000003C0001003B0000003B0088
:1019700001003A0000003A0001003900000039007F
:101980000100380000003800000038000100370076
:10199000000037000100360000003600000036006D
:1019A0000100350000003500000035000100340062
:1019B0000000340000003400010033000000330058
:1019C000000033000100320000003200000032004D
:1019D0000100310000003100000031000100300042
:1019E000000030000000300001002F0000002F0038
:1019F00000002F0000002F0001002E0000002E002C
:101A000000002E0001002D0000002D0000002D0020
:101A100000002D0001002C0000002C0000002C0014
:101A200000002C0001002B0000002B0000002B0008
:101A300000002B0001002A0000002A0000002A00FC
:101A400000002A00010029000000290000002900F0
:101A500000002900000029000100280000002800E3
:101A600000002800000028000000280001002700D6
:101A700000002700000027000000270000002700CA
:101A800001002600000026000000260000002600BD
:101A900000002600010025000000250000002500B0
:101AA00000002500000025000000250001002400A2
:101AB0000000240000002400000024000000240096
:101AC0000100230000002300000023000000230089
:101AD000000023000000230000002300010022007A
:101AE000000022000000220000002200000022006E
:101AF0000000220001002100000021000000210060
:101B00000000210000002100000021000000210051
:101B10000100200000002000000020000000200044
:101B20000000200000002000000020000000200035
:101B300001001F0000001F0000001F0000001F0028
:101B400000001F0000001F0000001F0001001E0019
:101B500000001E0000001E0000001E000000C23138
:101B600000001C260000F4190000D80F0000EB084C
:101B70000000C00400007502000040010000526532
:101B800073656E643A20002042002050006F6B00A5
:101B9000627573793A2070617573656420666F723F
:101BA00020696E7075740A00627573793A207061ED
:101BB0007573656420666F7220757365720A0062C2
:101BC0007573793A2070726F63657373696E670A13
:101BD000004B494C4C45442E20004B494C4C206353
:101BE000617573656420627920746F6F206D756311
:101BF0006820696E6163746976652074696D65201B
:101C00002D2063757272656E7420636F6D6D616EE9
:101C1000643A20005072696E7465722068616C7459
:101C200065642E206B696C6C28292063616C6C657F
:101C300064210A00000040C0CDCC364300001F43A1
:101C40000000F0410000F0410000004100000000F1
:101C50005761726E696E673A20486F6D696E6720D2
:101C600042756D702044697669736F72203C203133
:101C70000A000202040000A0400000A04000000092
:101C80004000002543CDCC3D4300002143FF01012E
:101C900048617264636F6465642044656661756C55
:101CA000742053657474696E6773204C6F6164654A
:101CB000640A00282300002823000064000000E8D4
:101CC000030000000096430000964300000041001E
:101CD0000020420000C9420000C9420000C8440080
:101CE00000D2433A0A0020286D6D290020450020CB
:101CF0005A0020204D3930372058005374657070D9
:101D00006572206D6F746F722063757272656E7488
:101D1000733A0A0020204D393030204B004C696E58
:101D200065617220416476616E63653A0A00202025
:101D30004D383531205A005A2D50726F6265204F50
:101D400066667365740020440020490020204D33EE
:101D5000303420500020440020490020204D3330F2
:101D6000312050005049442073657474696E677364
:101D70003A0A0020204D3432302053004175746FF0
:101D800020426564204C6576656C696E673A0A008E
:101D9000205A0020590020204D323036205800486B
:101DA0006F6D65206F66667365743A0A00204500A2
:101DB000205A0020590020580020540020530020B1
:101DC000204D32303520420020453C6D61785F6502
:101DD0005F6A65726B3E0020583C6D61785F785F8A
:101DE0006A65726B3E20593C6D61785F795F6A6508
:101DF000726B3E205A3C6D61785F7A5F6A65726BE8
:101E00003E00416476616E6365643A20423C6D69D0
:101E10006E5F7365676D656E745F74696D655F7520
:101E2000733E20533C6D696E5F66656564726174D4
:101E3000653E20543C6D696E5F74726176656C5FBF
:101E400066656564726174653E002054002052002E
:101E500020204D323034205000416363656C657240
:101E60006174696F6E2028756E6974732F733229DF
:101E70003A20503C7072696E745F616363656C3EBA
:101E800020523C726574726163745F616363656C58
:101E90003E20543C74726176656C5F616363656C6F
:101EA0003E0A00204500205A0020590020204D32D3
:101EB00030312058004D6178696D756D2041636344
:101EC000656C65726174696F6E2028756E697473D4
:101ED0002F7332293A0A00204500205A0020590069
:101EE00020204D3230332058004D6178696D756D7A
:101EF000206665656472617465732028756E697407
:101F0000732F73293A0A00204500205A00205900F7
:101F100020204D393220580053746570732070654D
:101F20007220756E69743A0A0020204D32303020DC
:101F300044300A0020204D323030204400204469D3
:101F40007361626C65640A0046696C616D656E74EC
:101F50002073657474696E67733A002020473231CC
:101F6000202020203B004D6963726F73746570738D
:101F700020756E617661696C61626C650A0045303E
:101F80003A20005A3A2000593A2000583A20004D91
:101F900053312C4D53322050696E730A00457272D2
:101FA0006F722077726974696E6720746F2045457F
:101FB00050524F4D210A00556E6B6E6F776E206345
:101FC0006F6D6D616E643A2022006563686F3A0040
:101FD00000000A0B02090C0D0E08070304010000A3
:101FE00000000000000000000000000000000000F1
:101FF00000000000000000000000000012111000AE
:1020000000000000000000000000000000000000D0
:1020100000000000000050726F62696E6720666108
:10202000696C65640A00205A3A200020593A200061
:1020300042656420583A20004572726F723A00453A
:102040003120544845524D414C2052554E41574144
:10205000590042454420544845524D414C20525568
:102060004E4157415900546865726D616C2052753C
:102070006E617761790000002200250028002B00A6
:102080002E003100340002010000050108010B019F
:1020900000002100240027002A002D00300033001A
:1020A00001010000040107010A01050505050705F6
:1020B00008080808020202020A0A080804040404C4
:1020C00001010101010101010303030303030303F0
:1020D000040707070C0C0C0C0C0C0C0C020202027F
:1020E00006060606060606060B0B0B0B0B0B0B0B68
:1020F000010210202008081020401020408002011A
:1021000002010804020101020408102040808040FE
:1021100020100804020180040201804020100804FD
:10212000020108040201010204081020408001029B
:1021300004081020408040A411241FBECFEFD1E23C
:10214000DEBFCDBF00E00CBF13E0A0E0B2E0E8EFDF
:10215000F9E601E00BBF02C007900D92A631B1076E
:10216000D9F72EE0A6E1B3E001C01D92AB3DB20766
:10217000E1F710E1CCE9D0E100E006C021970109C8
:10218000802FFE010E94B4B4CB39D10780E008074C
:10219000A9F70E942B770C94FAB40C9400002F92AC
:1021A0003F924F925F926F927F928F929F92AF92E7
:1021B000BF92CF92DF92EF92FF920F931F93CF9334
:1021C000DF93CDB7DEB7C459D1090FB6F894DEBF9F
:1021D0000FBECDBFC257DF4F8883CE58D04021E01D
:1021E0002093E40C8091060E8D3411F40C946B1B3B
:1021F000843511F40C949928873411F00C94DC2860
:10220000E090040EF090050E3AE1E316F10409F4B3
:1022100071C7CCF454E0E516F1044CF482E0E81602
:10222000F1040CF062C0F7FE34C00C94671B94E01C
:10223000E916F10409F4FDC5ACE0EA16F10409F46D
:102240002DC60C94671BBEE1EB16F10411F40C943F
:102250005B1B4CF4FCE1EF16F10409F4E5C70CF448
:102260004DC70C94191B3BE5E316F10411F40C94D3
:102270005F1B4CE5E416F10411F40C94631B5AE562
:10228000E516F10411F00C94671B10921D030C94D9
:10229000DE2880911F02882311F40C94DE288AE541
:1022A0000E947535482F89E5C057DF4F4883C059D4
:1022B000D0400E947535682F88E5C157DF4F68838D
:1022C000CF58D0400E947535C057DF4F4881C05964
:1022D000D040C157DF4F6881CF58D0400E94853031
:1022E00081110C94DE280C94EB2841E061E081E040
:1022F0000E94853081110C94DE2880911F02882372
:1023000011F40C94DE2811E0B2E0EB16F10409F0B0
:1023100010E00E94C83582E50E94BC35882309F48C
:102320003CC10E943E356B017C014090260E5090CE
:10233000270E6090280E7090290E20912A0E309161
:102340002B0E40912C0E50912D0E2DA73EA74FA77E
:1023500058AB8091290D90912A0DA0912B0DB09131
:102360002C0D89AB9AABABABBCAB20912D0D309152
:102370002E0D40912F0D5091300D2DAB3EAB4FAB3C
:1023800058AF20E030E0A901C701B6010E9474AD4A
:10239000882309F434C5A301920169A97AA98BA9FC
:1023A0009CA90E9474AD81110DC02DA53EA54FA51D
:1023B00058A96DA97EA98FA998AD0E9474AD8823F4
:1023C00009F41DC520E030E0A901C701B6010E9453
:1023D00074AD881F8827881F18130BC080E090E019
:1023E000A0E8BFE329968CAF9DAFAEAFBFAF2997F2
:1023F0000AC020E030E040E85FEB29962CAF3DAF0B
:102400004EAF5FAF2997A301920169A97AA98BA961
:102410009CA90E94D7B121966CAF7DAF8EAF9FAFC4
:1024200021972DA53EA54FA558A96DA97EA98FA9D5
:1024300098AD0E94D7B125966CAF7DAF8EAF9FAFA0
:10244000259721962CAD3DAD4EAD5FAD2197CA01CC
:10245000B9010E94D9AD4B015C0125962CAD3DAD73
:102460004EAD5FAD2597CA01B9010E94D9AD9B0160
:10247000AC01C501B4010E94D8B10E9443B469AF58
:102480007AAF8BAF9CAF20E030E040E05FE30E948A
:10249000D9AD4B015C01A7019601C701B6010E94AD
:1024A000D9AD6B017C01A5019401C501B4010E9465
:1024B000D9AD9B01AC01C701B6010E94D7B10E9402
:1024C00043B49B01AC0129966CAD7DAD8EAD9FAD43
:1024D00029970E94D9AD4B015C0129A93AA94BA9C2
:1024E0005CA9C301B2010E94D8B120E030E040E015
:1024F0005FE30E94D9AD6B017C0125966CAD7DAD8B
:102500008EAD9FAD2597905829AD3AAD4BAD5CADE2
:102510000E94B4B29B01AC01C501B4010E94D9ADC7
:102520009B01AC01C701B6010E94D8B1A301920181
:102530000E94D7B16B017C012DA93EA94FA958ADCE
:102540006DA57EA58FA598A90E94D8B120E030E0A6
:1025500040E05FE30E94D9AD2B013C0129AD3AADCB
:102560004BAD5CAD21966CAD7DAD8EAD9FAD219731
:102570000E94B4B29B01AC01C501B4010E94D9AD67
:102580009B01AC01C301B2010E94D8B12DA53EA5AB
:102590004FA558A90E94D7B114C089E40E94BC3548
:1025A000882329F00E943E356B017C0103C0C12CB9
:1025B000D12C76018AE40E94BC358823D9F00E9490
:1025C0003E356DAB7EAB8FAB98AF20E030E0A9011C
:1025D000C701B6010E9474AD81111AC020E030E03D
:1025E000A9016DA97EA98FA998AD0E9474AD811132
:1025F0000FC005C420E030E0A901C701B6010E9468
:1026000074AD882309F4FBC31DAA1EAA1FAA18AE25
:10261000D701C601B0588DA79EA7AFA7B8AB2DA90B
:102620003EA94FA958AD505829AB3AAB4BAB5CAB68
:102630009C01AD01BC01CD010E94D9AD4B015C01F3
:1026400029A93AA94BA95CA9CA01B9010E94D9AD2F
:102650009B01AC01C501B4010E94D8B10E9443B4F2
:1026600065966CAF7DAF8EAF9FAF65978091260E5C
:102670009091270EA091280EB091290E89AF9AAFA4
:10268000ABAFBCAFA7019601BC01CD010E94D8B190
:1026900029966CAF7DAF8EAF9FAF299720912A0E00
:1026A00030912B0E40912C0E50912D0E21962CAF77
:1026B0003DAF4EAF5FAF21972DA93EA94FA958ADB1
:1026C00021966CAD7DAD8EAD9FAD21970E94D8B1A6
:1026D00069966CAF7DAF8EAF9FAF69978091290DE2
:1026E00090912A0DA0912B0DB0912C0D25968CAFB9
:1026F0009DAFAEAFBFAF259729962CAD3DAD4EAD8A
:102700005FAD2997BC01CD010E94D7B16B017C015F
:1027100020912D0D30912E0D40912F0D5091300DA7
:102720002D962CAF3DAF4EAF5FAF2D9769962CAD78
:102730003DAD4EAD5FAD69972D966CAD7DAD8EAD67
:102740009FAD2D970E94D7B14B015C0180912E0E59
:1027500090912F0EA091300EB091310E61968CAFFA
:102760009DAFAEAFBFAF61979C01AD016091310DE0
:102770007091320D8091330D9091340D0E94D7B13C
:102780002B013C012091350D3091360D4091370DD4
:102790005091380DA1962CAF3DAF4EAF5FAFA197D2
:1027A0008091320E9091330EA091340EB091350E7F
:1027B0006D968CAF9DAFAEAFBFAF6D97A701960181
:1027C0006DA57EA58FA598A90E94D9ADA5966CAFE1
:1027D0007DAF8EAF9FAFA597A501940169A97AA996
:1027E0008BA99CA90E94D9AD9B01AC01A5966CADAB
:1027F0007DAD8EAD9FADA5970E94D8B1A5966CAF6B
:102800007DAF8EAF9FAFA597A50194016DA57EA565
:102810008FA598A90E94D9AD4B015C01A701960133
:1028200069A97AA98BA99CA90E94D9AD9B01AC0189
:10283000C501B4010E94D7B1A5962CAD3DAD4EADFA
:102840005FADA5970E944BB26B017C0120E030E0A8
:10285000A9010E9474AD87FF0AC02BED3FE049EC4F
:1028600050E4C701B6010E94D8B16B017C0111236D
:1028700051F02BED3FE049EC50E4C701B6010E9456
:10288000D7B16B017C0120E030E0A901C701B6019E
:102890000E9474AD811126C025962CAD3DAD4EAD84
:1028A0005FAD259769AD7AAD8BAD9CAD0E9474ADDF
:1028B000811118C02D962CAD3DAD4EAD5FAD2D975D
:1028C00021966CAD7DAD8EAD9FAD21970E9474AD0C
:1028D000811108C00BEDC02E0FE0D02E09ECE02EC8
:1028E00000E4F02EA701960165966CAD7DAD8EAD2E
:1028F0009FAD65970E94D9AD4B015C0120E030E0AF
:10290000A901C301B2010E9474AD8823C9F0A501D9
:102910009401C501B4010E94D9AD4B015C01A30132
:102920009201C301B2010E94D9AD9B01AC01C50166
:10293000B4010E94D8B10E9443B44B015C010DC0A8
:1029400020E030E0A901C501B4010E94FEB387FF79
:1029500004C0B7FAB094B7F8B0942FE632E143E878
:102960005AE3C501B4010E9474AD87FF02C00C9404
:10297000DE28C501B4010E944DB30E9421B31B01A2
:10298000672B19F422242394312CB10180E090E0CC
:102990000E9478AD4B015C019B01AC01C701B601FF
:1029A0000E94B4B269AF7AAF8BAF9CAFA50194011E
:1029B000C301B2010E94B4B265966CAF7DAF8EAF19
:1029C0009FAF65976D962CAD3DAD4EAD5FAD6D97EC
:1029D000A1966CAD7DAD8EAD9FADA1970E94D7B194
:1029E000A50194010E94B4B2A1966CAF7DAF8EAFE9
:1029F0009FAFA19729AD3AAD4BAD5CADCA01B9010E
:102A00000E94D9AD20E030E040E05FE30E94D9AD04
:102A10009B01AC0160E070E080E89FE30E94D7B1C9
:102A20002D966CAF7DAF8EAF9FAF2D9761962CAD7D
:102A30003DAD4EAD5FAD619729873A874B875C8787
:102A40006D968CAD9DADAEADBFAD6D978D879E87FC
:102A5000AF87B88B6091000270910102072E000CC5
:102A6000880B990B0E947AAD20915D0230915E0235
:102A700040915F02509160020E94D9AD2AE037ED8B
:102A800043E25CE30E94D9AD6DA37EA38FA398A718
:102A90000E945C3C9B01AC0128533F4F4F4F5F4F5E
:102AA00061962CAF3DAF4EAF5FAF61974DA45EA472
:102AB0006FA478A841E050E023965FAF4EAF239714
:102AC00059E15DAF23962EAD3FAD23972215330517
:102AD00009F43AC10E94194F0E945C3CDC01CB0111
:102AE00061962CAD3DAD4EAD5FAD6197821B930BF2
:102AF000A40BB50BB7FD10C00E945C3C9B01AC0160
:102B000028533F4F4F4F5F4F61962CAF3DAF4EAFB5
:102B10005FAF61970E94B5943DAD31503DAF332317
:102B200009F441C02D962CAD3DAD4EAD5FAD2D9756
:102B300069A97AA98BA99CA90E94D9AD6B017C01D6
:102B400029AD3AAD4BAD5CADB201C3010E94D9AD28
:102B5000A70196010E94D8B17B018C012D962CAD66
:102B60003DAD4EAD5FAD2D97B201C3010E94D9AD11
:102B70004B015C0129AD3AAD4BAD5CAD69A97AA9B9
:102B80008BA99CA90E94D9AD9B01AC01C501B401E0
:102B90000E94D7B12B013C01C701D80189AB9AAB88
:102BA000ABABBCAB53C023964EAD5FAD2397BA0120
:102BB00080E090E00E9478AD29AD3AAD4BAD5CADC0
:102BC0000E94D9AD4B015C010E94B1B26B017C0146
:102BD000C501B4010E9439B44B015C01A701960103
:102BE0006DA57EA58FA598A90E94D9AD2B013C01AA
:102BF000A50194016DA97EA98FA998AD0E94D9ADB8
:102C00009B01AC01C301B2010E94D8B12B013C0170
:102C1000A50194016DA57EA58FA598A90E94D9ADA7
:102C20004B015C01A70196016DA97EA98FA998AD02
:102C30000E94D9AD9B01AC01C501B4010E94D7B17E
:102C400069AB7AAB8BAB9CAB59E15DAF9201A30151
:102C500029966CAD7DAD8EAD9FAD29970E94D8B100
:102C600069837A838B839C8329A93AA94BA95CA9A0
:102C700069966CAD7DAD8EAD9FAD69970E94D8B160
:102C80006D837E838F83988765962CAD3DAD4EAD69
:102C90005FAD659769857A858B859C850E94D8B1E3
:102CA00069877A878B879C87A1962CAD3DAD4EAD09
:102CB0005FADA1976D857E858F8598890E94D8B17B
:102CC0006D877E878F87988BCE0101960E94B8977B
:102CD000E09018031D8E1E8E1F8E18A289819A8186
:102CE000AB81BC81898B9A8BAB8BBC8B8D819E8198
:102CF000AF81B8858D8B9E8BAF8BB88F89859A8578
:102D0000AB85BC85898F9A8FAB8FBC8FAE01475E38
:102D10005F4FBE016B5E7F4FCE0141960E946D48B2
:102D2000CE014D966C018E010B5D1F4F9E01235FFE
:102D30003F4FAE01475E5F4FBE016B5E7F4F0C970A
:102D40000E94D851811151C0E090180319A21AA213
:102D50001BA21CA28091290D90912A0DA0912B0DF0
:102D6000B0912C0D898B9A8BAB8BBC8B80912D0DE8
:102D700090912E0DA0912F0DB091300D8D8B9E8BCB
:102D8000AF8BB88F8091310D9091320DA091330DA2
:102D9000B091340D898F9A8FAB8FBC8FAE01475E97
:102DA0005F4FBE016B5E7F4FCE0141960E946D4822
:102DB000DE0191966D018E010B5D1F4F25E33DE015
:102DC000AE01475E5F4FBE016B5E7F4FCE01419605
:102DD0000E94D85180E1E9E2FDE0A6E2BEE0019068
:102DE0000D928A95E1F70C94DE282396EEADFFADA7
:102DF000239731962396FFAFEEAF239763CEE8E398
:102E0000F0E284918F010F5F1F4F882321F00E9411
:102E1000D876F801F6CFEDE1F2E084918F010F5FF3
:102E20001F4F882311F40C94DE280E94D876F801F5
:102E3000F4CF80E50E94BC35882329F00E94FE343F
:102E40006B017C0103C0C12CD12C760183E50E946B
:102E5000BC35882361F00E943E3520E030E04AE72F
:102E600054E40E94D9AD0E9421B36B017C010E9401
:102E70005F630E945C3CC60ED71EE81EF91E0E94CE
:102E80005C3CDC01CB018C199D09AE09BF09B7FD83
:102E900002C00C94DE280E94B594F1CF41E061E0BD
:102EA00081E00E94853081110C94DE2880E50E942B
:102EB000BC35882321F00E940E35162F01C010E08A
:102EC00083E50E94BC35882321F00E940E355B010A
:102ED00003C0BCE0AB2EB12C84E50E94BC3581114F
:102EE0000E940E3582E50E94BC35882329F00E949D
:102EF0003E352B013C0106C0412C512CA0ED6A2E21
:102F0000A0E47A2E113011F40C94DE28123009F06E
:102F10008DC03A2C80E090E0A4E3B2E489839A83E8
:102F2000AB83BC8380E090E0ACE2B3E48D839E830E
:102F3000AF83B88780E090E0A0E0BFEB89879A87F5
:102F4000AB87BC87AA2011F40C94DE28198A1A8A50
:102F50001B8A1C8AAE014F5E5F4F6A017C018D01A6
:102F600020E030E04CE253E460E070E084E392E47F
:102F70000E944231F12C00E010E0198A1A8A1B8A63
:102F80001C8AB801012E000C880B990B0E947AADA7
:102F90002CE739ED40E25FE30E94D9AD4B015C01C3
:102FA0000E94B1B2A30192010E94D9AD20E030E0AD
:102FB0004CE253E40E94D8B16D8F7E8F8F8F98A31F
:102FC000C501B4010E9439B4A30192010E94D9AD98
:102FD00020E030E044E352E40E94D8B169A37AA330
:102FE0008BA39CA3AE014F5E5F4FBE01635E7F4F1C
:102FF000CE0181960E9465320F5F1F4F0A30110586
:1030000009F0BBCFF394F31408F4B5CF198A1A8AE8
:103010001B8A1C8AAE014F5E5F4FBE016B5F7F4F04
:10302000CE0101960E9465320C94DE2880E090E08B
:10303000A6EEB2E489839A83AB83BC8340E050E080
:103040006CE273E44D835E836F83788780E090E069
:10305000A0E0BFEB89879A87AB87BC8700E010E0D0
:1030600024E332E4098B1A8B2B8B3C8B4D8B5E8BCC
:103070006F8B788F898F9A8FAB8FBC8F1D8E1E8E32
:103080001F8E18A2CE014D966C01E12CF12C00E0B0
:103090001FEB9A01AB0160E070E084E392E40E94D0
:1030A0004231BB24B594A79410E0812F90E08A159B
:1030B0009B0514F00C94DE281D8E1E8E1F8E18A208
:1030C000AE01435E5F4FBE016B5F7F4FCE01019645
:1030D0000E9465321D8E1E8E1F8E18A2AE01435EA9
:1030E0005F4FBE016B5E7F4FCE0141960E946532FD
:1030F0001F5FDBCF20931F020C94DE2841E061E0CC
:1031000081E00E94853081110C94DE2880E090E0FF
:10311000A0E2B1E489839A83AB83BC838DEC9CEC01
:10312000ACE2B3E48D839E83AF83B88780E090E008
:10313000A0EAB1E489879A87AB87BC8780E50E94C3
:10314000BC35882319F00E940E3501C060E080E094
:1031500090E0A8ECB2E489A39AA3ABA3BCA380E05F
:1031600090E0A0EAB0E48D8F9E8FAF8FB8A361305E
:1031700019F0623039F029C0BE01635E7F4FCE0185
:10318000099644C029853A854B855C8560912E0E51
:1031900070912F0E8091300E9091310E0E94D8B117
:1031A0006B017C0120E030E04FE153E40E9474ADFC
:1031B00087FD06C0C12CD12C3FE1E32E33E4F32E72
:1031C000C98ADA8AEB8AFC8A1CC0A0902E0EB090C5
:1031D0002F0EC090300ED090310EE984FA840B850A
:1031E0001C859501A601B701C8010E94FEB31816FF
:1031F00014F075018601C701D801898B9A8BAB8BBE
:10320000BC8BBE01635E7F4FCE0141960E94863229
:10321000AE014F5D5F4FBE016B5F7F4FCE010196E8
:103220000E9465320C94DE288091F004877087300C
:1032300071F48FE40E94BC35882319F00E942F3569
:1032400003C08FE40E94753581110C94DE280E9422
:103250005F639091620D22969FAF229780E00E945B
:10326000BA340E94233111E01093EF0488E50E94E4
:1032700075358DA789E50E947535382E8AE50E943F
:103280007535082FADA5A11105C0311005C0282E38
:10329000212605C0311002C0212C01C0282E80E15A
:1032A000E6E2FEE0A9E2BDE001900D928A95E1F729
:1032B000211002C0002319F082E00E94D59282E51D
:1032C0000E94BC35882361F00E943E356B017C0171
:1032D00020E030E0A9010E9474AD882381F106C08E
:1032E000C12CD12C20E8E22E20E4F22E211006C0C1
:1032F000BDA5B11103C0332009F414C1C092310D32
:10330000D092320DE092330DF092340D20912E0EBA
:1033100030912F0E4091300E5091310EC701B60101
:103320000E94FEB318165CF419821A821B821C825A
:10333000BE016F5F7F4F81E39DE00E9486322110C6
:103340000EC0EDA5EE2309F403C1311008C080E0E2
:103350000E94D592222011F40C941B2FE0C01092F1
:103360002A0E10922B0E10922C0E10922D0E1092EF
:10337000260E1092270E1092280E1092290E0E94EF
:103380007334EDE8FCE1249126962FAF2697E1E80F
:10339000FCE185909590A590B490E5E8FCE1C5909E
:1033A000D590E590F490A7019601C501B4010E9463
:1033B000FEB318162CF4A5019401C701B60104C090
:1033C000A7019601C501B4010E94B4B22B013C01D2
:1033D000E4E4FCE185919591A591B49189AB9AAB18
:1033E000ABABBCABE0E4FCE1259135914591549148
:1033F0002DAB3EAB4FAB58AF9C01AD016DA97EA983
:103400008FA998AD0E9474AD87FD08C019A93AA98B
:1034100039AF4BA94DAF5CA959AB07C01DA98EA907
:1034200089AF9FA99DAFA8ADA9ABA3019201C3012C
:10343000B2010E94D9AD20E030E040E85FE30E9495
:10344000D8B10E9443B49B01AC01612F79AD8DAD21
:1034500099A90E94D9AD6D8F7E8F8F8F98A3EEE8CA
:10346000FCE1149120E030E040EC5FE3C701B601DD
:103470000E94D9AD6B017C01612F110F770B880B76
:10348000990B0E947AAD9B01AC01C701B6010E9465
:10349000D9AD69837A838B839C8320E030E040EC54
:1034A0005FE3C501B4010E94D9AD6B017C01269692
:1034B000BFAD26976B2FBB0F770B880B990B0E9424
:1034C0007AAD9B01AC01C701B6010E94D9AD698BF1
:1034D0007A8B8B8B9C8BAE01435E5F4FBE016F5F1F
:1034E0007F4FCE0141960E9465320E946237109252
:1034F0002A0E10922B0E10922C0E10922D0E10925E
:10350000260E1092270E1092280E1092290E2110CE
:103510001ECF5DA551110C94182F332019F081E0B6
:103520000E94D5920E9473341091EE041092EF0421
:103530001092EE04C12CD12C90EAE92E90E4F92EE1
:10354000C982DA82EB82FC82211018C00C943B2FD6
:103550003110E5CF0E9473341091EE041092EF0405
:103560001092EE0480E090E0A0EAB0E489839A83B0
:10357000AB83BC83002311F40C94312F80E090E0E6
:10358000ADE1B3E4898B9A8BAB8BBC8BBE016F5FD3
:103590007F4FCE0141960E94863280E090E0A0EA03
:1035A000B0E489839A83AB83BC8321100BC03110B4
:1035B00009C080912A0E90912B0EA0912C0EB091F3
:1035C0002D0E04C080E090E0A1E3B3E4898B9A8BD8
:1035D000AB8BBC8B21100CC0EDA5E11109C0809113
:1035E000260E9091270EA091280EB091290E04C0AE
:1035F00080E090E0A0EAB0E48D8F9E8FAF8FB8A3FB
:10360000AE014F5F5F4FBE016F5E7F4FCE014D96A3
:103610000E9465321093EF041093EE0422968FAD52
:1036200022970E94BA340E940A310E9407410C94EA
:10363000DE2880E00E94BA3413E001E01092090E07
:1036400010920A0E10920B0E10920C0E0093F104C1
:1036500024982C9A149A0E9424671092F104249AB8
:103660002C9814988091620D882351F08091620DFE
:10367000882369F081EB92E00E940B940C94DE2881
:1036800081EE92E00E940B941150C1F6EFCFE8EC6E
:10369000F2E084918F010F5F1F4F882321F00E9479
:1036A000D876F801F6CF82E492E00E940B9483E38F
:1036B00092E00E9485940E942F660C94DE2820934D
:1036C0001D030C94DE280E945D650C94DE280E9488
:1036D00008A90C94DE288091040E9091050E8B3978
:1036E000910509F4DAC10CF09EC08C35910509F4FE
:1036F000D5C20CF04FC08B34910509F454C134F598
:103700008231910509F47AC284F497FF02C00C94C7
:103710009628823091050CF43EC1419711F00C942B
:1037200096280E9476970C94DE288A32910509F437
:1037300036C18934910511F40C94DE284F9711F0AD
:103740000C9496280E94A0450C94DE2881359105A2
:1037500009F42AC27CF48D34910509F488C10CF473
:1037600071C18E34910511F00C9496280E94214469
:103770000C94DE288335910509F43BC20CF435C264
:103780008435910509F43AC28535910509F46BC277
:103790000C9496288137910509F475C114F58B3680
:1037A000910509F4EFC17CF48936910509F46FC1E4
:1037B0000CF0CAC18836910511F00C9496280E942D
:1037C00006440C94DE288E36910509F454C18F36D8
:1037D000910509F454C18D36910511F00C94962889
:1037E00060C18637910509F446C36CF483379105AF
:1037F00009F4E3C20CF4DBC28537910511F40C9493
:10380000DE280C9496288837910509F452C40CF4EC
:1038100083C38937910509F453C48C38910509F4A1
:103820005EC10C9496288F35F1E09F0711F40C943B
:10383000E8250CF04FC0833D910509F4D9C414F577
:103840008B3C910509F4ADC474F4883C910509F4EE
:103850003DC4893C910509F481C48E3B910511F06A
:103860000C9496285AC18D3C910509F4BBC40CF404
:10387000B6C48E3C910511F00C9496280E94E34248
:103880000C94DE288D3241E0940709F4C7C474F427
:103890008D3D910509F4BCC4823E910509F4BBC479
:1038A0008C3D910511F00C949628A5C48F32A1E0AF
:1038B0009A0709F4B9C40CF4B4C48033E1E09E075C
:1038C00011F40C9436258E35914011F40C94B325E7
:1038D0000C949628843F31E0930711F40C945927F7
:1038E0005CF5823951E0950711F40C944C2694F460
:1038F0008039B1E09B0711F40C94432614F00C942A
:1039000046268336914011F00C949628E8E3F0E2C5
:103910000C942C26893A21E0920711F40C94DB26B2
:103920008C3A31E0930709F460C4843A914011F075
:103930000C9496280C945226883F51E0950711F478
:103940000C946B276CF4863FB1E09B0711F40C9448
:103950005C2714F00C945F270E94919F0C94DE2842
:103960008438F3E09F0711F40C94F3273CF483357B
:10397000934011F40C948D270C9496288B3843E0D7
:10398000940711F40C944A28873E934011F40C9448
:1039900083280C9496280E94CB640C94DE280E9405
:1039A0003A450C94DE281091DC04113011F40C948B
:1039B000DE28123059F40E94683C6093D004709362
:1039C000D1048093D2049093D30418C01092D804E9
:1039D0001092D9041092DA041092DB041092D404ED
:1039E0001092D5041092D6041092D7041092D004ED
:1039F0001092D1041092D2041092D30481E08093EB
:103A0000DC040E945C3C6093D8047093D9048093DA
:103A1000DA049093DB04123011F40C94DE288091C8
:103A2000DE049091DF0401969093DF048093DE041E
:103A30001092FB0C1092FC0C1092FD0C1092FE0CDC
:103A40000C94DE288091DC04813011F00C94DE2887
:103A500082E08093DC040E945C3C6093D404709309
:103A6000D5048093D6049093D7040C94DE280E944A
:103A70009B3C0C94DE280E94AC430C94DE280E94F0
:103A800035430C94DE280E940B430C94DE280E94E0
:103A9000E9431092E40C0C94652F0E94BC430C94F3
:103AA000DE288DE690E00E94763681110C94DE28A7
:103AB0008091030583FF02C00C94DE2883E50E94F9
:103AC000BC3526968FAF269781110C94082A82E583
:103AD0000E94BC3581110C94082A0C94DE28809138
:103AE000030583FF02C00C94DE2883E50E94BC35E9
:103AF000882311F40C94DE280E943E350E941CB3EA
:103B00006639710514F066E970E0709305046093FE
:103B100004040E94FE4B0C94DE288091030583FF71
:103B200002C00C94DE2883E50E94BC3526968FAF38
:103B3000269781110C94722B82E50E94BC3581116D
:103B40000C94722B0C94DE2880E50E94BC35811108
:103B500006C083E50E94BC35882361F006C00E9440
:103B60001E3581110C94DE28F4CF0E940E356F3F74
:103B7000710510F06FEF70E070931F0460931E04E6
:103B80000C94DE2880E50E94BC35811106C010929D
:103B90001F0410921E040C94DE280E940E35672B21
:103BA00011F00C94DE28F3CF0E94944C0E946F63B6
:103BB00010921F0410921E0400E010E062E370E017
:103BC00080E090E00E94223C0E94194F0F5F1F4F3F
:103BD0000331110599F762E370E080E090E00E9404
:103BE000223C0E94194F0C94DE2810921C030C9466
:103BF000DE2881E080931C030C94DE2883E50E947C
:103C0000BC358823A1F00E943E3520E030E04AE731
:103C100054E40E94D9AD0E9421B360935402709382
:103C2000550280935602909357020C94DE2888E543
:103C30000E94753581110C94E52C89E50E9475353B
:103C400081110C94E52C8AE50E94753581110C9444
:103C5000E52C85E40E94753581110C94E52C0E94B9
:103C60006F630C94DE2883E50E947535882311F478
:103C70000C94DE280E943E3520E030E04AE754E410
:103C80000E94D9AD0E9421B36093F70C7093F80C99
:103C90008093F90C9093FA0C0C94DE28B4E0CB2EB0
:103CA000B3E0DB2E1BEAE12E1DE0F12E10E0D60181
:103CB0008D916D010E947535882309F46DC0133014
:103CC00009F063C00E943E354B015C0120E030E00A
:103CD00040EA51E40E9474AD87FF4EC0A5019401F3
:103CE0006091B70D7091B80D8091B90D9091BA0D9A
:103CF0000E94B4B22B013C019B01AC0160916F0D9D
:103D00007091700D8091710D9091720D0E94D9ADDE
:103D100060936F0D7093700D8093710D9093720D81
:103D2000A30192016091A70D7091A80D8091A90D3A
:103D30009091AA0D0E94D9AD6093A70D7093A80D24
:103D40008093A90D9093AA0D6091F8067091F906E1
:103D50008091FA069091FB060E9478ADA301920132
:103D60000E94D9AD0E9421B36093F8067093F906C2
:103D70008093FA069093FB068092B70D9092B80D4F
:103D8000A092B90DB092BA0D07C00E943E35F7015E
:103D900060837183828393831F5FF4E0EF0EF11CD5
:103DA000143009F084CF0E94E0900C94DE280E9429
:103DB0005F630E9407410C94DE28EAE4F4E08491FA
:103DC0008F010F5F1F4F882321F00E94D876F801E2
:103DD000F6CF60E08AE394E00E94C34061E083E3B1
:103DE00094E00E94C34061E088E294E00E94C340F6
:103DF00061E088E194E00E94C34060E08FE094E0DD
:103E00000E94C34061E085E094E00E94C34061E00D
:103E10008BEF93E00E94C34061E083EF93E00E9448
:103E2000C34061E085EE93E00E94C34060E087ED0F
:103E300093E00E94C34060E088EC93E00E94C3409E
:103E400060E08AEB93E00E94C34060E084EA93E084
:103E50000E94C34061E083E993E00E94C34060E0B8
:103E60008EE793E00E94C34061E08BE693E00E94FE
:103E7000C3400C94DE280091020E1091030E83E0E3
:103E8000D12C40E08150E9F0D8019C91292F2B7F63
:103E90002134C1F711962C912133A1F7913421F0EF
:103EA000953421F441E002C0DD24D39498012E5FC3
:103EB0003F4F89012F5F3F4FF80190819032C9F346
:103EC000E1CF442369F0EAECFFE184917F012FEF19
:103ED000E21AF20A882321F00E94D876F701F5CF82
:103EE000DD2069F0EDE3F5E084917F013FEFE31A17
:103EF000F30A882321F00E94D876F701F5CFD80184
:103F00008D918D01882319F00E94D876F8CF8AE030
:103F10000E94D8760C94DE2881E08093F1042498E6
:103F20002C9A149AE1E7F5E084918F010F5F1F4FFF
:103F3000882321F00E94D876F801F6CFE9E6F5E073
:103F400084918F010F5F1F4F882321F00E94D87644
:103F5000F801F6CF1E9B03C009EE12E002C00EEE80
:103F600012E0F80181918F01882319F00E94D87620
:103F7000F8CF8AE00E94D876E1E6F5E084918F01DF
:103F80000F5F1F4F882321F00E94D876F801F6CFEB
:103F9000379B03C009EE12E002C00EEE12E0D8011A
:103FA0008D918D01882319F00E94D876F8CF8AE090
:103FB0000E94D876E9E5F5E084918F010F5F1F4FED
:103FC000882321F00E94D876F801F6CF1D9B03C00C
:103FD00009EE12E002C00EEE12E0F80181918F01AD
:103FE000882319F00E94D876F8CF8AE00E94D8760C
:103FF000E1E5F5E084918F010F5F1F4F882321F0E9
:104000000E94D876F801F6CF029B03C009EE12E0B9
:1040100002C00EEE12E0D8018D918D01882319F0B7
:104020000E94D876F8CF8AE00E94D876E9E4F5E0DD
:1040300084918F010F5F1F4F882321F00E94D87653
:10404000F801F6CF1C9B03C009EE12E002C00EEE91
:1040500012E0F80181918F01882319F00E94D8762F
:10406000F8CF8AE00E94D876E1E4F5E084918F01F0
:104070000F5F1F4F882321F00E94D876F801F6CFFA
:10408000019B03C009EE12E002C00EEE12E0D8015F
:104090008D918D01882319F00E94D876F8CF8AE09F
:1040A0000E94D8761092F104249A2C9814980C94BB
:1040B000DE2881E08093EF048093EE040C94DE28E8
:1040C0001092EF041092EE040C94DE2888EC90E03D
:1040D0000E94763681110C94DE2884E40E947535A6
:1040E0008823C1F10E943E3511E020E030E0A901B3
:1040F0000E9474AD811101C010E01093BF0D112317
:1041000049F10E943E35E091FF03B4E0EB9FF001DE
:104110001124E554F24F608371838283938320E0FE
:1041200030E0A9016091BB0D7091BC0D8091BD0D77
:104130009091BE0D0E9474AD81110CC080E090E0A2
:10414000A0E4B0E48093BB0D9093BC0DA093BD0D93
:10415000B093BE0D0E94F3480C94DE28FBE8EF2ECE
:10416000FDE0FF2E04E013E0A4E0DA2ED00EF8010B
:1041700081918F010E947535882351F00E943E3550
:104180000E9421B3D7016D937D938D939C931397D8
:10419000B4E0EB0EF11CD012EACF0E94648F0C94B5
:1041A000DE287BE9E72E7DE0F72E04E013E0E4E073
:1041B000DE2ED00EF80181918F010E947535882383
:1041C00041F00E943E35D7016D937D938D939C9372
:1041D0001397B4E0EB0EF11CD012ECCFEFC70E94A6
:1041E0004C40ECC70E94E23FE9C70E94F441E6C799
:1041F0000E94043FE3C783E50E94BC35882309F48D
:10420000DDC70E940E357093010260930002D6C78D
:104210000E948F3ED3C70E94473ED0C70E94A53D53
:10422000CDC70E94513DCAC785E40E94BC35882392
:1042300021F00E940E357B0102C0E12CF12C83E4B9
:104240000E94BC35882331F00E940E35AC966FAFCA
:10425000AC9704C045E0AC964FAFAC9785E50E94A3
:10426000BC35882319F00E942F3503C085E50E94D4
:104270007535E8968FAFE897F7FC07C0812C912C35
:1042800066E1A62E63E4B62E06C0812C912C5CE874
:10429000A52E52E4B52E83E50E94BC35882321F07B
:1042A0000E943E354B015C01E114F10411F41092BF
:1042B000FF03EDA60E945C3C2B013C015DA557FF6E
:1042C0000DC00CE310E080E090E0A0E0B1E4EC96DB
:1042D0008CAF9DAFAEAFBFAFEC970CC004E110E068
:1042E00020E030E040E551E4EC962CAF3DAF4EAF1E
:1042F0005FAFEC9761E06E0D623068F0E4E2F7E0EA
:1043000084918F010F5F1F4F882309F457C70E94C4
:10431000D876F801F5CFEEE4F7E084917F013FEF26
:10432000E31AF30A882321F00E94D876F701F5CF2B
:104330000E94944C4DA547FF04C08FE78093FE0375
:1043400008C05DA5E52F550FFF0BE350FC4F8FE72D
:104350008083C501B4010E941CB3072E000C880B9A
:10436000990B0E947AAD69AF7DAF22968FAF2297ED
:1043700026969FAF26979801A8EEB3E00E94C8B199
:10438000C458DF4F688379838A839B83CC57D0409E
:10439000DC01CB01840D951DA61DB71DC857DF4F4D
:1043A00088839983AA83BB83C858D04081E08093D7
:1043B0005802E3964CAE5DAE6EAE7FAEE397C0584A
:1043C000DF4F488259826A827B82C058D040AF96C4
:1043D0001FAEAF97CC57DF4F188219821A821B820B
:1043E000C458D0406A961FAE6A9790E462969FAF19
:1043F0006297ACE16E96AFAF6E97B6E4A296BFAF90
:10440000A297A6961FAEA697A7961FAEA797A896A7
:104410001FAEA897A9961FAEA99761961CAE1DAEB8
:104420001EAE1FAE61972D961CAE1DAE1EAE1FAE0A
:104430002D97C12CD12C76012FE730E040E050E0E1
:104440002DAB3EAB4FAB58AF3FE7832E912CA12C49
:10445000B12CE7961CAE1DAE1EAE1FAEE79731E045
:10446000AE963FAFAE9767961FAE1EAE679710E051
:10447000212C312C00E04DA5842F440F990BDC0139
:10448000A350BC4FC457DF4FB983A883CC58D0404A
:10449000880F991F880F991FFC01EF5DFB4FAB96AA
:1044A000FFAFEEAFAB97AC962FADAC97022E000CE2
:1044B000330BAD963FAF2EAFAD9780915802882356
:1044C00009F41CC10E945C3C69AB7AAB8BAB9CAB22
:1044D0008091EC03882309F4F1C00E944E4D3DA564
:1044E00037FF09C0109100042090010430900204AD
:1044F000009103040DC0AB96AEADBFADAB971C9160
:1045000011962C90119712963C90129713960C913D
:10451000212F322D432D502FA6966FADA697A7962B
:104520007FADA797A8968FADA897A9969FADA9979D
:104530000E9474AD87FF0CC0A6961FAFA697A796E2
:104540002FAEA797A8963FAEA897A9960FAFA997A9
:10455000212F322D432D502F6A966FAD6A976296A8
:104560007FAD62976E968FAD6E97A2969FADA29724
:104570000E94FEB3181664F46A961FAF6A9762969B
:104580002FAE62976E963FAE6E97A2960FAFA29730
:10459000AE96BFADAE9729AD3DAD22964FAD2297F9
:1045A00026965FAD2697612F722D832D902FBB230A
:1045B00009F468C00E94FEB318160CF07FC029A948
:1045C0003AA94BA95CA92419350946095709CF56C0
:1045D000DF4F288339834A835B83C159D040DA0196
:1045E000C90188589341A109B109B7FD67C0D50138
:1045F000C4012DA93EA94FA958AD821B930BA40B52
:10460000B50B3DA5B595A7959795879537FF03C041
:104610008093FE0307C0C457DF4FE881F981CC586F
:10462000D0408083CF56DF4F288139814A815B811A
:10463000C159D040E7962CAF3DAF4EAF5FAFE79783
:1046400039ADA6963FAFA6974DADA7964FAFA797AA
:1046500022965FAD2297A8965FAFA89726968FAD5A
:104660002697A9968FAFA99729A93AA94BA95CA922
:10467000E3962CAF3DAF4EAF5FAFE397AE961FAE64
:10468000AE971CC00E9474AD87FF18C089A99AA973
:10469000ABA9BCA9E3962CAD3DAD4EAD5FADE397A4
:1046A000821B930BA40BB50BAC01BD0148585341C1
:1046B0006109710977FD02C00C94112D20E030E0F2
:1046C00040EA51E469AD7DAD22968FAD22972696E2
:1046D0009FAD26970E94D8B19B01AC01612F722D2E
:1046E000832D902F0E94FEB318167CF4E0EBF6E0C9
:1046F00084918F010F5F1F4F811103C00E94944C62
:104700005DC50E94D876F801F3CF89A99AA9ABA913
:10471000BCA9C058DF4F288139814A815B81C058CC
:10472000D040821B930BA40BB50BB7FDBAC00E94FF
:10473000ED508AE00E94D87689A99AA9ABA9BCA9B4
:104740008053984FAF4FBF4FC058DF4F8883998336
:10475000AA83BB83C058D040AF969FADAF9791114D
:104760007BC0CC57DF4F288139814A815B81C45897
:10477000D040612F722D832D902F0E94FEB318160A
:104780000CF04DC020E030E040E050E4612F722D8D
:10479000832D902F0E94D8B1CC57DF4F6883798347
:1047A0008A839B83C458D04029A93AA94BA95CA904
:1047B000C458DF4F88819981AA81BB81CC57D040F2
:1047C000280F391F4A1F5B1FC857DF4F28833983C3
:1047D0004A835B83C858D040EC962CAD3DAD4EADBE
:1047E0005FADEC9769AD7DAD22968FAD2297269691
:1047F0009FAD26970E94D7B19B01AC0191E0AF9687
:104800009FAFAF97612F722D832D902F0E94FEB323
:1048100018160CF446C0AF961FAEAF9742C089A9D8
:104820009AA9ABA9BCA9C857DF4F288139814A8111
:104830005B81C858D040821B930BA40BB50BB7FD0E
:1048400030C03DA53F3F19F04CE756E002C04EE8AE
:1048500056E061EA76E022C020E030E040EA51E430
:1048600069AD7DAD22968FAD229726969FAD269796
:104870000E94D7B19B01AC01612F722D832D902F27
:104880000E9474AD87FF0DC04DA54F3F19F045E460
:1048900056E002C048E556E06CE676E08DA50E9441
:1048A0006D4D89A99AA9ABA9BCA9880F991FAA1F08
:1048B000BB1FE3962CAD3DAD4EAD5FADE397821BC4
:1048C000930BA40BB50B84199509A609B709813878
:1048D0009F44A241B10568F0E7E2F6E084918F01C0
:1048E0000F5F1F4F882309F409CF0E94D876F80183
:1048F000F5CF67964EAD5FAD6797AD968EAD9FAD28
:10490000AD97841795070CF0D8CDEAECF5E08491CB
:104910008F010F5F1F4F882321F00E94D876F80186
:10492000F6CF9DA597FD03C00FEF12E002C008EF80
:1049300012E0B80189EB95E00E94B051B701A601E1
:1049400085EB95E00E9499508AE00E94D876B801E4
:1049500084EA95E00E94B0512D964CAD5DAD6EADF0
:104960007FAD2D9780EA95E00E9499508AE00E94E1
:10497000D876B8018FE895E00E94B05161964CADB1
:104980005DAD6EAD7FAD61978BE895E00E9499506B
:104990008AE00E94D876E896AFADE897AA2309F49A
:1049A0000DC4BDA5B7FF31C0C092520DD092530DBA
:1049B000E092540DF092550D2CEA35EC47E25EE39F
:1049C0002D966CAD7DAD8EAD9FAD2D970E94D9AD6E
:1049D00060934E0D70934F0D8093500D9093510D39
:1049E0002CEA35EC47E25EE361966CAD7DAD8EADB1
:1049F0009FAD61970E94B4B260934A0D70934B0DC6
:104A000080934C0D90934D0DD9C3C0925E0DD09202
:104A10005F0DE092600DF092610D2CEA35EC47E2FB
:104A20005EE32D966CAD7DAD8EAD9FAD2D970E9452
:104A3000D9AD60935A0D70935B0D80935C0D90938C
:104A40005D0D2CEA35EC47E25EE361966CAD7DAD21
:104A50008EAD9FAD61970E94B4B26093560D709376
:104A6000570D8093580D9093590DA8C380E50E946F
:104A70007535882351F00E943E356093520D709336
:104A8000530D8093540D9093550D89E40E94753514
:104A9000882381F00E943E352CEA35EC47E25EE344
:104AA0000E94D9AD60934E0D70934F0D8093500DC1
:104AB0009093510D84E40E947535882381F00E9403
:104AC0003E352CEA35EC47E25EE30E94B4B26093D7
:104AD0004A0D70934B0D80934C0D90934D0DEAEC65
:104AE000FFE184918F010F5F1F4F882321F00E9407
:104AF000D876F801F6CF4091520D5091530D609148
:104B0000540D7091550D8AE697E00E9499502CEA59
:104B100035EC47E25EE360914E0D70914F0D809150
:104B2000500D9091510D0E94B4B2AB01BC0186E6CC
:104B300097E00E9499502CEA35EC47E25EE36091E1
:104B40004A0D70914B0D80914C0D90914D0D0E942E
:104B5000D9ADAB01BC0182E697E00E9499508AE092
:104B60000E94D8762BC383E50E947535811106C05B
:104B700054E0E52E53E0F52E10E00EC010E00E9448
:104B80001E35682F812F0E94BDA21F5F1530B9F717
:104B9000EFCF1F5F143071F0F70181917F010E9408
:104BA00075358823B1F30E941E35682F812F0E942E
:104BB000BDA2EFCF82E40E947535882331F00E94B8
:104BC0001E35682F84E00E94BDA20E94D1A1F6C2CA
:104BD00083E50E94BC358823E1F10E941E358130B7
:104BE00041F08230B1F534E0E32E33E0F32E10E0F3
:104BF00021C044E0E42E43E0F42E10E0D7018D9173
:104C00007D010E94BC35882339F00E941E354FEF8C
:104C1000682F812F0E9468A21F5F143079F782E409
:104C20000E94BC358823A9F00E941E3512C01F5F68
:104C30001430A9F3F70181917F010E94BC358823CC
:104C4000B1F30E941E35482F6FEF812F0E9468A29A
:104C5000EECF0E94D1A1B2C284918F010F5F1F4F8E
:104C6000882321F00E94D876F801F6CFEEE6F7E02F
:104C700084918F010F5F1F4F882309F49FC20E9408
:104C8000D876F801F5CF0E945F6398C281E00E9458
:104C90001F320E94074192C280E00E941F320E9490
:104CA00007418CC283E50E947535882349F00E9434
:104CB0002F35182F811106C080E00E94BA3402C03F
:104CC0001091620D8091260E9091270EA091280ED2
:104CD000B091290E89839A83AB83BC8380912A0E7D
:104CE00090912B0EA0912C0EB0912D0E8D839E8352
:104CF000AF83B88780912E0E90912F0EA091300E29
:104D0000B091310E89879A87AB87BC8786E50E9470
:104D10007535882321F08AEA97E00E9494A8812FB4
:104D20000E94BA34111103C0EAECFFE11CC080916B
:104D3000620D8111F9CFE8E3F0E284918F010F5FFA
:104D40001F4F882321F00E94D876F801F6CFEBE8B8
:104D5000F7E084918F010F5F1F4F882329F30E9492
:104D6000D876F801F6CF84918F010F5F1F4F88230B
:104D700021F00E94D876F801F6CF8091620D811162
:104D800003C060E073E002C06CEF72E08DE797E073
:104D90000E94B0518AE00E94D8764CE050E066E272
:104DA0007EE0CE0101960E94C2B4892B09F406C2AE
:104DB0000E94074103C28AE50E947535882329F1C4
:104DC0008091160390911703892B19F00E943E35AC
:104DD00008C06091090E70910A0E80910B0E90919F
:104DE0000C0E60931104709312048093130490933B
:104DF000140480E090E0A0E8BFE380931504909352
:104E00001604A0931704B093180486E40E94753525
:104E1000882381F10E943E3520E030E040E85FE3E6
:104E20000E94FEB318166CF40E943E3520E030E07C
:104E300040E85FE30E94FEB3181684F00E943E35FE
:104E400011C00E943E3520E030E0A9010E9474ADFF
:104E500087FFEACF60E070E0CB0104C060E070E063
:104E600080E89FE360931504709316048093170401
:104E70009093180483E50E947535882351F00E94B1
:104E80003E35609327027093280280932902909305
:104E90002A028AE50E947535811190C186E40E943C
:104EA000753581118BC183E50E947535811186C1ED
:104EB0003AC70E94BC8182C10E94249E7FC183E5C3
:104EC0000E947535882321F00E942F3591E08927B3
:104ED0000E94AA9973C12093390D0E942B7C1092D5
:104EE000390D882309F46AC1EAECFFE184918F014E
:104EF0000F5F1F4F882321F00E94D876F801F6CF6C
:104F0000E9EAF8E084918F010F5F1F4F882309F4CD
:104F100055C10E94D876F801F5CF8AE50E94BC35CC
:104F2000882309F438C00E943E356B017C0120E0E3
:104F300030E040E050EC0E94FEB387FD13C020E05B
:104F400030E040EA50E4C701B6010E9474AD181683
:104F50004CF0C092360ED092370EE092380EF0929E
:104F6000390E2CC1E8E3F0E284918F010F5F1F4FEF
:104F700081110DC0E6ECF8E084918F010F5F1F4FA7
:104F8000882309F41BC10E94D876F801F5CF0E944E
:104F9000D876F801E9CFEAECFFE184918F010F5F49
:104FA0001F4F882321F00E94D876F801F6CFE7EB57
:104FB000F8E084918F010F5F1F4F882321F00E943A
:104FC000D876F801F6CF4091360E5091370E6091A9
:104FD000380E7091390E84EB98E00E9499508AE067
:104FE0000E94D876EBC08BE40E94BC358823B1F1D7
:104FF0008BE40E94BC358823B1F00E943E356B01E2
:105000007C0120E030E0A9010E94FEB387FD19C0B9
:1050100020E030E040E251E4C701B6010E9474ADE7
:1050200018167CF003C0C12CD12C76010E945F635E
:10503000C092460DD092470DE092480DF092490D76
:10504000BDC0E1EEF8E084918F010F5F1F4F882310
:1050500009F4B4C00E94D876F801F5CFEAECFFE17C
:1050600084918F010F5F1F4F882321F00E94D87613
:10507000F801F6CF4091460D5091470D6091480DD3
:105080007091490D80E099E00E9499508AE00E9459
:10509000D87694C088E50E9475358823F1F00E9487
:1050A0000E358B01072E000C220B330B00933A0DAB
:1050B00010933B0D20933C0D30933D0DDB012FEF02
:1050C00030E00E94BCB420ED37E040E050E00E94A8
:1050D000A2B1B9018EE20E945B3B8AE50E94753560
:1050E000882329F00E940E3581E00E94F0A285E419
:1050F0000E947535882309F461C00E940E3582E054
:105100000E94F0A25BC081E080931F0283E50E94B1
:10511000BC35882339F00E942F3581114FC00E9481
:1051200079984CC083E50E947535F7CF0E9408A995
:1051300045C0F090040E0E945F63FF2029F1EAEC65
:10514000FFE184918F010F5F1F4F882321F00E94A0
:10515000D876F801F6CF84E50E94D8766F2D70E0FE
:1051600080E090E04AE00E94077B80E20E94D876CF
:10517000EDE1F9E084918F010F5F1F4F8823F1F07B
:105180000E94D876F801F6CF10921803EAECFFE1FE
:1051900084918F010F5F1F4F882321F00E94D876E2
:1051A000F801F6CF60E070E08BE099E00E94975143
:1051B0008AE00E94D87602C00E9408A91092E40CEE
:1051C000C257DF4FF881CE58D040FF2309F47DC687
:1051D0000E940D987AC60E94C83589E29DE00E941F
:1051E000B8978091030583FDA5C0C090350DD09080
:1051F000360DE090370DF090380D2091320E309141
:10520000330E4091340E5091350EC701B6010E9405
:1052100074AD882309F48EC060912104709122043A
:10522000809123049091240420912004211129C00D
:105230000E941CB320912F02309130026217730735
:1052400004F5C092320ED092330EE092340EF092FA
:10525000350EEAECFFE184918F010F5F1F4F882329
:1052600021F00E94D876F801F6CFE2E0F2E08491D6
:105270008F010F5F1F4F882321F00E94D876F8011D
:10528000F6CF8090350D9090360DA090370DB090F0
:10529000380D2091320E3091330E4091340E5091E2
:1052A000350EC501B4010E94D7B16B017C0120E02D
:1052B00030E0A9010E94FEB387FF04C0F7FAF09422
:1052C000F7F8F094E091180384E0E89FF0011124CE
:1052D000E55DFD4F2081318142815381C701B601D7
:1052E0000E94D9AD20E030E048E453E40E94FEB3D0
:1052F000181604F58092320E9092330EA092340E5E
:10530000B092350EEAECFFE184918F010F5F1F4FE1
:10531000882321F00E94D876F801F6CFE3EEF1E081
:1053200084918F010F5F1F4F882321F00E94D87650
:10533000F801F6CF6091000270910102072E000C77
:10534000880B990B0E947AAD20915D0230915E022C
:1053500040915F02509160020E94D9AD2AE037ED82
:1053600043E25CE30E94D9AD6D8F7E8F8F8F98A34F
:10537000E09018038091310D9091320DA091330D82
:10538000B091340D40912D0D50912E0D60912F0D47
:105390007091300D0091290D10912A0D20912B0D47
:1053A00030912C0D09831A832B833C83498B5A8BB4
:1053B0006B8B7C8B8DA39EA3AFA3B8A719A61AA64F
:1053C0001BA61CA6AE014B5D5F4FBE016F5E7F4FFB
:1053D000CE0101960E946D48DE0199966D018E0105
:1053E000035E1F4F25E33DE0AE014B5D5F4FBE0105
:1053F0006F5E7F4FCE0101960E94D85180E1E9E2B5
:10540000FDE0A6E2BEE001900D928A95E1F7D6CECE
:105410000E943E350E941CB37093070460930604FB
:1054200080E00E94494C81E08093580219AA1AAA90
:105430001BAA1CAA69961CAE1DAE1EAE1FAE6997B4
:105440001DA62A961FAE2A972CE32E962FAF2E97D5
:105450003CE16A963FAF6A9746E462964FAF629727
:10546000C12CD12C90E8E92E2FEBF22E812C912C1F
:1054700054016091060470910704072E000C880BFC
:10548000990B0E947AAD262E172F082F392E262F22
:10549000372F482F592FB601C7010E9474AD8823BA
:1054A000E9F020912104309122044091230450918D
:1054B0002404622D712F802F932D0E9474AD881FBC
:1054C0008827881F8DA726968FAD2697882351F0B1
:1054D0009DA5992339F08091580270CE2C2C1D2D5A
:1054E0000E2D3F2C0E945C3C6B017C01DC01CB014A
:1054F00069962CAD3DAD4EAD5FAD6997821B930BA8
:10550000A40BB50BB7FD3DC0D701C60188519C4F18
:10551000AF4FBF4F69968CAF9DAFAEAFBFAF69972E
:105520000E94ED50E3E6F3E084913F019FEF691A9A
:10553000790A882321F00E94D876F301F5CF8114EF
:105540009104A104B104B9F0D501C40188519C4F64
:10555000AF4FBF4FBC01CD016C197D098E099F096A
:1055600028EE33E040E050E00E9480B1CA01B9016A
:105570000E946D7B03C08FE30E94D8768AE00E9470
:10558000D8760E94B5940E945C3C6093F30C7093B3
:10559000F40C8093F50C9093F60CA0912104ADAB24
:1055A000B0912204B9AFE0912304EDAFF09124044F
:1055B0002296FFAF22979D01AF01622D712F802FA0
:1055C000932D0E94D7B12B013C0120E030E0A901CE
:1055D0000E94FEB387FF04C077FA709477F8709446
:1055E00020E030E040E251E4C301B20181149104B3
:1055F000A104B10429F40E9474AD87FF07C004C060
:105600000E94FEB3181614F4460157012DA522235B
:1056100009F44CC089A99AA9ABA9BCA9892B8A2BEA
:105620008B2B61F0D701C60129A93AA94BA95CA926
:10563000821B930BA40BB50BB7FD38C02DA939AD58
:105640004DAD22965FAD22972A966FAD2A972E9682
:105650007FAD2E976A968FAD6A9762969FAD6297DF
:105660000E94D7B120E030E040EC5FE30E9474ADCF
:1056700087FD31CFD701C601805A9541AF4FBF4F4B
:1056800089AB9AABABABBCAB9DA92A969FAF2A97CF
:10569000A9AD2E96AFAF2E97BDAD6A96BFAF6A97F4
:1056A0002296EFAD22976296EFAF629780915802F3
:1056B000882309F410CF81149104A104B10429F4C2
:1056C000C22CD12EE02EF32CD4CEF8EECF1AF3E07C
:1056D000DF0AE108F108C818D908EA08FB08F7FE54
:1056E000FACEEECF0E943E350E941CB3663971059A
:1056F0000CF068C170930504609304040E94FE4B93
:1057000081E080935802809118038093FF0319AAC7
:105710001AAA1BAA1CAA69961CAE1DAE1EAE1FAE0D
:1057200069971DA62A961FAE2A972CE32E962FAFB7
:105730002E973CE16A963FAF6A9746E462964FAF78
:105740006297C12CD12C00E8E02E8FEBF82E812C33
:10575000912C54016091040470910504072E000CF3
:10576000880B990B0E947AAD262E172F082F392E01
:10577000262F372F482F592FB601C7010E9474AD2D
:105780008823E1F02091000430910104409102044B
:1057900050910304622D712F802F932D0E9474ADC0
:1057A000881F8827881F8DA726965FAD26975523CB
:1057B00049F0882339F08091580200CD2C2C1D2D02
:1057C0000E2D3F2C0E945C3C6B017C01DC01CB0167
:1057D00069962CAD3DAD4EAD5FAD6997821B930BC5
:1057E000A40BB50BB7FD3DC0D701C60188519C4F36
:1057F000AF4FBF4F69968CAF9DAFAEAFBFAF69974C
:105800000E94ED50E7E6F3E084913F019FEF691AB3
:10581000790A882321F00E94D876F301F5CF81140C
:105820009104A104B104B9F0D501C40188519C4F81
:10583000AF4FBF4FBC01CD016C197D098E099F0987
:1058400028EE33E040E050E00E9480B1CA01B90187
:105850000E946D7B03C08FE30E94D8768AE00E948D
:10586000D8760E94B5940E945C3C6093F30C7093D0
:10587000F40C8093F50C9093F60CA0910004ADAB62
:10588000B0910104B9AFE0910204EDAFF0910304CF
:105890002296FFAF22979D01AF01622D712F802FBD
:1058A000932D0E94D7B12B013C0120E030E0A901EB
:1058B0000E94FEB387FF04C077FA709477F8709463
:1058C00020E030E040EA50E4C301B20181149104C9
:1058D000A104B10429F40E9474AD87FF07C004C07D
:1058E0000E94FEB3181614F4460157012DA5222379
:1058F00009F44CC089A99AA9ABA9BCA9892B8A2B08
:105900008B2B61F0D701C60129A93AA94BA95CA943
:10591000821B930BA40BB50BB7FD38C02DA939AD75
:105920004DAD22965FAD22972A966FAD2A972E969F
:105930007FAD2E976A968FAD6A9762969FAD6297FC
:105940000E94D7B120E030E040EC5FE30E9474ADEC
:1059500087FD31CFD701C601805A9541AF4FBF4F68
:1059600089AB9AABABABBCAB9DA92A969FAF2A97EC
:10597000A9AD2E96AFAF2E97BDAD6A96BFAF6A9711
:105980002296EFAD22976296EFAF62978091580210
:10599000882309F410CF81149104A104B10429F4DF
:1059A000C22CD12EE02EF32CD5CEF8EECF1AF3E098
:1059B000DF0AE108F108C818D908EA08FB08F7FE71
:1059C000FACEEECF66E970E095CE0E945F6388E57F
:1059D0000E947535882331F0179A8091F0048E7FEC
:1059E0008093F00489E50E947535882331F0169A7A
:1059F0008091F0048D7F8093F0048AE50E947535D4
:105A0000882331F0159A8091F0048B7F8093F00405
:105A100085E40E947535882309F4D0CB0E947094E8
:105A2000CDCB67964EAD5FAD6797452B09F43AC174
:105A3000E7964CAC5DAC6EAC7FACE797480E591E58
:105A40006A1E7B1EE7962CAD3DAD4EAD5FADE79770
:105A5000281B390B4A0B5B0BCA01B9012DA93EA9C2
:105A60004FA958AD0E9471B1A30192010E94A2B149
:105A7000D501C401820F931FA41FB51F8431910566
:105A8000A105B105FCF04C015D018C3E9105A1051D
:105A9000B1052CF0FBEE8F2E912CA12CB12C40E8FF
:105AA00084169104A104B104DCF08EEF90E0A0E034
:105AB000B0E088199909AA09BB098DAB9EABAFABC1
:105AC000B8AF12C0E4E18E2E912CA12CB12C24E1B0
:105AD00030E040E050E02DAB3EAB4FAB58AF04C0E0
:105AE0008DAA9EAAAFAAB8AEB501A4018CE197E039
:105AF0000E9470514DA95EA96FA978AD87E197E02A
:105B00000E9470516A964FAD6A9762965FAD629738
:105B10006E966FAD6E97A2967FADA29780E197E0EB
:105B20000E949950A6964FADA697A7965FADA797EE
:105B3000A8966FADA897A9967FADA99789E097E041
:105B40000E94995067964EAD5FAD679743305105FF
:105B50000CF4A8C06DA97EA98FA998AD0E947AAD5A
:105B600020E030E040E850E40E94D9AD6B017C01B8
:105B70006A962FAD6A9762963FAD62976E964FAD6B
:105B80006E97A2965FADA297A6966FADA697A796C1
:105B90007FADA797A8968FADA897A9969FADA99717
:105BA0000E94D7B12BED3FE049E450E40E94D9AD0B
:105BB00020E030E040E05FE30E94D9AD9B01AC0102
:105BC000C701B6010E94B4B26B017C01C301B201EE
:105BD0000E947AAD2FE632E143E85AE30E94D9AD44
:105BE0002B013C01B701A60183E097E00E94995088
:105BF000B301A2018DEF96E00E9499502AE939E99C
:105C000049E15FE3C701B6010E94D9AD6B017C0198
:105C10009B01AC010E94D8B1A30192010E94B4B2D1
:105C20002D966CAF7DAF8EAF9FAF2D97A3019201E4
:105C3000C701B6010E94D9AD20E030E040E05EE34C
:105C40000E94D9AD61966CAF7DAF8EAF9FAF61976B
:105C5000EDEEF6E084913F015FEF651A750A882347
:105C600021F00E94D876F301F5CFB701A60187EEA7
:105C700096E00E9499502D964CAD5DAD6EAD7FAD16
:105C80002D9781EE96E00E94995061964CAD5DADE6
:105C90006EAD7FAD61978BED96E00E9499508AE0E2
:105CA0000E94D8768DA99EA9AFA9B8AD880D991D7F
:105CB000AA1DBB1DEDA5B595A79597958795E7FFFF
:105CC00003C08093FE0307C0C457DF4FE881F9810A
:105CD000CC58D040808367962EAD3FAD67972F5F3D
:105CE0003F4F67963FAF2EAF679739AD6A963FAF8C
:105CF0006A974DAD62964FAF629722965FAD22973D
:105D00006E965FAF6E9726968FAD2697A2968FAF51
:105D1000A29749A85AA86BA87CA891E0AE969FAF1D
:105D2000AE970C945E234091090E50910A0E60913B
:105D30000B0E70910C0E8CE898E00E9499508AE04E
:105D40000E94D8768AE00E94D87620E030E0A9014F
:105D500060911104709112048091130490911404C5
:105D60000E94FEB318160CF056C020E030E0A901E6
:105D70006091150470911604809117049091180495
:105D80000E94FEB318160CF046C0EAE4F8E08491D5
:105D90008F010F5F1F4F882321F00E94D876F801F2
:105DA000F6CF409111045091120460911304709148
:105DB000140480E398E00E9499508AE00E94D8760B
:105DC00040912702509128026091290270912A0285
:105DD00086E198E00E9499508AE00E94D87640912E
:105DE00015045091160460911704709118048CEFFB
:105DF00097E00E9499508AE00E94D876E7ECF7E09D
:105E000084918F010F5F1F4F882309F4D7C90E9427
:105E1000D876F801F5CFEAE6F8E084918F010F5FBC
:105E20001F4F882309F4BDCF0E94D876F801F5CF23
:105E300080E00E94D59231100C948F1A54D51091A5
:105E4000EE041092EF041092EE04C12CD12C80EAE3
:105E5000E82E80E4F82EC982DA82EB82FC820111FE
:105E600020C080912E0E90912F0EA091300EB091F7
:105E7000310E0C94C21A0023A1F380E090E0ADE152
:105E8000B3E4898B9A8BAB8BBC8BBE016F5F7F4F6A
:105E9000CE0141963BD3C982DA82EB82FC820C941C
:105EA000D71A80E090E0ADE1B3E4898B9A8BAB8B9D
:105EB000BC8BBE016F5F7F4FCE01419627D3C98255
:105EC000DA82EB82FC820C94D91ACC56DF4F0FB6E3
:105ED000F894DEBF0FBECDBFDF91CF911F910F9120
:105EE000FF90EF90DF90CF90BF90AF909F908F90FA
:105EF0007F906F905F904F903F902F9008950895FE
:105F000090E0FC013197E231F10508F04EC088279E
:105F1000EE58FF4F8F4F0C94B4B4809180008F7770
:105F200003C0809180008F7D8093800008958091D0
:105F30008000877FF9CF84B58F7702C084B58F7DCD
:105F400084BD08958091B0008F7703C08091B00028
:105F50008F7D8093B0000895809190008F7707C067
:105F6000809190008F7D03C080919000877F809307
:105F7000900008958091A0008F7707C08091A000C5
:105F80008F7D03C08091A000877F8093A00008953B
:105F9000809120018F7707C0809120018F7D03C001
:105FA00080912001877F8093200108953FB7F89466
:105FB0008091230390912403A0912503B09126039F
:105FC00026B5A89B05C02F3F19F00196A11DB11D54
:105FD0003FBFBA2FA92F982F8827820F911DA11D8F
:105FE000B11DBC01CD0142E0660F771F881F991FCC
:105FF0004A95D1F70895CF92DF92EF920F931F93B6
:10600000CF93DF93CDB7DEB760970FB6F894DEBFBE
:106010000FBECDBFE0901803E6E2FEE080859185DB
:10602000A285B38544815581668177810081118184
:106030002281338109831A832B833C834D835E83C2
:106040006F83788789879A87AB87BC871D861E8672
:106050001F86188AAE01475F5F4FBE016B5F7F4F9F
:10606000CE0101960E946D48CE010D966C010DE5A2
:1060700012E022E33EE0AE01475F5F4FBE016B5F7F
:106080007F4F0C970E94D85160960FB6F894DEBFF0
:106090000FBECDBFDF91CF911F910F91EF90DF9099
:1060A000CF900895FF920F931F93CF93DF93FC013E
:1060B00020812B3319F1D091E606D530F8F4F62E75
:1060C000BC01C09134030C2F10E0F0E6CF9FC0015B
:1060D00011248C5F9A4F0E94DAB4F801E250FB4F12
:1060E000F082CF5FC53018F4C093340302C0109221
:1060F0003403DF5FD093E60681E001C080E0DF91EA
:10610000CF911F910F91FF900895EF92FF920F93FF
:106110001F93CF93DF93882329F0D091280DD0953A
:10612000D17001C0D0E0662341F01091280D11FB21
:10613000882780F911E0182701C010E0442341F0BE
:10614000C091280DC2FB882780F9C1E0C82701C093
:10615000C0E0D11102C0112319F0EAECFFE103C045
:10616000C111FBCF4FC084917F019FEFE91AF90A5B
:10617000882321F00E94D876F701F5CFE2EDFAE00E
:1061800084917F019FEFE91AF90A882321F00E9488
:10619000D876F701F5CFDD2369F0E0EDFAE08491E0
:1061A0007F019FEFE91AF90A882321F00E94D8762F
:1061B000F701F5CF112361F0EEECFAE084918F0145
:1061C0000F5F1F4F882321F00E94D876F801F6CF89
:1061D000C11103C0E4ECFAE00BC0ECECFAE08491EE
:1061E000EF0121968823B1F30E94D876FE01F7CF04
:1061F0008491EF012196882321F00E94D876FE0138
:10620000F7CFC1E08C2FDF91CF911F910F91FF90BD
:10621000EF90089580919C0390919D03A0919E031F
:10622000B0919F0380935D0290935E02A0935F0202
:10623000B093600280919A0390919B039093010226
:1062400080930002089580915D0290915E02A0917A
:106250005F02B091600280939C0390939D03A09392
:106260009E03B0939F03809100029091010290934E
:106270009B0380939A0384E690E0909301028093BD
:10628000000208954F925F926F927F928F929F9239
:10629000AF92BF92CF92DF92EF92FF920F931F9334
:1062A000CF93DF93CDB7DEB72C970FB6F894DEBF50
:1062B0000FBECDBF6D837E838F83988729873A87F2
:1062C0004B875C8747015801360180915D029091B0
:1062D0005E02A0915F02B091600289839A83AB83D2
:1062E000BC83D601CD90DD90ED90FC9020E030E0B5
:1062F000A901C701B6010E9474AD811106C0E8E48E
:10630000FCE1C590D590E590F490A50194016091D1
:106310002E0E70912F0E8091300E9091310E0E94B2
:1063200074AD87FF11C0C0925D02D0925E02E09210
:106330005F02F092600280922E0E90922F0EA09239
:10634000300EB092310E57DEF301408051806280F2
:10635000738020E030E0A901C301B2010E9474AD56
:10636000811108C04090590250905A0260905B021F
:1063700070905C0240925D0250925E0260925F02F9
:10638000709260028D819E81AF81B8858093260EC8
:106390009093270EA093280EB093290E89859A8595
:1063A000AB85BC8580932A0E90932B0EA0932C0E68
:1063B000B0932D0E20DEA501940160912E0E7091F8
:1063C0002F0E8091300E9091310E0E94FEB3181660
:1063D0008CF4C0925D02D0925E02E0925F02F09275
:1063E000600280922E0E90922F0EA092300EB092EC
:1063F000310E01DE0E945F6389819A81AB81BC818D
:1064000080935D0290935E02A0935F02B09360025E
:106410002C960FB6F894DEBF0FBECDBFDF91CF91A3
:106420001F910F91FF90EF90DF90CF90BF90AF90B2
:106430009F908F907F906F905F904F900895BF9244
:10644000CF92DF92EF92FF920F931F93CF93DF9340
:1064500000D01F92CDB7DEB79091F104981731F1BB
:10646000B82E81110E940DA66091260E7091270E04
:106470008091280E9091290E20912A0E30912B0E9A
:1064800040912C0E50912D0E19821A821B821C8273
:10649000E0902E0EF0902F0E0091300E1091310EE4
:1064A000FE0131966F01EEDEB092F10480E00F90B4
:1064B0000F900F900F90DF91CF911F910F91FF9050
:1064C000EF90DF90CF90BF900895CF92DF92EF9240
:1064D000FF920F931F936A01E0902E0EF0902F0E03
:1064E0000091300E1091310EFB01208131814281EB
:1064F0005381FC016081718182819381C3DE1F9190
:106500000F91FF90EF90DF90CF900895CF92DF92A0
:10651000EF92FF920F931F936B01FC01E080F180DB
:1065200002811381E6E2FEE02481358146815781B4
:106530006081718182819381A5DE1F910F91FF900F
:10654000EF90DF90CF9008950F931F93CF93DF9339
:1065500094E0899FE00111248E01035F114FFE0139
:10656000EE50FB4FDE01A45EB24F2D913D914D9157
:106570005C9160817181828193810E94D8B1F80120
:106580006083718382839383FE01E455F54F859187
:106590009591A591B491FE01ED5EFD4F80839183AD
:1065A000A283B383FE01E854F54F85919591A5919F
:1065B000B491CA5BDD4F88839983AA83BB83DF9143
:1065C000CF911F910F910895CF92DF92EF92FF929A
:1065D0000F931F93CF93DF938091E606853008F0E9
:1065E00003C10E94F87BAC0197FDFEC0982F20915B
:1065F0003A0E30913B0E8A3019F09D3009F0C2C03E
:10660000109299032115310519F40E94194FE4CF16
:10661000F901E75CFC4F108210923B0E10923A0E8B
:1066200029E333E0E90188812F5F3F4F8032D1F3C6
:106630007E018E3409F081C0209709F47EC064E9A0
:106640007AE0CE010E942BAD11E0892B11F410E00D
:1066500009C06EE470E0CE0104960E94CFB40097AA
:1066600009F07C014AE050E060E070E0C70101966B
:106670000E948CAA6093350370933603809337038E
:1066800090933803C0903C0ED0903D0EE0903E0EAB
:10669000F0903F0E2FEFC21AD20AE20AF20A6C15EE
:1066A0007D058E059F0529F0111103C081EA99E04F
:1066B0002AC06AE270E0CE010E94EFB49C0100970C
:1066C00001F1982F9C1B10E0992339F09150FE01A5
:1066D000E90FF11D80811827F7CF4AE050E060E014
:1066E00070E0C90101960E948CAA012F10E020E001
:1066F00030E0601771078207930779F085E79AE029
:1067000002C08BE49AE0DF91CF911F910F91FF902F
:10671000EF90DF90CF900C94B6A5809135039091C7
:106720003603A0913703B091380380933C0E9093C9
:106730003D0EA0933E0EB0933F0E80911F0281113B
:106740001CC067E470E0CE010E94CFB40097A9F0AE
:106750004AE050E060E070E001960E948CAA64304C
:10676000710558F4E4EDF9E08491EF012196882356
:1067700021F00E94D876FE01F7CF61E089E393E033
:1067800091DC2ACF2F3531050CF026CF9C35C1F492
:106790000E94F87B97FD20CF2091990321111CCFF7
:1067A00020913A0E30913B0EA9014F5F5F4F5093FD
:1067B0003B0E40933A0EF901E75CFC4F80830CCF0F
:1067C0009B3319F481E0809399038091990381119F
:1067D00003CFC901019690933B0E80933A0EF901C5
:1067E000E75CFC4F4083F8CEDF91CF911F910F9172
:1067F000FF90EF90DF90CF900895BF92CF92DF92FD
:10680000EF92FF920F931F93CF93DF93CDB7DEB735
:106810006E970FB6F894DEBF0FBECDBF6091320306
:10682000709133036115710561F14DE150E0CE01C6
:1068300001967C010E941CAD1E8EF7018F010E197E
:106840001F09B190BB2031F19AE0B912F7CF22C0F5
:10685000B70184E999E00E94B05182E20E94D876A3
:106860008AE00E94D876BB2059F10F5F1F4F8091BC
:10687000320390913303080F191F109333030093D1
:10688000320381E02091320330913303232BD9F47A
:1068900080E019C0F701E00FF11F108260E0C7012E
:1068A00001DC882371F3EAECFFE184916F019FEF33
:1068B000C91AD90A882361F20E94D876F601F5CF69
:1068C00000E010E0DACF6E960FB6F894DEBF0FBE90
:1068D000CDBFDF91CF911F910F91FF90EF90DF908F
:1068E000CF90BF9008950F931F93CF93DF93CDB7B1
:1068F000DEB72C970FB6F894DEBF0FBECDBFE6E231
:10690000FEE080859185A285B385448155816681AD
:106910007781008111812281338109831A832B833E
:106920003C834D835E836F83788789879A87AB87A3
:10693000BC87AE01475F5F4FBE016B5F7F4FCE01EB
:1069400001960E946D4822E33EE0AE01475F5F4F33
:10695000BE016B5F7F4FCE0101960E94CE8F2C96B9
:106960000FB6F894DEBF0FBECDBFDF91CF911F9160
:106970000F9108959091620D891791F08093620DA7
:10698000811109C00E947B9789E19EE00E94AD635E
:106990000E94CB9204C086E29EE00E94AD63A3CF2A
:1069A000089580E0E7DFEDE4FEE080E090E0A0E81D
:1069B000BFE380839183A283B383148215821682FE
:1069C00017821086118612861386148615861686FF
:1069D0001786808B918BA28BB38B148A158A168AAB
:1069E000178A108E118E128E138E148E158E168E9F
:1069F000178E80A391A3A2A3B3A308958091160339
:106A000090911703009731F04AE050E060E070E0A9
:106A10000C94B4AB60E070E0CB0108958091160354
:106A200090911703009731F04AE050E060E070E089
:106A30000C948CAA60E070E0CB010895EFDF97FD25
:106A40000AC0ECDF6F3F71058105910509F02CF458
:106A5000E5DF862F089580E008958FEF08958091F7
:106A6000160390911703892B31F0E8DF91E0811133
:106A700003C090E001C091E0892F08950F931F9308
:106A8000CF938091160390911703009711F1FC01A9
:106A90008F01C1912C2F2F7DA9F0C53411F0C5367F
:106AA000B9F7F801108260E070E0809116039091D0
:106AB00017030E9425A9F801C083562F472F382FAE
:106AC000292F0BC060E070E0CF911F910F910C94C3
:106AD00025A950E040E030E020E0652F742F832F9F
:106AE000922FCF911F910F91089581548A3108F010
:106AF00041C0A82FB0E04091FE0D5091FF0D609174
:106B0000000E7091010E04C07695679557954795D4
:106B10008A95D2F740FF2EC0E091070EF091080E43
:106B2000AC51B24F8C918823E9F0E80FF11D8081C0
:106B300090ED980F9A3098F08E3211F481810CC04C
:106B40008D3211F08B3271F4818190ED980F9A3073
:106B500030F08E3239F4828180538A3018F49E2FBF
:106B60008F2F02C090E080E090931603809317036C
:106B700081E0089580E00895B8DF882341F081E046
:106B80002091160330911703232B09F480E0089518
:106B9000AF92BF92CF92DF92EF92FF920F931F932B
:106BA000CF93DF9384E0A82E83E0B82E99E2E92EFC
:106BB0009DE0F92E06E21EE02DE0C22E2EE0D22E40
:106BC000C0E0D0E0F50181915F018FDF882319F1EA
:106BD00055DFFE01E75EFC4F2081211104C02091AA
:106BE0001D03222341F0F80120813181428153812C
:106BF0000E94D8B10AC0C330D10539F0F601208116
:106C00003181428153810E94D7B1F7016083718342
:106C1000828393830AC0F80180819181A281B3812C
:106C2000F70180839183A283B3832196F4E0EF0E72
:106C3000F11C0C5F1F4F84E0C80ED11CC430D1057D
:106C400009F0C0CF86E498DF8823B9F017DF20E091
:106C500030E0A9010E94FEB318167CF40FDF20E09B
:106C600030E040E752E40E94B4B260935D0270935A
:106C70005E0280935F02909360028091030583FD22
:106C80002AC06091350D7091360D8091370D90912D
:106C9000380D2091320E3091330E4091340E5091C8
:106CA000350EE091DD04EE23B1F00E94D7B19B01D7
:106CB000AC016091EA047091EB048091EC04909136
:106CC000ED040E94D8B16093EA047093EB048093C2
:106CD000EC049093ED04DF91CF911F910F91FF9001
:106CE000EF90DF90CF90BF90AF900895EF92FF921A
:106CF0000F931F93CF93DF937C0184E53DDFD82F63
:106D0000882341F19BDEC82F181604F5EAECFFE159
:106D100084918F010F5F1F4F882321F00E94D87646
:106D2000F801F6CF8DE40E94D876B70180E090E0BC
:106D30004AE00E94077B6C2FCC0F770B89E99AE021
:106D40000E9497518AE00E94D87608C08093FF0382
:106D5000D0E004C0809118038093FF038D2FDF9152
:106D6000CF911F910F91FF90EF9008958091310383
:106D70001E9902C0816001C08E7F80933103809193
:106D80003103379902C0806101C08F7E8093310347
:106D9000809131031D9902C0826001C08D7F809374
:106DA000310380913103029902C0806201C08F7D5E
:106DB00080933103809131031C9902C0846001C02B
:106DC0008B7F8093310380913103019902C08064ED
:106DD00001C08F7B80933103909130038091310308
:106DE000981731F097E090932F038093300309C0F8
:106DF00080912F03882329F0815080932F038823CB
:106E000049F08091EF04811108C08091F104811153
:106E100004C0089590932E03F4CF8091D30C80FF8B
:106E200016C09091920C80912E0390FF06C080FFB7
:106E30000EC08091250E816005C084FF08C080913E
:106E4000250E80618093250E80E00E949CA3809196
:106E5000D30C81FF16C09091920C80912E0391FF6C
:106E600006C081FF0EC08091250E826005C085FF9F
:106E700008C08091250E80628093250E81E00E94DB
:106E80009CA38091D30C82FF1CC08091920C82FF46
:106E90000CC08091F1048823A1F080912E0382FF21
:106EA00010C08091250E846007C080912E0386FF5C
:106EB00008C08091250E80648093250E82E00C949A
:106EC0009CA308958091250E882319F01092250E19
:106ED000089586E899E00E9485942F923F924F9200
:106EE0005F926F927F929F92AF92BF92CF92DF920A
:106EF000EF92FF920F931F93CF93DF93CDB7DEB73F
:106F000064970FB6F894DEBF0FBECDBF2A013B01D8
:106F1000902EA12E6901082F10E0F801E357F34EDF
:106F2000E491BB24B3941E160CF4B12CFF24F3940B
:106F300020E030E0A901C301B2010E94FEB318169F
:106F40000CF0F12C000F111F000F111FC8018A5DFA
:106F5000914F1C01FC011082118212821382C3DC4A
:106F6000F1014082518262827382E090180320E036
:106F700030E0A901692D7A2DC6010E9474AD8111FE
:106F800008C0F801E05CF34E85919591A591B4910C
:106F900003C0892D9A2DD601898B9A8BAB8BBC8B24
:106FA00080912E0E90912F0EA091300EB091310E47
:106FB00040912A0E50912B0E60912C0E70912D0E47
:106FC0000091260E1091270E2091280E3091290E47
:106FD00009831A832B833C834D835E836F83788779
:106FE00089879A87AB87BC871D861E861F86188A6D
:106FF000AE01475F5F4FBE016B5F7F4FCE010196D1
:107000000E946D48CE010D966C018E010F5E1F4FE0
:1070100022E33EE0AE01475F5F4FBE016B5F7F4FF3
:107020000C970E94D8510E945F63BF104BDF64969B
:107030000FB6F894DEBF0FBECDBFDF91CF911F9189
:107040000F91FF90EF90DF90CF90BF90AF909F9007
:107050007F906F905F904F903F902F900895809118
:10706000DD04882341F040E150E063E370E08EED01
:1070700094E00C9442B1089581E08093DD04EEED3C
:10708000F4E080E1DF011D928A95E9F7E8DF66E12F
:1070900082E390E00C9463B14F925F926F927F9283
:1070A000AF92BF92CF92DF92EF92FF92CF93DF9396
:1070B000EB01FC0160817181828193812CE3C22EFE
:1070C000D12CE12CF12CA70196010E9480B1B62EA3
:1070D000A72ECA01B901A70196010E9480B16B01D8
:1070E0007C01CA01B90128E130E040E050E00E9493
:1070F00080B12B013C01C9016DE671E00E94A0B492
:1071000061157105D9F0AF92BF92DF92CF925F9275
:107110004F929F938F937F936F9382E799E09F9312
:107120008F93DF93CF930E9445AD8DB79EB70E9698
:107130000FB6F8949EBF0FBE8DBF61C00097C9F017
:10714000AF92BF92DF92CF925F924F929F938F93B5
:1071500082E699E09F938F93DF93CF930E9445AD92
:10716000EDB7FEB73C960FB6F894FEBF0FBEEDBF6D
:1071700046C04114510461047104B9F0AF92BF924A
:10718000DF92CF925F924F9286E599E09F938F9323
:10719000DF93CF930E9445AD8DB79EB70A960FB689
:1071A000F8949EBF0FBE8DBF2AC0C114D104E10464
:1071B000F104A9F0AF92BF92DF92CF928EE499E0F2
:1071C0009F938F93DF93CF930E9445ADEDB7FEB7AA
:1071D00038960FB6F894FEBF0FBEEDBF10C0AF9249
:1071E000BF928AE499E09F938F93DF93CF930E949D
:1071F00045AD0F900F900F900F900F900F90DF9173
:10720000CF91FF90EF90DF90CF90BF90AF907F90A5
:107210006F905F904F9008951F920F920FB60F924C
:1072200011240BB60F922F933F934F935F936F935D
:107230007F938F939F93AF93BF93EF93FF93E091CF
:107240001002F09111021995FF91EF91BF91AF914A
:107250009F918F917F916F915F914F913F912F916E
:107260000F900BBE0F900FBE0F901F9018951F929E
:107270000F920FB60F9211240BB60F922F933F93DC
:107280004F935F936F937F938F939F93AF93BF932E
:10729000EF93FF93E0910E02F0910F021995FF9189
:1072A000EF91BF91AF919F918F917F916F915F917E
:1072B0004F913F912F910F900BBE0F900FBE0F90EB
:1072C0001F9018951F920F920FB60F9211240BB6B4
:1072D0000F922F933F934F935F936F937F938F936F
:1072E0009F93AF93BF93EF93FF93E0910402F091CC
:1072F00005021995FF91EF91BF91AF919F918F91E9
:107300007F916F915F914F913F912F910F900BBEA5
:107310000F900FBE0F901F9018951F920F920FB6EF
:107320000F9211240BB60F922F933F934F935F93BD
:107330006F937F938F939F93AF93BF93EF93FF933D
:10734000E0910202F09103021995FF91EF91BF9134
:10735000AF919F918F917F916F915F914F913F91ED
:107360002F910F900BBE0F900FBE0F901F9018958E
:107370001F920F920FB60F9211240BB60F922F93FC
:107380003F934F935F936F937F938F939F93AF93AD
:10739000BF93EF93FF93E0910C02F0910D021995CA
:1073A000FF91EF91BF91AF919F918F917F916F91DD
:1073B0005F914F913F912F910F900BBE0F900FBE99
:1073C0000F901F9018951F920F920FB60F921124D5
:1073D0000BB60F922F933F934F935F936F937F93CF
:1073E0008F939F93AF93BF93EF93FF93E0910A0224
:1073F000F0910B021995FF91EF91BF91AF919F9181
:107400008F917F916F915F914F913F912F910F904D
:107410000BBE0F900FBE0F901F9018951F920F92EA
:107420000FB60F9211240BB60F922F933F934F93E9
:107430005F936F937F938F939F93AF93BF93EF93DC
:10744000FF93E0910802F09109021995FF91EF91E5
:10745000BF91AF919F918F917F916F915F914F916C
:107460003F912F910F900BBE0F900FBE0F901F906A
:1074700018951F920F920FB60F9211240BB60F9210
:107480002F933F934F935F936F937F938F939F932C
:10749000AF93BF93EF93FF93E0910602F091070241
:1074A0001995FF91EF91BF91AF919F918F917F912E
:1074B0006F915F914F913F912F910F900BBE0F9065
:1074C0000FBE0F901F901895CF93DF93282F30E0B9
:1074D000F901E053F04E8491F901E051FF4DD49150
:1074E000F901E655FF4DC491CC2391F081110E9422
:1074F000802FEC2FF0E0EE0FFF1FE15DF64FA5911E
:10750000B491EC91ED2381E090E021F480E002C0A1
:1075100080E090E0DF91CF9108951F93CF93DF93A8
:10752000282F30E0F901E053F04E8491F901E05149
:10753000FF4DD491F901E655FF4DC491CC23C9F01C
:10754000162F81110E94802FEC2FF0E0EE0FFF1F0D
:10755000EA58FF4DA591B4918FB7F894111105C069
:107560009C91ED2FE095E92302C0EC91ED2BEC937B
:107570008FBFDF91CF911F9108951F920F920FB689
:107580000F9211240BB60F922F933F934F935F935B
:107590006F937F938F939F93AF93BF93EF93FF93DB
:1075A00080912A0390912B03A0912C03B0912D037D
:1075B000892B8A2B8B2B59F180912903E09127038A
:1075C000F091280390818927808380912A039091EC
:1075D0002B03A0912C03B0912D03181619061A063F
:1075E0001B060CF055C080912A0390912B03A091AB
:1075F0002C03B0912D030197A109B10980932A03AF
:1076000090932B03A0932C03B0932D0341C0809142
:107610001202E9E4F9E0E4919FEF90931202E23064
:10762000C9F050F4EE2399F0E13081F590916F00AC
:107630009D7F90936F002AC0E43019F1E0F0E530AF
:1076400029F5909173009D7F909373001FC0109255
:107650006E001CC0909170009D7F9093700091E02F
:107660009093B0009091B100987F94609093B10096
:107670001092B3000BC0909171009D7F90937100A8
:1076800005C0909172009D7F9093720060E045DF8D
:10769000FF91EF91BF91AF919F918F917F916F91EA
:1076A0005F914F913F912F910F900BBE0F900FBEA6
:1076B0000F901F9018951F93CF93DF93182FEB0116
:1076C0000E94C7A4209711F460E004C0CF3FD10509
:1076D00031F461E0812FDF91CF911F911ECFE12F17
:1076E000F0E0E053F04EE4914E2F50E0FA01319774
:1076F000E231F10508F09DC08827EC57FF4F8F4F0E
:107700000C94B4B484B5806884BDC7BD97C084B5FB
:10771000806284BDC8BD92C08091800080688093E3
:107720008000D0938900C093880088C08091800039
:10773000806280938000D0938B00C0938A007EC0CB
:1077400080918000886080938000D0938D00C093EA
:107750008C0074C08091B00080688093B000C093AA
:10776000B3006CC08091B00080628093B000C09381
:10777000B40064C080919000806880939000D093A2
:107780009900C09398005AC08091900080628093C5
:107790009000D0939B00C0939A0050C080919000BD
:1077A000886080939000D0939D00C0939C0046C059
:1077B0008091A00080688093A0008091A0008F7BC2
:1077C0008093A000D093A900C093A80037C08091F7
:1077D000A00080628093A000D093AB00C093AA0069
:1077E0002DC08091A00088608093A000D093AD0050
:1077F000C093AC0023C08091200180688093200159
:10780000D0932901C093280119C080912001806282
:1078100080932001D0932B01C0932A010FC0809147
:107820002001886080932001D0932D01C0932C010A
:1078300005C0C038D1050CF04CCF46CFDF91CF91B9
:107840001F9108958F929F92AF92BF92CF92DF9235
:10785000EF92FF926B017C010E94D62F4B015C01DD
:10786000C114D104E104F104F1F00E94D62FDC012F
:10787000CB0188199909AA09BB09883E9340A10543
:10788000B10570F321E0C21AD108E108F10888EED1
:10789000880E83E0981EA11CB11CC114D104E10420
:1078A000F10419F7DDCFFF90EF90DF90CF90BF90FC
:1078B000AF909F908F9008952FB7F89460911F0319
:1078C0007091200380912103909122032FBF08958E
:1078D0000F931F938091DC04813011F4EDDF08C019
:1078E0006091D4047091D5048091D6049091D7040E
:1078F0000091D8041091D9042091DA043091DB046E
:10790000601B710B820B930B28EE33E040E050E0DC
:107910000E9480B18091D0049091D104A091D204B2
:10792000B091D304BC01CD01620F731F841F951F5A
:107930001F910F910895CF92DF92EF92FF920F93D4
:107940001F938091DC048150823010F080E058C099
:107950001092DC04B1DF6093D4047093D50480935B
:10796000D6049093D7048091E0049091E1040196AD
:107970009093E1048093E004C090FB0CD090FC0C49
:10798000E090FD0CF090FE0CA3DF6093FB0C709375
:10799000FC0C8093FD0C9093FE0C0091E20410917E
:1079A000E3042091E4043091E5040C191D092E092B
:1079B0003F09DC01CB01800F911FA21FB31F8093F1
:1079C000E2049093E304A093E404B093E50480DF21
:1079D0000091E6041091E7042091E8043091E90455
:1079E000061717072807390748F472DF6093E60483
:1079F0007093E7048093E8049093E90430DB81E01E
:107A00001F910F91FF90EF90DF90CF9008951F92FC
:107A10000F920FB60F9211242F933F938F939F9342
:107A2000AF93BF9380911F0390912003A0912103F6
:107A3000B091220330911E0323E0230F2D3720F451
:107A40000196A11DB11D05C026E8230F0296A11DB8
:107A5000B11D20931E0380931F0390932003A093D6
:107A60002103B09322038091230390912403A091DA
:107A70002503B09126030196A11DB11D8093230318
:107A800090932403A0932503B0932603BF91AF9155
:107A90009F918F913F912F910F900FBE0F901F904C
:107AA0001895CF93DF9383E520D8C82F882371F0F2
:107AB0000E943E350E941CB37093300260932F02E7
:107AC00021E0672B09F020E02093200480E50DD809
:107AD000882359F020912F0230913002232B11F08E
:107AE0000E942F35809320042DC0C1112BC0EAECD9
:107AF000FFE18491EF012196882321F00E94D8763E
:107B0000FE01F7CF80912004811103C068E073E08B
:107B100002C06BEE72E08DE79CE00E94B051609174
:107B20002F02709130028CE69CE00E949751E8E6AB
:107B3000FCE08491EF012196882321F00E94D87601
:107B4000FE01F7CFDF91CF910895CF93DF9385E4C6
:107B500013D8811110C080E50E947535882391F0FB
:107B60000E943E3560935E0D70935F0D8093600DB3
:107B70009093610D07C00E941E35882361F3E8E3EE
:107B8000F0E26EC089E40E947535882381F00E947E
:107B90003E352CEA35EC47E25EE30E94D9AD6093B6
:107BA0005A0D70935B0D80935C0D90935D0D84E492
:107BB0000E947535882381F00E943E352CEA35EC11
:107BC00047E25EE30E94B4B26093560D7093570D86
:107BD0008093580D9093590DEAECFFE18491EF01E9
:107BE0002196882321F00E94D876FE01F7CF40919C
:107BF0005E0D50915F0D6091600D7091610D82E599
:107C00009CE00E9499502CEA35EC47E25EE36091DB
:107C10005A0D70915B0D80915C0D90915D0D0E94ED
:107C2000B4B2AB01BC018EE49CE00E9499502CEAF6
:107C300035EC47E25EE36091560D7091570D8091EF
:107C4000580D9091590D0E94D9ADAB01BC018AE449
:107C50009CE00E9499508AE0DF91CF910C94D876F5
:107C60008491EF012196882321F00E94D876FE01AD
:107C7000F7CFE6E5FCE08491EF012196882321F01F
:107C80000E94D876FE01F7CFDF91CF910895CF9271
:107C9000DF92EF92FF92CF93DF9380E50E947535DC
:107CA0008823B1F10E940E356B017C0183E50E94AF
:107CB000BC35882321F00E940E35EB0102C0CFEFC6
:107CC000DFEF9E012F5F3F4F2330310508F5D7FCD2
:107CD0001FC00E945F63CF3F8FEFD80729F0219725
:107CE00069F4C1E0D0E00CC08C2DEEDB31E020E087
:107CF000892B09F030E0C32FD22F02C0C0E0D0E0C2
:107D00008C2DE2DB8C179D0719F00E94B594F8CFFB
:107D1000DF91CF91FF90EF90DF90CF9008950F9378
:107D20001F93CF93DF938DED90E00E947636811103
:107D300066C083E50E94BC358823B9F1C091FF037A
:107D4000D0E00E940E35CC0FDD1FCB5DDD4F798377
:107D500068838091FF0390E0EC01CC0FDD1FCC0F16
:107D6000DD1F8E01055D1D4F880F991FFC01EB5D26
:107D7000FD4F60817181072E000C880B990B0E94CA
:107D80007AAD2AE037ED43E25CE30E94D9ADC85FEB
:107D9000DB4F288139814A815B810E94D9ADF8018E
:107DA00060837183828393832AC0EAECFFE184912C
:107DB000EF012196882321F00E94D876FE01F7CFAB
:107DC00085E40E94D8768091FF03805D0E94D8767A
:107DD000E091FF03F0E0EE0FFF1FEB5DFD4F6081D0
:107DE000718182E49CE00E94975185E20E94D876DE
:107DF0008AE0DF91CF911F910F910C94D876DF919B
:107E0000CF911F910F910895CF93DF93EAECFFE19B
:107E10008491EF012196882321F00E94D876FE01FB
:107E2000F7CF83E50E947535882321F00E942F3516
:107E300080935202E2E3FCE08491EF0121968823D3
:107E400021F00E94D876FE01F7CF80915202811175
:107E500003C0EEE2FCE002C0EAE2FCE08491EF0144
:107E60002196882321F00E94D876FE01F7CFE2E226
:107E7000FCE08491EF012196882321F00E94D876BE
:107E8000FE01F7CF20910D0E30910E0E40910F0E96
:107E90005091100E6091130270911402809115029E
:107EA000909116020E94D8B1AB01BC0180E29CE027
:107EB0000E9499502091110E3091120E4091130E94
:107EC0005091140E6091170270911802809119025E
:107ED00090911A020E94D8B1AB01BC018DE19CE0E7
:107EE0000E9499502091150E3091160E4091170E58
:107EF0005091180E60911B0270911C0280911D021E
:107F000090911E020E94D8B1AB01BC018AE19CE0B5
:107F10000E949950E2E1FCE08491EF0121968823D0
:107F200021F00E94D876FE01F7CF20910D0E3091FE
:107F30000E0E40910F0E5091100E609146027091FE
:107F4000470280914802909149020E94D8B1AB014A
:107F5000BC0180E19CE00E9499502091110E30916B
:107F6000120E4091130E5091140E60914A027091BE
:107F70004B0280914C0290914D020E94D8B1AB010E
:107F8000BC018DE09CE00E9499502091150E30912B
:107F9000160E4091170E5091180E60914E0270917E
:107FA0004F0280915002909151020E94D8B1AB01D2
:107FB000BC018AE09CE00E9499508AE0DF91CF9159
:107FC0000C94D87682E40E947535882351F00E9483
:107FD000FE3460937B0D70937C0D80937D0D9093A8
:107FE0007E0D83E50E947535882351F00E943E3551
:107FF0006093770D7093780D8093790D90937A0D3F
:1080000084E50E947535882351F00E943E356093C7
:10801000730D7093740D8093750D9093760D88E5B4
:108020000E947535882351F00E943E356093630DA0
:108030007093640D8093650D9093660D89E50E94A1
:108040007535882351F00E943E356093670D70931B
:10805000680D8093690D90936A0D8AE50E947535CD
:10806000882351F00E943E3560936B0D70936C0D28
:1080700080936D0D90936E0D85E40E947535882375
:1080800051F00E943E3560936F0D7093700D809398
:10809000710D9093720D0895CF9383E50E94BC35C6
:1080A0008823A1F00E943E356093870D7093880D60
:1080B0008093890D90938A0D60937F0D7093800D4E
:1080C0008093810D9093820DC0E001C0C1E080E5F6
:1080D0000E94BC35882359F00E943E356093870D7D
:1080E0007093880D8093890D90938A0DC0E082E58E
:1080F0000E94BC35882359F00E943E356093830D61
:108100007093840D8093850D9093860DC0E084E577
:108110000E94BC35882359F00E943E3560937F0D44
:108120007093800D8093810D9093820D2AC0CC2393
:1081300041F14091870D5091880D6091890D7091AA
:108140008A0D8AEF9BE00E9499504091830D5091D7
:10815000840D6091850D7091860D87EF9BE00E94E4
:10816000995040917F0D5091800D6091810D7091DB
:10817000820D84EF9BE00E9499508AE0CF910C948D
:10818000D876CF910895EF92FF920F931F93CF93DC
:10819000DF931F92CDB7DEB7082F162FEFEEFBE06F
:1081A00084917F012FEFE21AF20A882331F099833C
:1081B0000E94D876F7019981F3CFE02FF92F8491AF
:1081C0007F019FEFE91AF90A882321F00E94D876EF
:1081D000F701F5CFEDEEFBE084917F012FEFE21A7E
:1081E000F20A882321F00E94D876F701F5CF612F9B
:1081F00070E080E090E00E946D7B8AE00F90DF915C
:10820000CF911F910F91FF90EF900C94D8764F92E1
:108210005F926F927F928F929F92AF92BF92CF9216
:10822000DF92EF92FF92CF93DF93EAEEFBE084912F
:10823000EF012196882321F00E94D876FE01F7CF26
:1082400020910D0E30910E0E40910F0E5091100E98
:108250006091260E7091270E8091280E9091290E24
:108260000E94D8B142E00E94877BE6EEFBE0849159
:10827000EF012196882321F00E94D876FE01F7CFE6
:108280002091110E3091120E4091130E5091140E48
:1082900060912A0E70912B0E80912C0E90912D0ED4
:1082A0000E94D8B142E00E94877BE2EEFBE084911D
:1082B000EF012196882321F00E94D876FE01F7CFA6
:1082C0002091150E3091160E4091170E5091180EF8
:1082D00060912E0E70912F0E8091300E9091310E84
:1082E0000E94D8B142E00E94877BEEEDFBE08491D2
:1082F000EF012196882321F00E94D876FE01F7CF66
:108300006091320E7091330E8091340E9091350E43
:1083100042E00E94877B80916F0081FB992790F952
:1083200081FF05C080916F008D7F80936F0040902A
:10833000D40D5090D50D6090D60D7090D70D8090D3
:10834000D80D9090D90DA090DA0DB090DB0DC090B3
:10835000DC0DD090DD0DE090DE0DF090DF0D992367
:1083600029F080916F00826080936F00E4EDFBE064
:108370008491EF012196882321F00E94D876FE0196
:10838000F7CFC301B2010E946D7BE0EDFBE0849169
:10839000EF012196882321F00E94D876FE01F7CFC5
:1083A000C501B4010E946D7BECECFBE08491EF0110
:1083B0002196882321F00E94D876FE01F7CFC701CD
:1083C000B6010E946D7B8AE0DF91CF91FF90EF9024
:1083D000DF90CF90BF90AF909F908F907F906F90E5
:1083E0005F904F900C94D8762F923F924F925F926D
:1083F0006F927F928F929F92AF92BF92CF92DF92B5
:10840000EF92FF920F931F93CF93DF93CDB7DEB719
:108410002F970FB6F894DEBF0FBECDBF41E061E0ED
:1084200081E00E9485308111B5C094E3892E9CE1E2
:10843000992E86E29EE09E878D87FE0131965F0130
:108440000DE81CE11F01F3E0F00FFF87F4016591D7
:10845000759185919491ED85FE85C190D190E190C3
:10846000F190FE87ED87A70196010E94D7B12B01FD
:108470003C0120E030E040EA51EC0E94FEB387FD71
:1084800010C020E030E040EA51E4C301B2010E9494
:1084900074AD181634F0F101408251826282738209
:1084A0000DC0F80184911816B4F7F7FAF094F7F8B4
:1084B000F094F101C082D182E282F382F101C19095
:1084C000D190E190F1901F0120E030E040EA51ECC2
:1084D000C701B6010E94FEB387FF03C0E8E3F0E2E4
:1084E0000BC020E030E040EA51E4C701B6010E9431
:1084F00074AD1816BCF4F2CF84918F010F5F1F4F3B
:10850000882321F00E94D876F801F6CFE0E9FCE05C
:1085100084918F010F5F1F4F8823E1F10E94D8766D
:10852000F801F6CFF4E08F0E911C0F5F1F4F8F857F
:1085300080138CCF82EFE82E84E0F82E10E0F50156
:1085400081919191A191B1915F01F70181939193F3
:10855000A193B1937F01812F0E94A4321F5F13303A
:1085600071F72F960FB6F894DEBF0FBECDBFDF9127
:10857000CF911F910F91FF90EF90DF90CF90BF9020
:10858000AF909F908F907F906F905F904F903F90B3
:108590002F903DCE2F960FB6F894DEBF0FBECDBF05
:1085A000DF91CF911F910F91FF90EF90DF90CF90CF
:1085B000BF90AF909F908F907F906F905F904F9003
:1085C0003F902F900895EF92FF920F931F93CF93B8
:1085D00084E0E82E83E0F82E02EF14E0C0E0F7011B
:1085E00081917F010E947535882351F00E943E35AC
:1085F000F80160837183828393838C2F0E94A4325D
:10860000CF5F0C5F1F4FC33051F7CF911F910F9178
:10861000FF90EF90FCCDCF93DF9383E50E94BC35B4
:10862000882351F00E941E358D3308F08CE380932F
:108630005302DF91CF910895EAECFFE18491EF01BD
:108640002196882321F00E94D876FE01F7CF409131
:10865000530250E060E070E085EC9BE00E947C50AB
:108660008AE0DF91CF910C94D876DF92EF92FF925F
:108670000F931F93CF93DF9383E50E947535882373
:1086800059F083E50E94BC35882319F00E941E35FD
:1086900001C080E080930305EAECFFE18491EF01E3
:1086A0002196882321F00E94D876FE01F7CFEEEBC9
:1086B000FBE08491EF012196882321F00E94D87677
:1086C000FE01F7CF80910305882389F180EBE82E26
:1086D0008BE0F82E00E010E020E08091030590E0B0
:1086E000002E02C0959587950A94E2F780FF16C088
:1086F000DD24D394D20E222319F08CE20E94D87686
:10870000F70125913491F9018491E901219688239B
:1087100021F00E94D8769E01F6CF2D2D0F5F1F4FBE
:10872000F2E0EF0EF11C05301105B9F60BC0EAEBD3
:10873000FBE08491EF012196882321F00E94D876F6
:10874000FE01F7CF8AE0DF91CF911F910F91FF904B
:10875000EF90DF900C94D8768EE40E94BC3588238D
:1087600051F00E940E3560933C0E70933D0E809345
:108770003E0E90933F0E0895CF92DF92EF92FF92BC
:10878000CF9383E50E94BC358823E9F00E941E3513
:10879000C82F8D3308F0CCE3C0931B0D8DD86B012F
:1087A0007C012C2F30E0A8EEB3E00E94C8B1C60EC9
:1087B000D71EE81EF91EC092170DD092180DE09238
:1087C000190DF0921A0DCF91FF90EF90DF90CF909E
:1087D0000895CF93DF9389E690E00E947636811169
:1087E00012C0EDEAFBE08491EF012196882321F08D
:1087F0000E94D876FE01F7CF0E94ED508AE0DF910B
:10880000CF910C94D876DF91CF91089588E690E0CF
:108810000E947636811114C08091030583FD10C03B
:1088200083E50E94BC35882359F00E943E350E94A2
:108830001CB3709307046093060480E00C94494CC9
:108840000895EF92FF920F931F93CF93DF93CDB7CD
:10885000DEB769970FB6F894DEBF0FBECDBF83E5D4
:108860000E94BC35811103C0E5EAFBE008C00E940C
:108870000E356E347105C1F70E943C38EEC084910C
:108880008F010F5F1F4F882321F00E94D876F801D7
:10889000F6CFECE9FBE084918F010F5F1F4F882337
:1088A00021F00E94D876F801F6CF6091DE04709135
:1088B000DF0480E090E04AE00E94077BEFE8FBE005
:1088C00084918F010F5F1F4F882321F00E94D8767B
:1088D000F801F6CF6091E0047091E10480E090E04F
:1088E0004AE00E94077BE4E8FBE084918F010F5F80
:1088F0001F4F882321F00E94D876F801F6CF6091AF
:10890000DE047091DF048091E0049091E104681B23
:10891000790B8091DC04815021E030E0823010F04E
:1089200020E030E0621B730B80E090E04AE00E94A0
:10893000077B8AE00E94D876ECE7FBE084918F0108
:108940000F5F1F4F882321F00E94D876F801F6CFE1
:108950008091E2049091E304A091E404B091E504D5
:108960008E8B9F8BA88FB98FBE016F5F7F4FCE011B
:1089700046960E944C38EFE6FBE084918F010F5F32
:108980001F4F811105C0CE0101967C018C0104C0EE
:108990000E94D876F801F1CFF80181918F018823E8
:1089A00019F00E94D876F8CF8091E6049091E70400
:1089B000A091E804B091E9048E8B9F8BA88FB98FAA
:1089C000BE016F5F7F4FCE0146960E944C38EFE5A7
:1089D000FBE084918F010F5F1F4F882321F00E94DD
:1089E000D876F801F6CFF70181917F01882319F03D
:1089F0000E94D876F8CF8AE00E94D876E7E5FBE0BF
:108A000084918F010F5F1F4F882321F00E94D87639
:108A1000F801F6CFE7E4FBE084918F010F5F1F4F71
:108A2000882321F00E94D876F801F6CF20E030E0CC
:108A30004AE754E46091EA047091EB048091EC04FD
:108A40009091ED040E94B4B242E00E94877B8DE6D3
:108A50000E94D8768AE00E94D87669960FB6F8947C
:108A6000DEBF0FBECDBFDF91CF911F910F91FF9061
:108A7000EF9008950F931F93CF9383E50E94BC3529
:108A8000882309F459C00E941E35082F80E50E94F2
:108A9000BC35811110C081E0011101C080E08093DC
:108AA000F104882321F024982C9A149A45C0249A22
:108AB0002C98149841C080E50E94BC35882331F081
:108AC0000E941E35C82F87FF02C036C0CDE0EBE004
:108AD000FBE08DE28E0F9491C91721F031968E1331
:108AE000FACF18C0E8E3F0E284918F010F5F1F4FC7
:108AF000882321F00E94D876F801F6CFE8E3FBE066
:108B000084918F010F5F1F4F8823B1F00E94D876A8
:108B1000F801F6CF8C2F0E94C7A4602F8C2F0E94E3
:108B20008D3A10E0B8018C2F0E945B3BC83021F4D5
:108B300010931F0400931E04CF911F910F9108956D
:108B40000F931F93CF93DF93CDB7DEB769970FB61F
:108B5000F894DEBF0FBECDBF0E94683C6E8B7F8B4A
:108B6000888F998FBE016F5F7F4FCE0146960E941E
:108B70004C38EAECFFE184918F010F5F1F4F88238F
:108B800021F00E94D876F801F6CFBE016F5F7F4FCB
:108B90008EEF9AE00E94B0518AE00E94D8766996E2
:108BA0000FB6F894DEBF0FBECDBFDF91CF911F91FE
:108BB0000F9108954F925F926F927F928F929F9242
:108BC000AF92BF92CF92DF92EF92FF92CF93DF935B
:108BD000CDB7DEB72C970FB6F894DEBF0FBECDBF72
:108BE0008091000490910104A0910204B0910304CB
:108BF00089839A83AB83BC836091040470910504DC
:108C0000072E000C880B990B0E947AAD29813A81BE
:108C10004B815C810E94D7B16B017C016093CE03D4
:108C20007093CF038093D0039093D1032091520D82
:108C30003091530D4091540D5091550D0E94D9AD76
:108C40006D837E838F8398876093CA037093CB0371
:108C50008093CC039093CD032091C6033091C7033A
:108C60004091C8035091C903C701B6010E94D8B111
:108C70004B015C016093C6037093C7038093C803E4
:108C80009093C90320914E0D30914F0D4091500D9E
:108C90005091510D0E94D9AD69877A878B879C8747
:108CA0006093C2037093C3038093C4039093C5037E
:108CB00020ED3CEC4CE45DE360914A0D70914B0D6E
:108CC00080914C0D90914D0D0E94D9AD2B013C012E
:108CD0002091BE033091BF034091C0035091C10366
:108CE00069817A818B819C810E94D7B19B01AC0103
:108CF000C301B2010E94D9AD2B013C0123E333E350
:108D000043E75FE36091BA037091BB038091BC03BA
:108D10009091BD030E94D9AD9B01AC01C301B2018A
:108D20000E94D8B12B013C016093BA037093BB033E
:108D30008093BC039093BD0389819A81AB81BC81F0
:108D40008093BE039093BF03A093C003B093C1036D
:108D500029853A854B855C856D817E818F819885DB
:108D60000E94D8B1A30192010E94D7B12B013C010E
:108D700020E030E04FE753E40E94FEB320E030E013
:108D8000A9011816ACF4C701B6010E94FEB318166B
:108D90006CF5A7019601C501B4010E94D7B160939B
:108DA000C6037093C7038093C8039093C9031EC082
:108DB000C301B2010E9474AD87FF22C020E030E001
:108DC000A901C701B6010E9474AD87FF16C0A701B3
:108DD0009601C501B4010E94D7B16093C603709398
:108DE000C7038093C8039093C90307C0412C512C3B
:108DF0008FE7682E83E4782E03C0412C512C32017A
:108E0000C301B2012C960FB6F894DEBF0FBECDBFE2
:108E1000DF91CF91FF90EF90DF90CF90BF90AF9018
:108E20009F908F907F906F905F904F9008952F92BA
:108E30003F924F925F926F927F928F929F92AF92EA
:108E4000BF92CF92DF92EF92FF92CF93DF9300D049
:108E50001F92CDB7DEB76090060470900704809033
:108E6000210490902204A0902304B0902404B30124
:108E7000072C000C880B990B0E947AADA501940178
:108E80000E94D7B16B017C016093B6037093B70366
:108E90008093B8039093B90320ED3CEC4CE45DE380
:108EA0006091560D7091570D8091580D9091590D0C
:108EB0000E94D9AD1B012C012091B2033091B30364
:108EC0004091B4035091B503C501B4010E94D7B1DC
:108ED0009B01AC01C201B1010E94D9AD1B012C0163
:108EE00023E333E343E75FE36091AE037091AF03A5
:108EF0008091B0039091B1030E94D9AD9B01AC0168
:108F0000C201B1010E94D8B169837A838B839C83AB
:108F10006093AE037093AF038093B0039093B1035B
:108F20008092B2039092B303A092B403B092B503BF
:108F300020E030E040E251E4C701B6010E94FEB3F8
:108F4000181624F481E08093AD0389C020E030E05E
:108F500040E251ECC701B6010E9474AD87FD02C02A
:108F6000672821F481E08093AD039DC08091AD031B
:108F7000882351F01092A9031092AA031092AB0318
:108F80001092AC031092AD0320915E0D30915F0DF5
:108F90004091600D5091610DC701B6010E94D9AD9D
:108FA0002B013C016093A5037093A6038093A70354
:108FB0009093A8032091A9033091AA034091AB0399
:108FC0005091AC03C701B6010E94D8B14B015C01BE
:108FD0006093A9037093AA038093AB039093AC03AF
:108FE00020915A0D30915B0D40915C0D50915D0DBB
:108FF0000E94D9AD9B01AC016093A1037093A203C1
:109000008093A3039093A403C301B2010E94D8B13B
:1090100029813A814B815C810E94D7B12B013C01AF
:1090200020E030E04FE753E40E94FEB320E030E060
:10903000A9011816DCF4C701B6010E94FEB3181688
:1090400074F4A7019601C501B4010E94D7B16093E1
:10905000A9037093AA038093AB039093AC03412CB4
:10906000512C8FE7682E83E4782E20C0C301B20113
:109070000E9474AD87FF1AC020E030E0A901C7014B
:10908000B6010E9474AD87FF0EC0A7019601C5010D
:10909000B4010E94D7B16093A9037093AA0380938F
:1090A000AB039093AC03412C512C3201C301B201AC
:1090B0000F900F900F900F90DF91CF91FF90EF9056
:1090C000DF90CF90BF90AF909F908F907F906F90E8
:1090D0005F904F903F902F900895CF92DF92EF9244
:1090E000FF920F931F93CF93DF93CDB7DEB72897EF
:1090F0000FB6F894DEBF0FBECDBF2091620D2223C4
:1091000009F462C0C52ED42E8B017C0120E030E032
:1091100040E450E4FC0160817181828193810E946E
:10912000D8B16D837E838F8398872DEC3CEC46E32A
:1091300053E4F80160817181828193810E94D7B1EB
:1091400069837A838B839C83CF92DF92CE010196D1
:109150009F938F9304969F938F938DB79EB7849719
:109160000FB6F8949EBF0FBE8DBFADB7BEB71196B8
:1091700084E2EDE4FEE001900D928A95E1F70E9411
:10918000519120E030E040E450E46D817E818F8198
:1091900098850E94D7B1F70160837183828393839E
:1091A0002DEC3CEC46E353E469817A818B819C8110
:1091B0000E94D8B1F80160837183828393830FB6D4
:1091C000F894DEBF0FBECDBF28960FB6F894DEBF71
:1091D0000FBECDBFDF91CF911F910F91FF90EF9008
:1091E000DF90CF900895CF92DF92EF92FF9280911F
:1091F000BF0D882371F1C090BB0DD090BC0DE090E5
:10920000BD0DF090BE0D20E030E0A901C701B60110
:109210000E9474AD8823E9F020E030E040E05FE395
:10922000C701B6010E94D9AD9B01AC010E94D9AD26
:109230002BED3FE049E450E40E94D9AD9B01AC0125
:1092400060E070E080E89FE30E94B4B26B017C01B3
:1092500006C0C12CD12C80E8E82E8FE3F82EC092F6
:109260000804D0920904E0920A04F0920B04609181
:10927000250270912602072E000C880B990B0E9484
:109280007AAD2AE037ED43E25CE30E94D9ADA70155
:1092900096010E94D9AD60932B0270932C028093AB
:1092A0002D0290932E02FF90EF90DF90CF900895C3
:1092B0004F925F926F927F928F929F92AF92BF92E6
:1092C000CF92DF92EF92FF920F931F93CF93DF9392
:1092D000CDB7DEB768970FB6F894DEBF0FBECDBF2F
:1092E0008C015B014A01FC01EE5BFF4F60817181E3
:1092F000828193810E9478AD6B017C01D5012D9113
:109300003D914D915C910E94D9AD0E949EB20E9408
:1093100021B369877A878B879C87F401208131810B
:1093200042815381C701B6010E94D9AD0E949EB20D
:109330000E9421B36D877E878F87988B29853A8518
:109340004B855C85283731054105510540F488E798
:1093500090E0A0E0B0E089879A87AB87BC872D8535
:109360003E854F855889283731054105510540F420
:1093700088E790E0A0E0B0E08D879E87AF87B88B4C
:109380009801225B3F4FD9018D919D910D90BC9129
:10939000A02D89839A83AB83BC83BC01CD010E943D
:1093A0007AAD2B013C0169857A858B859C850E946D
:1093B00078AD698B7A8B8B8B9C8B20E030E0A90198
:1093C000C301B2010E9474AD882329F1A70196015F
:1093D000C701B6010E94D9AD4B015C0129893A89C8
:1093E0004B895C89CA01B9010E94D9AD9B01AC01CE
:1093F000C501B4010E94D7B14B015C01A3019201E8
:10940000C301B2010E94D8B19B01AC01C501B401F6
:109410000E94B4B203C060E070E0CB010E949EB233
:109420000E9421B36D837E838F83988769817A81BF
:109430008B819C8190958095709561957F4F8F4F22
:109440009F4F0E947AAD4B015C016D857E858F85B3
:1094500098890E9478AD69837A838B839C8320E00E
:1094600030E0A901C501B4010E9474AD882349F11F
:1094700029813A814B815C81CA01B9010E94D9AD31
:109480006D8B7E8B8F8B988FA7019601C701B601DC
:109490000E94D9AD9B01AC016D897E898F89988D21
:1094A0000E94D7B16B017C01A5019401C501B401F3
:1094B0000E94D8B19B01AC01C701B6010E94B4B2B1
:1094C00003C060E070E0CB010E944DB3F80185A0BD
:1094D00096A0A7A0B0A4750164012D813E814F81A3
:1094E0005885C21AD30AE40AF50A0E9421B3C61AA3
:1094F000D70AE80AF90AF7FE73C020E030E0A901B4
:10950000C301B2010E9474AD882309F443C0A301D2
:109510009201C301B2010E94D8B16B017C01C50167
:10952000B4010E9478AD9B01AC01C701B6010E9455
:10953000D9AD6B017C0129893A894B895C89CA01C3
:10954000B9010E94D9AD9B01AC01C701B6010E94CF
:10955000D7B16B017C0129813A814B815C81CA01C1
:10956000B9010E94D9AD9B01AC01C701B6010E94AF
:10957000D8B16B017C0120E030E040E850E4C30149
:10958000B2010E94D9AD9B01AC01C701B6010E9496
:10959000B4B203C060E070E0CB010E949EB27B01D8
:1095A0006C0120E030E0A9010E94FEB3181624F0FF
:1095B000E12CF12CC12CD12CB701C6010E9421B3A2
:1095C0006D837E838F83988786169706A806B906D3
:1095D00020F48D829E82AF82B886C12CD12C760178
:1095E0008D819E81AF81B885F80182A793A7A4A73A
:1095F000B5A7C80ED91EEA1EFB1EC6A6D7A6E0AAAE
:10960000F1AAEA5BFF4F29853A854B855C8520836B
:1096100031834283538334968D859E85AF85B88987
:1096200080839183A283B38368960FB6F894DEBFDC
:109630000FBECDBFDF91CF911F910F91FF90EF90A3
:10964000DF90CF90BF90AF909F908F907F906F9062
:109650005F904F9008954F925F926F927F928F929A
:109660009F92AF92BF92CF92DF92EF92FF920F93B1
:109670001F93CF93DF933C01B0E2A0E06A2F70E02C
:10968000AB014B0F511D559547954A1711F04B13E0
:109690000BC0ECE2FDE065917491072E000C880B85
:1096A000990B0E947AAD62C0CA010197880F991F79
:1096B000880F991FFC01E255F34F059114919A010F
:1096C000220F331F220F331FF901E255F34FC591CB
:1096D000D4916016710614F4B42FD2CFA42FC615FE
:1096E000D7050CF4CBCF8055934FFC01E590F49057
:1096F000F901E055F34FC590D490B7010F2C000C41
:10970000880B990B0E947AAD4B015C01B301601B81
:10971000710B072E000C880B990B0E947AAD2B0160
:109720003C01B6016E197F09072E000C880B990BBE
:109730000E947AAD9B01AC01C301B2010E94D9AD78
:109740006B017C01C01BD10BBE01DD0F880B990B97
:109750000E947AAD9B01AC01C701B6010E94B4B270
:109760009B01AC01C501B4010E94D8B1DF91CF913A
:109770001F910F91FF90EF90DF90CF90BF90AF902F
:109780009F908F907F906F905F904F9008950F9370
:109790000FB70F9300916E000B7F00936E007894CB
:1097A0000F930BB70F930CB70F921F922F933F930A
:1097B0004F935F936F937F938F939F93AF93BF93D9
:1097C000EF93FF93112409D2FF91EF91BF91AF91D5
:1097D0009F918F917F916F915F914F913F912F91C9
:1097E0001F900F900CBF0F910BBF0F910460F89466
:1097F00000936E000F910FBF0F911895CF92DF92DB
:10980000EF92FF92C0900004D0900104E090020417
:10981000F090030480910404909105040897BC0122
:10982000990F880B990B0E947AAD9B01AC01C7017F
:10983000B6010E9474AD87FF1FC020E030E040E019
:1098400050E4C701B6010E94D8B10E9421B37093C1
:10985000E7036093E6030E945C3CDC01CB01805A85
:109860009541AF4FBF4F8093E2039093E303A093E2
:10987000E403B093E50308C01092E2031092E303FF
:109880001092E4031092E503FF90EF90DF90CF90E9
:109890000895CF92DF92EF92FF92C0902104D09072
:1098A0002204E0902304F090240480910604909117
:1098B00007040D97BC01990F880B990B0E947AAD94
:1098C0009B01AC01C701B6010E9474AD87FF1FC0A8
:1098D00020E030E040E050E4C701B6010E94D8B17A
:1098E0000E9421B37093E1036093E0030E945C3C0B
:1098F000DC01CB01805E914BAF4FBF4F8093DC0307
:109900009093DD03A093DE03B093DF0308C01092B1
:10991000DC031092DD031092DE031092DF03FF9050
:10992000EF90DF90CF9008951092070410920604F4
:1099300080E0AFDF10920504109204045FDF0E9404
:109940009B3C109207041092060480E0A2DF109264
:10995000FD03759810920504109204041092FE0302
:10996000A59808954F925F926F927F928F929F92E7
:10997000AF92BF92CF92DF92EF92FF920F931F931D
:10998000CF93DF933C01BAE3A0E06A2F70E0AB0114
:109990004B0F511D559547954A1711F04B130BC0AE
:1099A000E3E8FEE065917491072E000C880B990B9B
:1099B0000E947AAD62C0CA010197880F991F880F73
:1099C000991FFC01E356F24F059114919A01220F61
:1099D000331F220F331FF901E356F24FC591D49183
:1099E0006016710614F4B42FD2CFA42FC615D70574
:1099F0000CF4CBCF8156924FFC01E590F490F90125
:109A0000E156F24FC590D490B7010F2C000C880B93
:109A1000990B0E947AAD4B015C01B301601B710B85
:109A2000072E000C880B990B0E947AAD2B013C018C
:109A3000B6016E197F09072E000C880B990B0E9446
:109A40007AAD9B01AC01C301B2010E94D9AD6B019B
:109A50007C01C01BD10BBE01DD0F880B990B0E944E
:109A60007AAD9B01AC01C701B6010E94B4B29B0163
:109A7000AC01C501B4010E94D8B1DF91CF911F9113
:109A80000F91FF90EF90DF90CF90BF90AF909F909D
:109A90008F907F906F905F904F90089560E08091DD
:109AA000EA039091EB03D7DD6093210470932204C5
:109AB00080932304909324048091E8039091E90318
:109AC00051DF60930004709301048093020490932B
:109AD0000304A8951092EC030895CF92DF92FF92B1
:109AE0000F931F93CF93DF931F921F92CDB7DEB7D3
:109AF000F82E8A0180911F02882309F444C0E8E30C
:109B0000F0E284916F019FEFC91AD90A882341F0CE
:109B100069837A830E94D876F60169817A81F1CFD0
:109B2000FB0184916F019FEFC91AD90A882321F0A4
:109B30000E94D876F601F5CFE3E3FDE084916F0152
:109B40009FEFC91AD90A882321F00E94D876F6011E
:109B5000F5CFF7FC0BC06F2DFF0C770B880B990B23
:109B60000E946D7B8AE00E94D8760DC0EEE2FDE097
:109B700084916F019FEFC91AD90A882321F00E94AE
:109B8000D876F601F5CF8091A003811108C010921C
:109B90001F0281E08093A003C8010E9485940F906A
:109BA0000F90DF91CF911F910F91FF90DF90CF9099
:109BB000BBCE8F3F19F048EB5EE002C048EC5EE0A0
:109BC00069ED7EE08ACF8F3F19F045E85EE002C084
:109BD00045E95EE066EA7EE080CF0F931F93CF9366
:109BE000DF93809124028F3790F08F579091FD037F
:109BF0009093FC03992311F0759A01C07598909188
:109C0000FE039093FB03992359F0A59A0AC0909103
:109C1000FC03891708F075989091FB03891708F0E9
:109C2000A5988F5F809324029091FA0381E08927A1
:109C30008093FA0380912302853018F4C1E0C80FA5
:109C400001C0C0E0823009F4ACC048F48823F9F0C8
:109C5000813009F0DAC010927B0080E4B8C0843013
:109C600009F4BDC008F4B0C0853009F0CEC09091B1
:109C7000F903911102C08093F9038091F903815097
:109C80008093F903882309F4C0C0C5E0BEC0809169
:109C900022028F5F80311CF480932202B6C01092A2
:109CA00022028091EC03811113C08091EF03909107
:109CB000F0039093EB038093EA038091ED0390917E
:109CC000EE039093E9038093E80381E08093EC0333
:109CD0008AE0EFEEF3E0DF011D928A95E9F710923A
:109CE000EE031092ED030091EA031091EB0311953E
:109CF00001951109D1E08091FD03811101C0D0E0EF
:109D00008091CC049091CD04919581959109801713
:109D1000910744F4DD2331F045E85EE066EA7EE039
:109D200080E0DBDE80913302909134029195819541
:109D300091090817190744F4DD2331F048EB5EE080
:109D400069ED7EE080E0C9DE11E08091FE038111C3
:109D500001C010E02091E8033091E9038091CA042A
:109D60009091CB048217930744F0112331F045E919
:109D70005EE066EA7EE08FEFB0DE20913102309146
:109D800032028091E8039091E90382179307ECF186
:109D90001123D9F148EC5EE069ED7EE08FEF9DDEA6
:109DA00034C080917A0086FD2DC08091780090911A
:109DB00079002091EF033091F003820F931F90936D
:109DC000F0038093EF0321C010927B0082E4809324
:109DD0007C0080917A00806480937A0016C0809124
:109DE0007A0086FD11C080917800909179002091D1
:109DF000ED033091EE03820F931F9093EE03809357
:109E0000ED0303C0C2E001C0C4E0C09323020E947E
:109E1000B6368091C10D9091C20D009729F001973F
:109E20009093C20D8093C10DDF91CF911F910F913F
:109E300008958F929F92AF92BF92CF92DF92EF924E
:109E4000FF920F93CF93DF9300D01F92CDB7DEB771
:109E50008091C30D8111F2C08091EC03811110C07B
:109E60000F900F900F900F90DF91CF910F91FF9077
:109E7000EF90DF90CF90BF90AF909F908F9008951C
:109E80000DDE0E945C3C4B015C01809120029091B0
:109E90002102181619060CF000C1019790932102B7
:109EA000809320026091060470910704072E000C35
:109EB000880B990B0E947AAD69837A838B839C838C
:109EC0003EE1E32EF12C00E09E012F5F3F4F41E287
:109ED00054E068ED73E087ED93E00E94E6A4C09043
:109EE0002104D0902204E0902304F0902404809177
:109EF000CE049091CF04BC01990F880B990B0E945E
:109F00007AAD9B01AC01C701B6010E94FEB31816E1
:109F10000CF4A9C060E06093FD038091DC03909194
:109F2000DD03A091DE03B091DF030097A105B10529
:109F300021F1A5019401281B390B4A0B5B0B57FD3E
:109F40001CC06091E0037091E10380E090E00E940A
:109F500078AD9B01AC016091210470912204809145
:109F60002304909124040E9474AD87FFB7C043E797
:109F70005DE065E87DE080E0B0DD8091E2039091F6
:109F8000E303A091E403B091E5030097A105B105B7
:109F900011F1881A990AAA0ABB0AB7FC1CC0609181
:109FA000E6037091E70380E090E00E9478AD9B01AA
:109FB000AC016091000470910104809102049091C1
:109FC00003040E9474AD87FF87C041E55DE064E64D
:109FD0007DE08FEF82DD6091040470910504072E0F
:109FE000000C880B990B0E947AAD69837A838B836E
:109FF0009C839AE0E92EF12C0FEF9E012F5F3F4FDB
:10A0000040E054E062ED73E086ED93E00E94E6A448
:10A010008090000490900104A0900204B09003048A
:10A0200020E030E040EA50E4C501B4010E94FEB3F4
:10A0300087FF08C060E06093FE0312CF84E99DE0D3
:10A040000E94859420E030E046E153E4C501B4016C
:10A050000E9474AD181674F30E94DA450E941CB376
:10A0600075956795E8CF6091350270913602072E9D
:10A07000000C880B990B0E947AAD9B01AC01C701C3
:10A08000B6010E9474AD87FF45CF80E00E9417475C
:10A090000E941CB3759567953ECFC0902104D09067
:10A0A0002204E0902304F090240420E030E848E902
:10A0B00053E4C701B6010E94FEB3181694F020E0E5
:10A0C00030E040EA50E4C701B6010E9474AD87FF5A
:10A0D000E9CE80E06EDDE6CE91DB7DCF80E0D9DB9E
:10A0E0004CCF80E070DDC0902104D0902204E0903D
:10A0F0002304F0902404E3CFCF92DF92EF92FF92FB
:10A10000CF93DF936A017B01FC018491EF012196DB
:10A11000882321F00E94D876FE01F7CF4AE0C701DC
:10A12000B601DF91CF91FF90EF90DF90CF900C942C
:10A13000077BCF92DF92EF92FF92CF93DF936A017A
:10A140007B01FC018491EF012196882321F00E947C
:10A15000D876FE01F7CF42E0C701B601DF91CF917B
:10A16000FF90EF90DF90CF900C94877BEF92FF925F
:10A170000F931F93CF93DF931F92CDB7DEB78C0160
:10A180007B0180E249830E94D87649814F3F11F0DC
:10A1900084E501C082E40E94D8768AE30E94D876E2
:10A1A000F801608171818281938142E00E94877B06
:10A1B000F70140815181628173818BEE9EE0B9DFAE
:10A1C00062E070E080E090E00F90DF91CF911F910E
:10A1D0000F91FF90EF900C94223C0F931F93CF931D
:10A1E000DF93CDB7DEB728970FB6F894DEBF0FBE6A
:10A1F000CDBF6091060470910704072E000C880BF8
:10A20000990B0E947AAD6D837E838F8398878091AE
:10A21000210490912204A0912304B0912404898305
:10A220009A83AB83BC834DEFBE016B5F7F4FCE0142
:10A2300001969CDF6091040470910504072E000CC8
:10A24000880B990B0E947AAD6D837E838F839887EC
:10A250008091000490910104A0910204B091030444
:10A2600089839A83AB83BC834FEFBE016B5F7F4FC3
:10A27000CE0101967BDFE3EFFEE084918F010F5F5B
:10A280001F4F882321F00E94D876F801F6CFE09185
:10A29000FF03F0E0E350FC4F608170E080E090E06D
:10A2A0000E946D7BEEEEFEE084918F010F5F1F4FE9
:10A2B000882321F00E94D876F801F6CF6091FE0342
:10A2C00070E080E090E00E946D7B28960FB6F894D5
:10A2D000DEBF0FBECDBFDF91CF911F910F910895CB
:10A2E0000F931F93CF93DF9300D01F92CDB7DEB7AC
:10A2F000FC0184918F010F5F1F4F882361F0498318
:10A300005A836B837C830E94D876F80149815A81F5
:10A310006B817C81EECFCB01BA010F900F900F9033
:10A320000F90DF91CF911F910F910C946D7B0F9344
:10A330001F93CF93DF938B01FC018491EF01219652
:10A34000882321F00E94D876FE01F7CFB801110FC3
:10A35000880B990BDF91CF911F910F910C946D7B1E
:10A360000F931F93CF93DF931F921F92CDB7DEB74A
:10A37000FC0184918F010F5F1F4F811102C08B017F
:10A3800008C069837A830E94D876F80169817A814E
:10A39000F0CFF80181918F01882319F00E94D876BF
:10A3A000F8CF0F900F90DF91CF911F910F910895EB
:10A3B0002F923F924F925F926F927F928F929F92D5
:10A3C000AF92BF92CF92DF92EF92FF920F931F93C3
:10A3D000CF93DF93CDB7DEB7CC57D1090FB6F89442
:10A3E000DEBF0FBECDBFE091C10DF091C20DEF2BCE
:10A3F00011F00C94475B6C96DFAECEAE6C9729964D
:10A40000EFAE299779016A015B01FC01208131815E
:10A4100042815381A6962CAF3DAF4EAF5FAFA6975A
:10A420002091AB0D3091AC0D4091AD0D5091AE0D22
:10A43000A6966CAD7DAD8EAD9FADA6970E94D9ADB1
:10A440000E9409B4E2966CAF7DAF8EAF9FAFE297EA
:10A45000D5018D919D910D90BC91A02DAA968CAFA8
:10A460009DAFAEAFBFAFAA972091AF0D3091B00DA9
:10A470004091B10D5091B20DBC01CD010E94D9ADFA
:10A480000E9409B4E6966CAF7DAF8EAF9FAFE697A2
:10A49000D6012D913D914D915C91AE962CAF3DAF83
:10A4A0004EAF5FAFAE972091B30D3091B40D409198
:10A4B000B50D5091B60DAE966CAD7DAD8EAD9FAD28
:10A4C000AE970E94D9AD0E9409B4EA966CAF7DAFF9
:10A4D0008EAF9FAFEA97D7012D913D914D915C9141
:10A4E0006A962CAF3DAF4EAF5FAF6A972091B70D24
:10A4F0003091B80D4091B90D5091BA0D6A966CAD7E
:10A500007DAD8EAD9FAD6A970E94D9AD0E9409B412
:10A51000A0966CAF7DAF8EAF9FAFA09780910305E3
:10A5200083FF1CC0A0962CAD3DAD4EAD5FADA09796
:10A530002093A10E3093A20E4093A30E5093A40E2D
:10A540006A968CAD9DADAEADBFAD6A978093910E0E
:10A550009093920EA093930EB093940ED801BC9159
:10A56000BBABF801F181F8AFD8011296BC91BCAF3A
:10A57000F801F3812D96FFAF2D9780914B0E9091AE
:10A580004C0E891B8F708F3019F40E94B594F5CF53
:10A5900000914B0EEB960FAFEB9780914B0E282E50
:10A5A000312C8091950E9091960EA091970EB091BE
:10A5B000980EE2968CAC9DACAEACBFACE297881A1C
:10A5C000990AAA0ABB0A8091990E90919A0EA091BD
:10A5D0009B0EB0919C0EE6964CAC5DAC6EAC7FAC25
:10A5E000E697481A590A6A0A7B0A80919D0E909153
:10A5F0009E0EA0919F0EB091A00EEA962CAD3DAD9F
:10A600004EAD5FADEA97281B390B4A0B5B0B2BA3B2
:10A610003CA34DA35EA38091A10E9091A20EA091A8
:10A62000A30EB091A40EA0960CAD1DAD2EAD3FAD06
:10A63000A097081B190B2A0B3B0B0FA318A729A7E0
:10A640003AA7012B022B032B09F4BDC06091210412
:10A65000709122048091230490912404209120047D
:10A66000211141C00E941CB320912F023091300271
:10A6700062177307C4F5A0962CAD3DAD4EAD5FAD2E
:10A68000A0972093A10E3093A20E4093A30E509357
:10A69000A40E6A968CAD9DADAEADBFAD6A978093AA
:10A6A000910E9093920EA093930EB093940EEAECB9
:10A6B000FFE184918F010F5F1F4F882321F00E94DB
:10A6C000D876F801F6CFE6E1FFE084918F010F5FC5
:10A6D0001F4F882321F00E94D876F801F6CF1FA2E1
:10A6E00018A619A61AA66FA178A589A59AA50E94F1
:10A6F0007AAD29960FAD2997A4E00A9FF0011124A5
:10A70000E55DFD4F20813181428153810E94D9ADA9
:10A710006B017C0120E030E0A9010E94FEB387FFBD
:10A7200004C0F7FAF094F7F8F0946091B70D7091C7
:10A73000B80D8091B90D9091BA0D0E941CB39B0188
:10A74000AC01A8ECB0E00E94BEB10E947AAD9B01C2
:10A75000AC01C701B6010E94FEB31816C4F5A0965D
:10A760002CAD3DAD4EAD5FADA0972093A10E3093C3
:10A77000A20E4093A30E5093A40E6A968CAD9DAD8D
:10A78000AEADBFAD6A978093910E9093920EA09359
:10A79000930EB093940EEAECFFE184918F010F5F6A
:10A7A0001F4F882321F00E94D876F801F6CFE7EFFB
:10A7B000FEE084918F010F5F1F4F882321F00E94DC
:10A7C000D876F801F6CF1FA218A619A61AA6D501A9
:10A7D000C4018827B7FD83959927AA27BB27182F7F
:10A7E00077FC12602BA13CA14DA15EA157FD146026
:10A7F0008FA198A5A9A5BAA5B7FD18606FA178A5E6
:10A8000089A59AA50E947AAD29960FAD2997A4E053
:10A810000A9FF0011124E55DFD4F208131814281C5
:10A8200053810E94D9AD6B017C0120E030E0A90189
:10A830000E94FEB387FF04C0C701B601905802C052
:10A84000C701B60120E030E040E05FE30E94D8B1EC
:10A850000E9421B36CAB7DAB8EAB9FAB88E5829D34
:10A86000F001839DF00D1124E45FF84F108216ABC8
:10A8700024968CAE9DAEAEAEBFAE2497B7FE0DC093
:10A8800022273327A901281939094A095B09249687
:10A890002CAF3DAF4EAF5FAF249788E5829DF001AE
:10A8A000839DF00D1124E45FF84F24968CAD9DAD8F
:10A8B000AEADBFAD2497858B968BA78BB08F62967C
:10A8C0004CAE5DAE6EAE7FAE629777FE0DC02227B6
:10A8D0003327A901241935094609570962962CAF77
:10A8E0003DAF4EAF5FAF629788E5829DF001839DDB
:10A8F000F00D1124E45FF84F62968CAD9DADAEADC6
:10A90000BFAD6297818F928FA38FB48F2BA13CA193
:10A910004DA15EA128962CAF3DAF4EAF5FAF2897FB
:10A9200057FF0DC050954095309521953F4F4F4FA3
:10A930005F4F28962CAF3DAF4EAF5FAF289788E5AD
:10A94000829DF001839DF00D1124E45FF84F28965D
:10A950008CAD9DADAEADBFAD2897858F968FA78F7F
:10A96000B0A3C501B4010E947AAD2091FC063091DC
:10A97000FD064091FE065091FF060E94D9AD6BA7DF
:10A980007CA78DA79EA7698B7A8B8B8B9C8BC30131
:10A99000B2010E947AAD20910007309101074091E9
:10A9A0000207509103070E94D9AD6FA778AB89AB1E
:10A9B0009AAB6D8B7E8B8F8B988F20910407309193
:10A9C0000507409106075091070766962CAF3DAFEB
:10A9D0004EAF5FAF66976BA17CA18DA19EA10E9437
:10A9E0007AAD66962CAD3DAD4EAD5FAD66970E94DB
:10A9F000D9AD4B015C01698F7A8F8B8F9C8F209131
:10AA000008073091090740910A0750910B07C701C9
:10AA1000B6010E94D9AD6B017C016D8F7E8F8F8F47
:10AA200098A324968CAD9DADAEADBFAD249706978F
:10AA3000A105B1057CF562962CAD3DAD4EAD5FAD87
:10AA40006297263031054105510524F528968CADD5
:10AA50009DADAEADBFAD28970697A105B105D4F465
:10AA600020E030E0A901C701B6010E94FEB387FFD4
:10AA700004C0F7FAF094F7F8F09488E5829DF001AD
:10AA8000839DF00D1124E45FF84FC586D686E786D6
:10AA9000F08AA1C16C96AEADBFAD6C97CD90DD9044
:10AAA000ED90FC9020E030E0A901C701B6010E94C2
:10AAB00074AD882369F088E5829DF001839DF00DD7
:10AAC0001124E45FF84FC586D686E786F08A34C045
:10AAD0002BA53CA54DA55EA5CA01B9010E94D9AD23
:10AAE0006B017C012FA538A949A95AA9CA01B9014E
:10AAF0000E94D9AD9B01AC01C701B6010E94D8B13B
:10AB00006B017C01A5019401C501B4010E94D9AD7E
:10AB10009B01AC01C701B6010E94D8B10E9443B4A9
:10AB200028E5229DF001239DF00D1124E45FF84FEC
:10AB3000658776878787908B8091620D882309F4DB
:10AB40004AC1C0901504D0901604E0901704F0900C
:10AB5000180420E030E0A901C701B6010E9474ADDD
:10AB6000882309F438C18090110490901204A090B9
:10AB70001304B090140420E030E0A901C501B40131
:10AB80000E9474AD882309F426C12BA13CA14DA1DC
:10AB90005EA1211531054105510509F41CC157FD80
:10ABA0000BC080E090E0A0E8BFE324968CAF9DAF9F
:10ABB000AEAFBFAF24970AC020E030E040E85FEBC3
:10ABC00024962CAF3DAF4EAF5FAF249712FB1127F9
:10ABD00010F9809110048117B1F110931004609165
:10ABE0000C0470910D0480910E0490910F040E944A
:10ABF0007AAD2B013C01A501940124966CAD7DAD8D
:10AC00008EAD9FAD24970E94D9ADA70196010E94F9
:10AC1000D9AD2091B30D3091B40D4091B50D509147
:10AC2000B60D0E94D9AD9B01AC01C301B2010E94D7
:10AC3000D8B10E941CB360930C0470930D048093F0
:10AC40000E0490930F0440900C0450900D046090FB
:10AC50000E0470900F048BA19CA1ADA1BEA118168B
:10AC600019061A061B0634F41414150416041704E6
:10AC70001CF0B1C077FEAFC0C301B2010E947AAD33
:10AC80004B015C0188E5829DF001839DF00D11244C
:10AC9000E45FF84F20912702309128024091290269
:10ACA00050912A0265857685878590890E94B4B285
:10ACB0006B017C0120E030E040E85FE30E94FEB3DE
:10ACC000181634F4C12CD12C30E8E32E3FE3F32ED8
:10ACD000A7019601C501B4010E94D9AD0E941CB321
:10ACE0006B017C01DC01CB01F7FE07C088279927A7
:10ACF000DC018C199D09AE09BF0928960CAD1DAD6C
:10AD00002EAD3FAD2897080F191F2A1F3B1FC90101
:10AD1000B80128E5229D8001239D100D1124045FB8
:10AD2000184FD8015D966D937D938D939C9390976A
:10AD30004C185D086E087F0840920C0450920D0478
:10AD400060920E0470920F040E9478AD9B01AC01DA
:10AD500024966CAD7DAD8EAD9FAD24970E94D9AD8C
:10AD600066962CAD3DAD4EAD5FAD66970E94D9ADF8
:10AD70006B017C01698F7A8F8B8F9C8F2BA53CA5F3
:10AD80004DA55EA5CA01B9010E94D9AD4B015C0178
:10AD90002FA538A949A95AA9CA01B9010E94D9AD5C
:10ADA0009B01AC01C501B4010E94D8B14B015C010B
:10ADB000A7019601C701B6010E94D9AD9B01AC0164
:10ADC000C501B4010E94D8B10E9443B4F80165875F
:10ADD00076878787908B88E5829DF001839DF00DB3
:10ADE0001124E45FF84F0CA91DA92EA93FA901A3C6
:10ADF00012A323A334A3458956896789708D058DD5
:10AE0000168D278D30A1818D928DA38DB48D8017E5
:10AE10009107A207B30710F4D901C8018417950759
:10AE2000A607B70710F4DB01CA010CA91DA92EA9BA
:10AE30003FA980179107A207B30710F4D901C801F1
:10AE400028E5229DF001239DF00D1124E45FF84FC9
:10AE500085A396A3A7A3B0A70697A105B10508F4FB
:10AE60000FC4DF01AE5ABF4F80911E0490911F04A2
:10AE70008D939C9329961FAD299711A7452B462B9F
:10AE8000472B09F0179888E5829DF001839DF00D0E
:10AE90001124E45FF84F818D928DA38DB48D892BA1
:10AEA0008A2B8B2B09F0169888E5829DF001839DF3
:10AEB000F00D1124E45FF84F858D968DA78DB0A11C
:10AEC000892B8A2B8B2B09F015982CA93DA94EA90B
:10AED0005FA9232B242B252B09F4DBC380911D04B0
:10AEE000882319F0815080931D0429960FAD29976E
:10AEF000011104C0149880E280931D04E090770D46
:10AF0000F090780D0091790D10917A0D9701A801BC
:10AF10006BA978AD8CAD2D969FAD2D970E9474AD29
:10AF200087FF06C0EBAAF8AE0CAF2D961FAF2D978A
:10AF300088E5829DF001839DF00D1124E45FF84FB8
:10AF400085849684A784B088A501940160E070E0B0
:10AF500080E89FE30E94B4B224966CAF7DAF8EAFC1
:10AF60009FAF24979B01AC016BA978AD8CAD2D965A
:10AF70009FAD2D970E94D9AD2B013C0180914B0EC6
:10AF80009091490E891B8F7025968FAF2597A3014D
:10AF9000920160E074E284E799E40E94B4B20E94F6
:10AFA00009B46B017C0125968FAD259782508630C0
:10AFB00008F478C3A3019201C501B4010E94D9AD80
:10AFC0009B01AC010E94D9AD62966CAF7DAF8EAF94
:10AFD0009FAF629788E5829D8001839D100D1124AB
:10AFE000045F184F62968CAD9DADAEADBFAD62975C
:10AFF000F80181839283A383B48325A136A147A15D
:10B0000050A528AF39AF4AAF5BAFCA01B9010E9462
:10B0100078AD6CAF7DAF8EAF9FAFA30192010E9460
:10B02000D9AD0E949EB20E9421B34B015C01F80190
:10B03000EE5BFF4F60837183828393838E010F5E8B
:10B040001F4F2A961FAF0EAF2A97005111092E9657
:10B050001FAF0EAF2E970BE91DE0A2961FAF0EAFEC
:10B06000A2978E010F5D1F4F1AA309A32E960EAD56
:10B070001FAD2E976C961FAF0EAF6C971BA21BA631
:10B0800010E81FA70FE30BAB2A96AEADBFAD2A9712
:10B090006D917D918D919D912A96BFAFAEAF2A970C
:10B0A000A30192010E94D9AD6B017C016C96EEADBB
:10B0B000FFAD6C9761937193819391936C96FFAF01
:10B0C000EEAF6C9720E030E0A9010E94FEB387FF4D
:10B0D00004C0F7FAF094F7F8F094A296AEADBFADC5
:10B0E000A2970D911D912D913D91A296BFAFAEAF4C
:10B0F000A29766960CAF1DAF2EAF3FAF6697A90122
:10B100009801C701B6010E94FEB318160CF404C3DF
:10B110002A960EAD1FAD2A9729A13AA1021713074F
:10B1200009F0B2CF20E030E040E85FE36BA17BA5FF
:10B130008FA59BA90E9474AD87FF53C07E0131E1AA
:10B14000E30EF11C2E960EAD1FAD2E972BA13BA545
:10B150004FA55BA9D8016D917D918D919C910E9425
:10B16000D9ADF80161937193819391938F01EE159D
:10B17000FF0561F728E5229DC001239D900D112454
:10B180008C01045F184F78010E5B1F4FC501B4019D
:10B190000E9478AD2BA13BA54FA55BA90E94D9AD1C
:10B1A0000E9421B3D8016D937D938D939C93139747
:10B1B0002BA13BA54FA55BA96BA17BA58FA59BA947
:10B1C0000E94D9AD9B01AC0162966CAD7DAD8EAD98
:10B1D0009FAD62970E94D9ADF7016183728383832B
:10B1E000948324962CAD3DAD4EAD5FAD24976CADF0
:10B1F0007DAD8EAD9FAD0E94D9AD6BA37CA38DA319
:10B200009EA388E5829D8001839D100D1124045F1B
:10B21000184FD80155968D909D90AD90BC90589741
:10B2200081149104A104B10409F092C259968D9140
:10B230009D910D90BC91A02D892B8A2B8B2B09F011
:10B2400087C2F801858D968DA78DB0A1892B8A2B99
:10B250008B2B09F07DC22091830D3091840D40919C
:10B26000850D5091860D6BA17CA18DA19EA10E94A0
:10B27000D9AD0E949EB20E9421B32B013C01D8019E
:10B28000D7961C9288E5829D8001839D100D112424
:10B29000045F184FF801E25BFF4F408251826282E7
:10B2A0007382C301B2010E9478AD6B017C012BA1B6
:10B2B0003CA14DA15EA10E94B4B22C966CAF7DAFB3
:10B2C0008EAF9FAF2C97D80151966D937D938D9340
:10B2D0009C9354972DEB37E346E051E4C701B60148
:10B2E0000E94D9AD0E9421B3F80162AB73AB84AB6D
:10B2F00095AB87A9882381F1FE9620813181428117
:10B3000053816091460D7091470D8091480D909149
:10B31000490D0E94D9AD2C962CAD3DAD4EAD5FAD23
:10B320002C970E94D9AD2091B70D3091B80D409166
:10B33000B90D5091BA0D0E94D9AD9B01AC0160E0EE
:10B3400074E284EF99E40E94B4B20E9421B3D80160
:10B35000D9967C936E93D89788E5829DF001839D62
:10B36000F00D1124E45FF84F0181128123813481B3
:10B3700024960CAF1DAF2EAF3FAF2497C901B80183
:10B380000E9443B4162F072F8BA39FA323E63DE013
:10B3900060963FAF2EAF60973E0131E1630E711CA6
:10B3A00043E65DE05DAF4CAF2E964EAC5FAC2E97A2
:10B3B0006BA77FA78BAB9CAB18AED201CD90DD9075
:10B3C000ED90FD902D0120E030E0A901C701B6010C
:10B3D0000E94FEB387FF04C0F7FAF094F7F8F094E8
:10B3E000ECADFDAD81909190A190B190FDAFECAF2F
:10B3F000A5019401C701B6010E94FEB318160CF412
:10B40000B4C446145704C9F65BA56B965FAF6B973F
:10B410008FA5A1968FAFA1979BA9EC969FAFEC97B4
:10B42000ACA9ED96AFAFED972596BFAD2597B111BD
:10B43000DCC46B968FAD6B97A1969FADA197EC96F0
:10B44000AFADEC97ED96BFADED9780931904909357
:10B450001A04A0931B04B0931C0488E5829D80010C
:10B46000839D100D1124045F184F2BA53FA54BA9F8
:10B470005CA96BA57FA58BA99CA90E94D9ADD80119
:10B4800019966D937D938D939C931C972C966CAD20
:10B490007DAD8EAD9FAD2C9790589B01AC010E9465
:10B4A000D8B1F80125853685478550890E94D9ADE8
:10B4B0009B01AC016BE077ED83E29BE30E94D7B187
:10B4C0009B01AC018BE097EDA3E2BBE3F801858320
:10B4D0009683A783B087108124966CAD7DAD8EAD29
:10B4E0009FAD24970E9474AD18160CF0BEC581E084
:10B4F000182B88E5829DF001839DF00D1124E45FF7
:10B50000F84F108380E1FE013196A5E7BEE001907F
:10B510000D928A95E1F724960CAD1DAD2EAD3FAD91
:10B5200024970093710E1093720E2093730E309334
:10B53000740EE2962CAD3DAD4EAD5FADE29720931B
:10B54000950E3093960E4093970E5093980EE69674
:10B550008CAD9DADAEADBFADE6978093990E909347
:10B560009A0EA0939B0EB0939C0EEA960CAD1DAD67
:10B570002EAD3FADEA9700939D0E10939E0E209343
:10B580009F0E3093A00EA0962CAD3DAD4EAD5FAD9D
:10B59000A0972093A10E3093A20E4093A30E509338
:10B5A000A40EA6968CAD9DADAEADBFADA697809313
:10B5B000850E9093860EA093870EB093880EAA9660
:10B5C0000CAD1DAD2EAD3FADAA970093890E109323
:10B5D0008A0E20938B0E30938C0EAE962CAD3DAD23
:10B5E0004EAD5FADAE9720938D0E30938E0E40938F
:10B5F0008F0E5093900E6A968CAD9DADAEADBFADE3
:10B600006A978093910E9093920EA093930EB093AD
:10B61000940E90914B0E80914C0E981303C084E6CB
:10B620008093480EEB968FADEB978F5F8F70809372
:10B630004B0E80914B0E90914A0E81508F70891362
:10B6400016C500914C0E0BA310914B0E1FA398E54D
:10B650000FA11BA1011394C5812C912CA12CB12CFD
:10B660001BA61FA61BAA1CAA212C312C00E010E04F
:10B67000FBA12FA1F21391C52114310409F042C698
:10B6800080916F00826080936F0081E0A0C780E0AE
:10B690009EC7E090730DF090740D0091750D1091A0
:10B6A000760D34CC80917B0D90917C0DA0917D0D19
:10B6B000B0917E0DC816D906EA06FB0608F07ACCD2
:10B6C0008C199D09AE09BF09BC01CD01660F771F1A
:10B6D000881F991F25964FAD2597042F10E020E075
:10B6E00030E0A90198010E9480B1CA01B9010E940D
:10B6F00078AD0E9409B46C0D7D1D8E1D9F1D0E94AA
:10B7000078AD9B01AC0160E074E284E799E40E94AB
:10B71000B4B22B013C014ECCA701960166966CADEC
:10B720007DAD8EAD9FAD66970E94B4B27B018C015A
:10B730009B01AC016BA17BA58FA59BA90E94FEB3C9
:10B7400018160CF0E5CCEBA2FBA60FA71BABE0CCC8
:10B750000CA91DA92EA93FA9012B022B032B49F0EF
:10B760006091870D7091880D8091890D90918A0D5F
:10B7700008C060917F0D7091800D8091810D909136
:10B78000820D2BA13CA14DA15EA10E94D9AD0E94CA
:10B790009EB20E9421B32B013C012CA93DA94EA9C8
:10B7A0005FA9232B242B252BC9F020E030E0A90131
:10B7B0006091460D7091470D8091480D9091490D13
:10B7C0000E9474AD882351F081E00FA118A529A52E
:10B7D0003AA510161106120613060CF080E098E543
:10B7E000929D8001939D100D1124045F184FD80184
:10B7F000D7968C93882309F4BAC02091850E309196
:10B80000860E4091870E5091880EA6966CAD7DAD48
:10B810008EAD9FADA6970E94D7B16FA378A789A7D9
:10B820009AA72091890E30918A0E40918B0E5091EB
:10B830008C0EAA966CAD7DAD8EAD9FADAA970E9481
:10B84000D7B16BA77CA78DA79EA720918D0E3091B5
:10B850008E0E40918F0E5091900EAE966CAD7DADD8
:10B860008EAD9FADAE970E94D7B16B017C012FA129
:10B8700038A549A55AA5CA01B9010E94D9AD6FA33F
:10B8800078A789A79AA72BA53CA54DA55EA5CA01B7
:10B89000B9010E94D9AD9B01AC016FA178A589A522
:10B8A0009AA50E94D8B16FA378A789A79AA7A701E4
:10B8B0009601C701B6010E94D9AD9B01AC016FA1F1
:10B8C00078A589A59AA50E94D8B10E9443B46B01BE
:10B8D0007C012091910E3091920E4091930E5091E7
:10B8E000940E6A966CAD7DAD8EAD9FAD6A970E9449
:10B8F000D7B1A70196010E94B4B26B017C01F80197
:10B90000FE96608371838283938320E030E040E47D
:10B9100050E40E94FEB318161CF4F80117AA27C0C1
:10B920002091460D3091470D4091480D5091490DA1
:10B93000C701B6010E94D9AD9B01AC0160916F0DAA
:10B940007091700D8091710D9091720D0E94B4B242
:10B950002BA13CA14DA15EA10E94D9AD0E9421B3B3
:10B96000641575058605970510F42B013C0180913F
:10B97000E8069091E906A091EA06B091EB0608ADC1
:10B9800019AD2AAD3BAD80179107A207B30708F4A4
:10B99000DCC081149104A104B10441F12091EC06B2
:10B9A0003091ED064091EE065091EF0624153505D5
:10B9B00046055705D8F468AD79AD8AAD9BAD0E94B8
:10B9C00071B16B017C01A3019201C501B4010E9418
:10B9D00071B1C616D706E806F90640F4C701B601EC
:10B9E000A50194010E9480B129013A0188E5829D58
:10B9F000F001839DF00D1124E45FF84FC18CD28CCF
:10BA0000E38CF48CC114D104E104F10441F12091E0
:10BA1000F0063091F1064091F2065091F30624159C
:10BA2000350546055705D8F468AD79AD8AAD9BADAF
:10BA30000E9471B14B015C01A3019201C701B601E3
:10BA40000E9471B186169706A806B90640F4C50192
:10BA5000B401A70196010E9480B129013A0188E54D
:10BA6000829DF001839DF00D1124E45FF84FC58C99
:10BA7000D68CE78CF0A0C114D104E104F10441F1AB
:10BA80002091F4063091F5064091F6065091F706A4
:10BA90002415350546055705D8F468AD79AD8AAD4E
:10BAA0009BAD0E9471B14B015C01A3019201C701E2
:10BAB000B6010E9471B186169706A806B90640F431
:10BAC000C501B401A70196010E9480B129013A0184
:10BAD00088E5829DF001839DF00D1124E45FF84F0D
:10BAE000C1A0D2A0E3A0F4A0C114D104E104F104E8
:10BAF00009F4C8CB2091F8063091F9064091FA0676
:10BB00005091FB06241535054605570508F0BACBBC
:10BB100068AD79AD8AAD9BAD0E9471B14B015C01FE
:10BB2000A3019201C701B6010E9471B18616970662
:10BB3000A806B90608F0A6CBC501B401A701960175
:10BB40000E9480B129013A019DCB81149104A10486
:10BB5000B104A9F16091EC067091ED068091EE06BA
:10BB60009091EF06641575058605970540F50E94CE
:10BB700078AD2CAD3DAD4EAD5FAD0E94D9AD6B0142
:10BB80007C01C501B4010E9478AD4B015C01C30189
:10BB9000B2010E9478ADA50194010E94D9ADA70120
:10BBA00096010E94FEB3181654F4A5019401C70132
:10BBB000B6010E94B4B20E9421B32B013C0188E57A
:10BBC000829DF001839DF00D1124E45FF84F818C7C
:10BBD000928CA38CB48C81149104A104B104A9F1BA
:10BBE0006091F0067091F1068091F2069091F30653
:10BBF000641575058605970540F50E9478AD2CAD56
:10BC00003DAD4EAD5FAD0E94D9AD6B017C01C5016C
:10BC1000B4010E9478AD4B015C01C301B2010E94E6
:10BC200078ADA50194010E94D9ADA70196010E94AB
:10BC3000FEB3181654F4A5019401C701B6010E9481
:10BC4000B4B20E9421B32B013C0188E5829DF00132
:10BC5000839DF00D1124E45FF84F858C968CA78CA2
:10BC6000B0A081149104A104B104A9F16091F4067B
:10BC70007091F5068091F6069091F70664157505AA
:10BC80008605970540F50E9478AD2CAD3DAD4EADD3
:10BC90005FAD0E94D9AD6B017C01C501B4010E946A
:10BCA00078AD4B015C01C301B2010E9478ADA501E2
:10BCB00094010E94D9ADA70196010E94FEB3181607
:10BCC00054F4A5019401C701B6010E94B4B20E94C8
:10BCD00021B32B013C0188E5829DF001839DF00D8D
:10BCE0001124E45FF84FC1A0D2A0E3A0F4A0C114D6
:10BCF000D104E104F10409F4C5CA6091F806709119
:10BD0000F9068091FA069091FB0664157505860583
:10BD1000970508F0B7CA0E9478AD2CAD3DAD4EAD89
:10BD20005FAD0E94D9AD4B015C01C701B6010E9415
:10BD300078AD6B017C01C301B2010E9478ADA7010F
:10BD400096010E94D9ADA50194010E94FEB3181678
:10BD50000CF098CAA7019601C501B4010E94B4B2C3
:10BD60000E9421B32B013C018DCAF8ADFF2329F1BC
:10BD7000A5019401612F702F8BA19FA10E94D9ADC5
:10BD80004B015C012BA53FA54BA95CA9C701B601DE
:10BD90000E94D9ADA50194010E94FEB3181614F5B6
:10BDA000A7019601C501B4010E94B4B26BA77FA799
:10BDB0008BAB9CAB21E028AF24CBA7019601C5013A
:10BDC000B4010E94B4B29B01AC016BA57FA58BA905
:10BDD0009CA90E94D9AD6BA77FA78BAB9CAB31E030
:10BDE00038AF0FCB41E048AF0CCBC090710ED09074
:10BDF000720EE090730EF090740E2DEB37E346E870
:10BE000055E3C701B6010E9474AD87FD12CBC7018F
:10BE1000B6010E9443B46B017C019B01AC01612F10
:10BE2000702F8BA19FA10E9474AD87FD04C01C2DB3
:10BE30000D2DEBA2FFA29601A701612F702F8BA100
:10BE40009FA10E94B4B266966CAF7DAF8EAF9FAFDC
:10BE50006697E5E7FEE02696FFAFEEAF269720E077
:10BE600030E040E85FE328AF39AF4AAF5BAF1CAECC
:10BE70002696AEADBFAD26976D917D918D919D912A
:10BE80002696BFAFAEAF269766962CAD3DAD4EADB4
:10BE90005FAD66970E94D9AD6B017C012E96EEAD29
:10BEA000FFAD2E9781909190A190B1902E96FFAF0B
:10BEB000EEAF2E97FCADFF2391F028AD39AD4AAD22
:10BEC0005BAD0E94D9AD6B017C0128AD39AD4AADA7
:10BED0005BADC501B4010E94D9AD4B015C01A50168
:10BEE0009401C701B6010E94FEB320E030E0A90131
:10BEF00018162CF5C501B4010E94FEB318164CF0BB
:10BF000020E030E0A901C701B6010E9474AD87FFAF
:10BF100005C0A5019401C701B60124C02401350163
:10BF200077FA709477F87094A3019201C701B60173
:10BF30000E94FEB318165CF52601370128C0C50122
:10BF4000B4010E9474AD87FD09C020E030E0A90172
:10BF5000C701B6010E94FEB318164CF4A701960162
:10BF6000C501B4010E94D7B12B013C0110C02601CC
:10BF7000370177FA709477F87094A5019401C301A2
:10BF8000B2010E94FEB3181614F024013501609628
:10BF9000AEADBFAD6097CD90DD90ED90FD90609619
:10BFA000BFAFAEAF6097A7019601C301B2010E9477
:10BFB000FEB31816ACF4A3019201C701B6010E94AA
:10BFC000B4B29B01AC0168AD79AD8AAD9BAD0E9466
:10BFD000D9AD68AF79AF8AAF9BAFBCADBF5FBCAF27
:10BFE0002696EEADFFAD2697E558FE4009F040CF0E
:10BFF0003CAD332371F028AD39AD4AAD5BAD612F57
:10C00000702F8BA19FA10E94D9AD162F072F8BA354
:10C010009FA324EA30E74DE75FE3612F702F8BA1E8
:10C020009FA10E94D9AD6B017C019B01AC01609185
:10C03000190470911A0480911B0490911C040E94B1
:10C04000FEB318165CF4A70196016BA57FA58BA91A
:10C050009CA90E94FEB318160CF4EBC91BA70FA7EE
:10C060000BA10BAB1FA11CABE4C983E041CAF0904C
:10C070004B0E8FEF8F0D8F708BA3B0904A0E809177
:10C080004B0EB81206C000914A0E0BA3C12CD12C46
:10C0900069C0C12CD12C1BA11B15A9F31BA1812E9A
:10C0A000912C28E5289D8001299D100D1124045F05
:10C0B000184FD8018C9183FD27C00BAB1CAB011529
:10C0C000110521F11996BC91BFA3F801F285FBA7D8
:10C0D000D8011B96BC91BFA7F801A4844580568067
:10C0E000678070842FA13BA54B2F5A2DC301B2014D
:10C0F0000E9474AD81117FC1C114D10439F0D60101
:10C100008C9180FD78C102C0CBAADCAA8BA18150A2
:10C110008F708BA380914A0EB81649F00BA10B15B6
:10C1200009F4B1CF81E08B0D8F70B82EF3CFCBA87F
:10C13000DCA8B1CF0BA1802E912C28E5289D800191
:10C14000299D100D1124045F184FD8018C9183FD97
:10C1500015C05801C114D10459F48BA18F5F8F70A1
:10C160008BA3650180914B0E1BA11813E3CF69CA05
:10C17000C6010E94E3A38111F0CFB3C15601EDCFF8
:10C180008FA181508F70989FF0011124E45FF84FC8
:10C19000208123FF61CA8FA35BCA28E53BA1239FAF
:10C1A000C0011124AC01445F584F1A01DA018C918F
:10C1B00083FD19C015966D917D918D919C91189775
:10C1C0000E9443B4F62EE72ED82EC92E0115110574
:10C1D00009F48AC0F801808180FD0AC0D1018C91E8
:10C1E00080FD06C081C0FBA4EFA4DBA8CCA881C061
:10C1F000F801808181608083C8010E94E3A38111DE
:10C200006FC0F80161817281838194810E9443B47F
:10C210002B013C019B01AC0160E070E080E89FE3F2
:10C220000E94B4B24B015C019B01AC016F2D7E2DCD
:10C230008D2D9C2D0E94D9AD69837A838B839C833D
:10C24000A50194016BA57FA58BA99CA90E94D9ADDE
:10C25000698B7A8B8B8B9C8BAE014F5F5F4FBE01DE
:10C260006F5E7F4FC8010E945849D801D7968C91C4
:10C270008823B1F12091460D3091470D4091480D32
:10C280005091490DF801FE96608171818281938100
:10C290000E94D9AD2091B70D3091B80D4091B90DE4
:10C2A0005091BA0D0E94D9AD4B015C019B01AC01CC
:10C2B000C301B2010E94D9AD0E9421B3F80173AF4E
:10C2C00062AFA50194016F2D7E2D8D2D9C2D0E94B6
:10C2D000D9AD0E9421B3D801DD967C936E93DC9793
:10C2E000F80180818E7F80838F2C9E2CAD2CBC2CFE
:10C2F00081018BA18F5F8F708BA3FBA6EFA6DBAABA
:10C30000CCAAB6C9D1018C9181608C93C8010E94DE
:10C31000E3A381116BC0F1016181728183819481FA
:10C320000E9443B46B017C019B01AC0160E070E0B2
:10C3300080E89FE30E94B4B22B013C012DEC3CEC61
:10C340004CE45DE30E94D9AD69837A838B839C833F
:10C35000A3019201B401C5010E94D9AD698B7A8B0A
:10C360008B8B9C8BAE014F5F5F4FBE016F5E7F4F2B
:10C37000C1010E945849D101D7968C918823B1F10F
:10C380002091460D3091470D4091480D5091490D37
:10C39000F101FE9660817181828193810E94D9AD05
:10C3A0002091B70D3091B80D4091B90D5091BA0D53
:10C3B0000E94D9AD4B015C019B01AC01C701B601E4
:10C3C0000E94D9AD0E9421B3F10173AF62AF2DEC91
:10C3D0003CEC4CE45DE3C501B4010E94D9AD0E9480
:10C3E00021B3D101DD967C936E93DC97F1018081BE
:10C3F0008E7F808345C928E5289DF001299DF00D99
:10C400001124E45FF84F808181FD3FC0C114D10445
:10C4100031F0F601C580D680E780F08408C08BE05B
:10C42000C82E87EDD82E83E2E82E8BE3F82E28E580
:10C43000289DF001299DF00D1124E45FF84F8189BA
:10C440009289A389B489BC01CD0190589B01AC01AC
:10C450000E94D8B1D8011D962D913D914D915C91CE
:10C4600050970E94D9AD9B01AC01C701B6010E9453
:10C47000D7B11B016C019B01AC016FA17BA58FA5FE
:10C480009A2D0E9474AD87FF04C02FA03BA4CFA4B7
:10C49000DA2C9101A601C301B2010E9474AD882378
:10C4A00009F434CEB8E5B89DC001B99D900D1124B2
:10C4B000FC01E45FF84F4F01808181608083C801F7
:10C4C0000E94E3A3882329F0D4018C918E7F8C9362
:10C4D0001DCEC101D601F40185839683A783B08761
:10C4E00015CED6018C9181FD50C0D60115962D91A7
:10C4F0003D914D915C9118972FA338A749A75AA752
:10C500001501B5E02B0E311CF8014580568067807F
:10C510007084A30192016FA178A589A59AA50E94B4
:10C5200074AD87FF32C0F60181899289A389B489ED
:10C53000BC01CD0190589B01AC010E94D8B1D6013D
:10C540001D962D913D914D915C9150970E94D9ADD2
:10C550009B01AC016FA178A589A59AA50E94D7B1CE
:10C560006B017C01A30192010E9474AD87FF0DC095
:10C57000D8018C9181608C93C5010E94E3A388232C
:10C58000E1F0F80180818E7F808318E5189DF0012D
:10C59000199DF00D1124E45FF84F21853285438504
:10C5A000548565817681878190850E9474AD811163
:10C5B000D4CD0BA100934A0ED0CDD101CD92DD9206
:10C5C000ED92FC9213970BA100934A0EDECFC45854
:10C5D000DF4F0FB6F894DEBF0FBECDBFDF91CF9116
:10C5E0001F910F91FF90EF90DF90CF90BF90AF9091
:10C5F0009F908F907F906F905F904F903F902F9083
:10C60000089580914B0E90914C0E891B8F708F3046
:10C6100019F40E94B594F5CF80914B0E8F5F8F7007
:10C62000E0914B0E98E59E9FF0011124E45FF84FD6
:10C63000DF011D929A95E9F798E090834091950E5D
:10C640005091960E6091970E7091980E458B568B77
:10C65000678B708F4091990E50919A0E60919B0E4E
:10C6600070919C0E418F528F638F748F40919D0EFD
:10C6700050919E0E60919F0E7091A00E458F568F27
:10C68000678F70A34091A10E5091A20E6091A30EEE
:10C690007091A40E41A352A363A374A320914B0EE7
:10C6A00090914C0E291303C094E69093480E80930A
:10C6B0004B0E80916F00826080936F00089590917F
:10C6C0004B0E80914C0E981719F00E94B594F7CF3D
:10C6D0008091C10D9091C20D892BB9F70895909169
:10C6E0004B0E80914C0E981719F00E94B594F7CF1D
:10C6F0008091C10D9091C20D892BB9F70C94729461
:10C70000CF93DF9390916F0091FB222720F991FF47
:10C7100005C090916F009D7F90936F0094E0899F7A
:10C72000E0011124FE01E853F24F608171818281A2
:10C730009381222329F020916F00226020936F00C3
:10C740000E947AADC450D94F288139814A815B81DA
:10C750000E94D9ADDF91CF9108952F923F924F92D1
:10C760005F926F927F928F929F92AF92BF92CF9281
:10C77000DF92EF92FF920F931F93CF93DF93CDB78A
:10C78000DEB7E8970FB6F894DEBF0FBECDBF20919D
:10C79000620D222309F4E6C01C010091510E109194
:10C7A000520E2091530E3091540E4090550E5090E1
:10C7B000560E6090570E7090580E4DA65EA66FA64E
:10C7C00078AA8090590E90905A0EA0905B0EB0906F
:10C7D0005C0E40915D0E50915E0E60915F0E709107
:10C7E000600E8091610E9091620EA091630EB091E7
:10C7F000640E89AB9AABABABBCABC090650ED0906E
:10C80000660EE090670EF090680E8091690E909130
:10C810006A0EA0916B0EB0916C0E40906D0E509010
:10C820006E0E60906F0E7090700E4DAA5EAA6FAA89
:10C8300078AE40904D0E50904E0E60904F0E70901E
:10C84000500E49825A826B827C828D829E82AF8298
:10C85000B886C986DA86EB86FC860D871E872F8709
:10C86000388B498B5A8B6B8B7C8B8D8B9E8BAF8BD4
:10C87000B88F8DA59EA5AFA5B8A9898F9A8FAB8FCC
:10C88000BC8F49A85AA86BA87CA84D8E5E8E6F8E6F
:10C8900078A28DA99EA9AFA9B8AD89A39AA3ABA38D
:10C8A000BCA320E030E040E450E4D1016D917D91E3
:10C8B0008D919C910E94D8B169A77AA78BA79CA75C
:10C8C0002DEC3CEC46E353E4F101648175818681F3
:10C8D00097810E94D7B16DA37EA38FA398A7C101B2
:10C8E00008969F938F93CE0185969F938F9304967E
:10C8F0009F938F938DB79EB784970FB6F8949EBF82
:10C900000FBE8DBFADB7BEB7119684E2FE01319662
:10C9100001900D928A95E1F70E94519120E030E05C
:10C9200040E450E469A57AA58BA59CA50E94D7B1E7
:10C93000D1016D937D938D939C9313972DEC3CECDB
:10C9400046E353E46DA17EA18FA198A50E94D8B1C2
:10C95000F10164837583868397830FB6F894DEBFF5
:10C960000FBECDBFE8960FB6F894DEBF0FBECDBFA9
:10C97000DF91CF911F910F91FF90EF90DF90CF90BB
:10C98000BF90AF909F908F907F906F905F904F90EF
:10C990003F902F900895CF92DF92EF92FF920F93E6
:10C9A0001F93CF93DF93C091020ED091030E80E5C9
:10C9B0000E94BC35882359F00E94FE346B017C0133
:10C9C00011E0672B682B692B31F410E004C010E0F4
:10C9D000C12CD12C760183E50E94BC35882309F453
:10C9E00069C00E943E3520E030E04AE754E40E94EE
:10C9F000D9AD0E9421B36B017C01111109C0672BD5
:10CA0000682B692B29F4209719F08881811102C0C5
:10CA100010E001C011E053DE1123A9F0EAECFFE1C0
:10CA200084918F010F5F1F4F882321F00E94D876D9
:10CA3000F801F6CF8991882319F00E94D876FACFB1
:10CA40008AE00E94D87683E08093E40C81E08093B2
:10CA5000C40DC114D104E104F10429F10E945C3C2D
:10CA6000C60ED71EE81EF91E0E945C3CDC01CB01FD
:10CA70008C199D09AE09BF09B7FD0EC01092C40DF7
:10CA800081E08093E40CDF91CF911F910F91FF9093
:10CA9000EF90DF90CF9008958091C40D882371F3BB
:10CAA0000E94B594E1CF8091C40D882339F30E9490
:10CAB000B594F9CF1111ACCFA6CF3F924F925F92B0
:10CAC0006F927F928F929F92AF92BF92CF92DF929E
:10CAD000EF92FF920F931F93CF93DF9384E0C82EC2
:10CAE00083E0D82E06E21EE09DE0E92E9EE0F92EBE
:10CAF000C0E0312CD0E0F60181916F010E94BC357D
:10CB00008823B9F10E943E354B015C01C33049F0E6
:10CB1000F70120813181428153810E94D7B14B01BD
:10CB20005C01F8012081318142815381C501B4014A
:10CB30000E94D7B12B013C012DEB37E346E855EBC2
:10CB40000E94FEB387FD0AC02DEB37E346E855E3AC
:10CB5000C301B2010E9474AD18165CF4C33019F021
:10CB60003324339401C0D1E0F80180829182A28203
:10CB7000B382CF5F0C5F1F4FF4E0EF0EF11CC430A7
:10CB800009F0B9CF332019F00E94733455C0DD236A
:10CB900009F452C0C090320ED090330EE090340EA3
:10CBA000F090350E2091B70D3091B80D4091B90D30
:10CBB0005091BA0DC701B6010E94D9AD0E9409B4C7
:10CBC0006093A10E7093A20E8093A30E9093A40E77
:10CBD000C092910ED092920EE092930EF092940E2B
:10CBE00090914B0E80914C0E981711F00ADD24C0E5
:10CBF00066DD80916F0081FB992790F981FF05C068
:10CC000080916F008D7F80936F004091A10E5091B5
:10CC1000A20E6091A30E7091A40E4093E00D50936C
:10CC2000E10D6093E20D7093E30D992329F080915B
:10CC30006F00826080936F00DF91CF911F910F9101
:10CC4000FF90EF90DF90CF90BF90AF909F908F902C
:10CC50007F906F905F904F903F900C9407418F9220
:10CC60009F92AF92BF92CF92DF92EF92FF921F936B
:10CC7000CF93DF93CDB7DEB728970FB6F894DEBF1A
:10CC80000FBECDBFC090260ED090270EE090280E8C
:10CC9000F090290E88E50E94BC35811108C020E083
:10CCA00030E0A901C701B6010E94D8B102C00E94BC
:10CCB0003E356D837E838F839887C0902A0ED090F7
:10CCC0002B0EE0902C0EF0902D0E89E50E94BC35C5
:10CCD000811108C020E030E0A901C701B6010E941F
:10CCE000D8B102C00E943E359B01AC0169837A83B2
:10CCF0008B839C836D817E818F8198850E94B79301
:10CD0000882309F48FC080E00E94BA340E94233146
:10CD100085E40E94BC35882321F00E942F35182F0E
:10CD200004C085E40E94753511E086E50E94BC359B
:10CD3000882321F00E940E35262F01C021E0412FCB
:10CD4000BE016F5F7F4FCE0105960E947BA66B01EF
:10CD50007C019B01AC010E9484B481115FC08D8075
:10CD60009E80AF80B88420E030E0A901C501B40105
:10CD70000E9474AD87FD05C027E137EB41E558E31C
:10CD800004C027E137EB41E558EBC501B4010E942F
:10CD9000D8B1AB01BC0182E691E10E949950898033
:10CDA0009A80AB80BC8020E030E0A901C501B401CD
:10CDB0000E9474AD87FD05C027E137EB41E558E3DC
:10CDC00004C027E137EB41E558EBC501B4010E94EF
:10CDD000D8B1AB01BC018DE591E10E94995020E0F2
:10CDE00030E0A901C701B6010E9474AD87FD05C0FE
:10CDF00027E137EB41E558E304C027E137EB41E594
:10CE000058EBC701B6010E94D8B1AB01BC0188E55F
:10CE100091E10E9499508AE00E94D8760E940A31DE
:10CE20000E94074128960FB6F894DEBF0FBECDBF13
:10CE3000DF91CF911F91FF90EF90DF90CF90BF9047
:10CE4000AF909F908F9008952F923F924F925F9254
:10CE50006F927F928F929F92AF92BF92CF92DF920A
:10CE6000EF92FF920F931F93CF93DF93CDB7DEB76F
:10CE7000C650D1400FB6F894DEBF0FBECDBF41E023
:10CE800061E081E00E94853081110C94BE76809132
:10CE9000620D882371F08FE40E94BC35882319F05D
:10CEA0000E942F3503C08FE40E94753581110C94C8
:10CEB000BE76FE0131968CE3DF011D928A95E9F77B
:10CEC0003090620D8AE40E947535882321F00E941B
:10CED000D1340C94BE7686E50E94BC35882349F097
:10CEE0000E940E35C153DF4F79836883CF5CD040F9
:10CEF00006C0C153DF4F19821882CF5CD040C153A6
:10CF0000DF4F08811981CF5CD0400530110570F0EA
:10CF1000E0E3F1E184918F010F5F1F4F882311F44B
:10CF20000C94BE760E94D876F801F4CF84E40E9477
:10CF3000BC35882319F00E942F3503C084E40E9479
:10CF40007535C251DF4F8883CE5ED040C153DF4F6D
:10CF500008811981CF5CD040033011058CF484E541
:10CF60000E94BC35882319F00E942F3503C084E548
:10CF70000E947535CD50DF4F8883C35FD04006C017
:10CF800011E0CD50DF4F1883C35FD04088E50E9489
:10CF9000BC35882321F00E940E35162F01C012E007
:10CFA00089E50E94BC35882321F00E940E35062FAA
:10CFB00001C002E080E50E94BC35811102C0612FF2
:10CFC00003C00E940E35062F623071F0E7E0F1E1F8
:10CFD00084918F010F5F1F4F882311F40C94BE764C
:10CFE0000E94D876F801F4CF023071F0EEEDF0E156
:10CFF00084918F010F5F1F4F882311F40C94BE762C
:10D000000E94D876F801F4CF83E50E94BC358823CE
:10D0100019F00E943E3504C060E070E88BEB95E4A7
:10D0200020E030E040E752E40E94B4B2609359023D
:10D0300070935A0280935B0290935C028CE40E948E
:10D04000BC35882381F00E943E3520910D0E309131
:10D050000E0E40910F0E5091100E0E94D7B10E94FB
:10D060001CB35B0104C01DEFA12EBB24BA9482E562
:10D070000E94BC35882381F00E943E3520910D0E20
:10D0800030910E0E40910F0E5091100E0E94D7B1AC
:10D090000E941CB37B0103C0B1EAEB2EF12C86E4A5
:10D0A0000E94BC35882381F00E943E352091110EEC
:10D0B0003091120E4091130E5091140E0E94D7B170
:10D0C0000E941CB36B0104C0A9EFCA2EDD24DA94C0
:10D0D00082E40E94BC35882381F00E943E35209175
:10D0E000110E3091120E4091130E5091140E0E94A9
:10D0F000D7B10E941CB38B0102C001EA10E0B60157
:10D100000D2C000C880B990B0E947AADC751DF4F94
:10D11000688379838A839B83C95ED040B5010B2CD9
:10D12000000C880B990B0E947AADC151DF4F6883C8
:10D1300079838A839B83CF5ED040C751DF4F28819C
:10D1400039814A815B81C95ED0400E94B7938111C9
:10D1500003C0E2ECF0E142C0B801012E000C880BE4
:10D16000990B0E947AAD9B01AC01B7010F2C000C0A
:10D17000880B990BCB5FDE4F2883C550D140CA5F27
:10D18000DE4F3883C650D140CD5FDE4F4883C35059
:10D19000D140CC5FDE4F5883C450D1400E947AAD5D
:10D1A000CB5FDE4F2881C550D140CA5FDE4F38814A
:10D1B000C650D140CD5FDE4F4881C350D140CC5FD7
:10D1C000DE4F5881C450D1400E94B793CC50DF4FFE
:10D1D0008883C45FD04081110DC0BBCF84918F0183
:10D1E0000F5F1F4F882311F40C94BE760E94D876EF
:10D1F000F801F4CFB7016A197B09072E000C880BE0
:10D20000990B0E947AADCB50DF4F688379838A8374
:10D210009B83C55FD040B8016C197D09072E000CB7
:10D22000880B990B0E947AADC750DF4F68837983D2
:10D230008A839B83C95FD040C153DF4F0881198126
:10D24000CF5CD040012B11F1ECEAF0E184918F0129
:10D250000F5F1F4F882321F00E94D876F801F6CF88
:10D26000C251DF4F0881CE5ED040002361F0E2EA78
:10D27000F0E184918F010F5F1F4F882321F00E94FE
:10D28000D876F801F6CF8AE00E94D87618DA80E0E6
:10D290000E94BA3481E00E941F32882329F0832D36
:10D2A0000E94BA340C94BE760E94233185E40E9419
:10D2B000BC35882359F00E942F35882359F011E09E
:10D2C000CB51DF4F1883C55ED0400AC085E40E9471
:10D2D0007535F3CF02E0CB51DF4F0883C55ED040F8
:10D2E000CD53DF4F19821882C35CD040C953DF4F42
:10D2F000188219821A821B82C75CD040CF52DF4F3E
:10D300001882C15DD0400FEF1FEFC954DF4F198362
:10D310000883C75BD040CB52DF4F188219821A8234
:10D320001B82C55DD0401FEFC752DF4F1883C95D18
:10D33000D040C553DF4F0883CB5CD04011E02CE0D8
:10D34000C954DF4F48815981C75BD040249FC00139
:10D35000259F900D1124DC01AB55B14FC554DF4F13
:10D36000B983A883CB5BD040440F551F440F551F92
:10D37000CF51DF4F59834883C15ED040EDE3F0E0E9
:10D38000EC0FFD1FE40FF51FC154DF4FF983E88355
:10D39000CF5BD040C352DF4F19821882CD5DD040A1
:10D3A000CD53DF4F28813981C35CD040032E000C60
:10D3B000440B550BC350DF4F288339834A835B836B
:10D3C000CD5FD040CD53DF4F48815981C35CD04001
:10D3D000440F551FCF5FDE4F59834883C150D14062
:10D3E000C553DF4F0881CB5CD040101709F496C2BB
:10D3F000C350DF4F688179818A819B81CD5FD040A6
:10D400000E947AAD9B01AC01CB50DF4F68817981DE
:10D410008A819B81C55FD0400E94D9AD9B01AC0140
:10D42000C151DF4F688179818A819B81CF5ED04075
:10D430000E94D8B14B015C01612F012E000C770BCB
:10D44000880B990B0E947AAD9B01AC01C750DF4F4E
:10D45000688179818A819B81C95FD0400E94D9AD62
:10D460009B01AC01C751DF4F688179818A819B8123
:10D47000C95ED0400E94D8B16B017C0120E030E051
:10D48000A901C501B4010E9474AD87FD05C020E06B
:10D4900030E040E05FE303C020E030E0A901C501D7
:10D4A000B4010E94D8B10E944DB3C355DF4F6883C9
:10D4B00079838A839B83CD5AD04020E030E0A90154
:10D4C000C701B6010E9474AD87FD05C020E030E0C1
:10D4D00040E05FE303C020E030E0A901C701B601EE
:10D4E0000E94D8B10E944DB3C755DF4F688379833E
:10D4F0008A839B83C95AD040C954DF4F8881998160
:10D50000C75BD0400196C954DF4F99838883C75BBE
:10D51000D040CF5FDE4FE881F981C150D140E10FAB
:10D52000F11D17FDFA95EE0FFF1FA1EAB0E0AC0F59
:10D53000BD1FEA0FFB1F91838083C153DF4F2881FA
:10D54000CF5CD040CB51DF4F4881C55ED040BE019B
:10D5500067557F4FCE0183559F4F0E947BA6C953CD
:10D56000DF4F688379838A839B83C75CD0409B01AC
:10D57000AC010E9484B4882321F0832D0E94BA3428
:10D58000E6C1C953DF4F288139814A815B81C75C7D
:10D59000D040CB52DF4F688179818A819B81C55D04
:10D5A000D0400E94D8B1CB52DF4F688379838A8301
:10D5B0009B83C55DD040C352DF4FE881F981CD5DCB
:10D5C000D040CF51DF4F28813981C15ED040E20F7A
:10D5D000F31F4DE650E04C0F5D1FE40FF51FC953DC
:10D5E000DF4F88819981AA81BB81C75CD040848349
:10D5F0009583A683B783C355DF4FC880D980EA805F
:10D60000FB80CD5AD040C154DF4FA881B981CF5B98
:10D61000D0401496CD92DD92ED92FC921797C755AB
:10D62000DF4F288039804A805B80C95AD040FD0195
:10D63000248A358A468A578A20E030E040E85FE352
:10D6400094962D933D934D935C939797A7019601E4
:10D6500069817A818B819C810E94D8B169837A83A8
:10D660008B839C83A20191016D817E818F8198853E
:10D670000E94D8B16D837E838F839887C953DF4F13
:10D68000288139814A815B81C75CD04069857A8570
:10D690008B859C850E94D8B169877A878B879C8708
:10D6A000A7019601C701B6010E94D9AD9B01AC014B
:10D6B0006D857E858F8598890E94D8B16D877E871C
:10D6C0008F87988BA2019101C201B1010E94D9AD4F
:10D6D0009B01AC0169897A898B899C890E94D8B1A8
:10D6E000698B7A8B8B8B9C8BC953DF4F2881398157
:10D6F0004A815B81C75CD040CA01B9010E94D9ADA3
:10D700009B01AC016D897E898F89988D0E94D8B16B
:10D710006D8B7E8B8F8B988FA2019101C701B60113
:10D720000E94D9AD9B01AC01698D7A8D8B8D9C8D4A
:10D730000E94D8B1698F7A8F8B8F9C8FC953DF4F2E
:10D74000288139814A815B81C75CD040C701B6011D
:10D750000E94D9AD9B01AC016D8D7E8D8F8D98A1FE
:10D760000E94D8B16D8F7E8F8F8F98A3C953DF4FE2
:10D77000288139814A815B81C75CD040C201B101F7
:10D780000E94D9AD9B01AC0169A17AA18BA19CA19A
:10D790000E94D8B169A37AA38BA39CA36DA07EA09D
:10D7A0000FA1B8A5C351DF4FB883CD5ED04020E0B4
:10D7B00030E0A901C701B6010E94FEB3460157013E
:10D7C00087FF04C0B7FAB094B7F8B0949301402F24
:10D7D000C351DF4F5881CD5ED040C501B4010E94D6
:10D7E000FEB318163CF04301A02EC351DF4FB880A2
:10D7F000CD5ED0408DA29EA2AFA2B8A669A47AA4A5
:10D800000BA5ECA5C351DF4FE883CD5ED04020E0EF
:10D8100030E0A901C201B1010E94FEB352014101F1
:10D8200087FF04C0B7FAB094B7F8B0949301402FC3
:10D83000C351DF4F5881CD5ED040C501B4010E9475
:10D84000FEB318163CF04301A02EC351DF4FB88041
:10D85000CD5ED04089A69AA6ABA6BCA620E030E05B
:10D8600040E85FE369AD7AAD8BAD9CAD0E94D8B165
:10D8700069AF7AAF8BAF9CAFC554DF4FA881B98138
:10D88000CB5BD0401C96CD92DD92ED92FC921F971F
:10D89000FD01208A318A428A538AC953DF4F288189
:10D8A00039814A815B81C75CD04054962D933D936A
:10D8B0004D935C9357970E94B594C752DF4F0881F0
:10D8C000C95DD040100FC554DF4F28813981CB5B33
:10D8D000D040245F3F4FC554DF4F39832883CB5B53
:10D8E000D040C352DF4F48815981CD5DD0404C5F5D
:10D8F0005F4FC352DF4F59834883CD5DD040C15441
:10D90000DF4F88819981CF5BD0400496C154DF4FAF
:10D9100099838883CF5BD040312C62CDCD53DF4FCC
:10D9200008811981C35CD0400130110581F0C953D1
:10D93000DF4F288139814A815B81C75CD040CA01B1
:10D94000B9010E9484B4882311F40C948B7680E092
:10D950000E941F32882329F0832D0E94BA340C9430
:10D960007E76C953DF4F288139814A815B81C75C4C
:10D97000D040CA01B9010E9484B481110C947E7612
:10D9800089AC9AACABACBCAC20E030E0A901C501DD
:10D99000B4010E9474AD882309F411C2A501940159
:10D9A00069817A818B819C810E94B4B2C954DF4F16
:10D9B000688379838A839B83C75BD04069837A833A
:10D9C0008B839C83A50194016D817E818F819885D5
:10D9D0000E94B4B2C554DF4F688379838A839B83E6
:10D9E000CB5BD0406D837E838F839887A5019401A4
:10D9F00069857A858B859C850E94B4B2C154DF4FBE
:10DA0000688379838A839B83CF5BD04069877A87D9
:10DA10008B879C87A50194016D857E858F8598896C
:10DA20000E94B4B26B017C01C954DF4F2881398157
:10DA30004A815B81C75BD040CA01B9010E94D9AD60
:10DA40009B01AC01C701B6010E94D7B1C553DF4F9E
:10DA5000688379838A839B83CB5CD0406D877E8784
:10DA60008F87988BA501940169897A898B899C8914
:10DA70000E94B4B26B017C01C554DF4F288139810B
:10DA80004A815B81CB5BD040CA01B9010E94D9AD0C
:10DA90009B01AC01C701B6010E94D7B1C752DF4F4D
:10DAA000688379838A839B83C95DD040698B7A8B35
:10DAB0008B8B9C8BA50194016D897E898F89988DB4
:10DAC0000E94B4B26B017C01C154DF4F28813981BF
:10DAD0004A815B81CF5BD040CA01B9010E94D9ADB8
:10DAE0009B01AC01C701B6010E94D7B16D8B7E8B43
:10DAF0008F8B988FA5019401698D7A8D8B8D9C8D6C
:10DB00000E94B4B26B017C01C554DF4F288139817A
:10DB10004A815B81CB5BD040C954DF4F68817981FA
:10DB20008A819B81C75BD0400E94D9AD9B01AC012B
:10DB3000C701B6010E94D7B1CD53DF4F6883798307
:10DB40008A839B83C35CD040698F7A8F8B8F9C8F35
:10DB5000A501940169A17AA18BA19CA10E94B4B2F4
:10DB60006B017C01C154DF4F288139814A815B817F
:10DB7000CF5BD040C554DF4F688179818A819B811A
:10DB8000CB5BD0400E94D9AD9B01AC01C701B6016F
:10DB90000E94D7B1CF52DF4F688379838A839B83FA
:10DBA000C15DD04069A37AA38BA39CA3A501940176
:10DBB0006D8D7E8D8F8D98A10E94B4B24B015C015A
:10DBC000C154DF4F288139814A815B81CF5BD040CE
:10DBD000C954DF4F688179818A819B81C75BD040BE
:10DBE0000E94D9AD9B01AC01C501B4010E94D7B11F
:10DBF0004B015C016D8F7E8F8F8F98A3C752DF4FD3
:10DC0000288139814A815B81C95DD040C553DF4F8E
:10DC1000688179818A819B81CB5CD0400E94D9AD9B
:10DC20002B013C01CD53DF4F288139814A815B8133
:10DC3000C35CD040CA01B9010E94D9AD9B01AC01BF
:10DC4000C301B2010E94D7B16B017C0120E030E03A
:10DC5000A9010E94FEB32601370187FF04C077FAAD
:10DC6000709477F8709429A53AA54BA55CA56DA191
:10DC70007EA18FA198A50E94D8B12FEF36EE4BED73
:10DC80005EE20E94D9AD9B01AC01C301B2010E94CA
:10DC900074AD18160CF093C0CD53DF4F2881398135
:10DCA0004A815B81C35CD040CF52DF4F688179816C
:10DCB0008A819B81C15DD0400E94D9AD2B013C017E
:10DCC000C752DF4F288139814A815B81C95DD040CD
:10DCD000C501B4010E94D9AD9B01AC01C301B201E1
:10DCE0000E94D7B1A70196010E94B4B22B013C015A
:10DCF0006DA77EA78FA798ABCD53DF4F28813981C1
:10DD00004A815B81C35CD040C501B4010E94D9AD9A
:10DD10004B015C01C553DF4F288139814A815B810A
:10DD2000CB5CD040CF52DF4F688179818A819B8163
:10DD3000C15DD0400E94D9AD9B01AC01C501B401C9
:10DD40000E94D7B1A70196010E94B4B26B017C0179
:10DD500069AB7AAB8BAB9CABC954DF4F288139815F
:10DD60004A815B81C75BD040C301B2010E94D9AD3B
:10DD70009B01AC01C154DF4F688179818A819B810D
:10DD8000CF5BD0400E94D8B14B015C01C554DF4F3E
:10DD9000288139814A815B81CB5BD040C701B601C4
:10DDA0000E94D9AD9B01AC01C501B4010E94D8B15C
:10DDB000DC01CB01B0588DAB9EABAFABB8AF2DA59E
:10DDC0003EA54FA558A9C554DF4F288339834A8300
:10DDD0005B83CB5BD0405058C154DF4F28833983DD
:10DDE0004A835B83CF5BD04089A99AA9ABA9BCA920
:10DDF000CD53DF4F88839983AA83BB83C35CD04014
:10DE00000DA91EA92FA938ADC151DF4F0883198371
:10DE10002A833B83CF5ED04020E030E040E85EE3E1
:10DE2000CB52DF4F688179818A819B81C55DD0406B
:10DE30000E94D9ADC752DF4F688379838A839B8361
:10DE4000C95DD040C153DF4F08811981CF5CD040FC
:10DE5000012B09F464C24090B90E5090BA0E609044
:10DE6000BB0E7090BC0E2091C50E3091C60E409135
:10DE7000C70E5091C80EC301B2010E94D7B1C35260
:10DE8000DF4F688379838A839B83CD5DD040C090C8
:10DE9000B50ED090B60EE090B70EF090B80E20916F
:10DEA000C10E3091C20E4091C30E5091C40EC701F5
:10DEB000B6010E94D7B1CF51DF4F688379838A833F
:10DEC0009B83C15ED0408090B10E9090B20EA09026
:10DED000B30EB090B40E2091BD0E3091BE0E4091A5
:10DEE000BF0E5091C00EC501B4010E94D7B1CB51F5
:10DEF000DF4F688379838A839B83C55ED0402091FE
:10DF0000AD0E3091AE0E4091AF0E5091B00EC55394
:10DF1000DF4F288339834A835B83CB5CD040A301E6
:10DF20009201C553DF4F688179818A819B81CB5CE7
:10DF3000D0400E94D7B1C751DF4F688379838A836D
:10DF40009B83C95ED0408091A90E9091AA0EA091AA
:10DF5000AB0EB091AC0ECB52DF4F88839983AA836E
:10DF6000BB83C55DD040A7019601BC01CD010E94D5
:10DF7000D7B16B017C010091A50E1091A60E2091E6
:10DF8000A70E3091A80ECF52DF4F088319832A8342
:10DF90003B83C15DD040A5019401CF52DF4F688122
:10DFA00079818A819B81C15DD0400E94D7B14B01AC
:10DFB0005C01CF51DF4F288139814A815B81C15E8D
:10DFC000D0400E94D9AD2B013C01CB51DF4F2881BD
:10DFD00039814A815B81C55ED040C701B6010E948C
:10DFE000D9AD9B01AC01C301B2010E94D7B1C954A4
:10DFF000DF4F688379838A839B83C75BD040CB5193
:10E00000DF4F288139814A815B81C55ED040C7518D
:10E01000DF4F688179818A819B81C95ED0400E94EF
:10E02000D9AD2B013C01C352DF4F288139814A8190
:10E030005B81CD5DD040C501B4010E94D9AD9B018B
:10E04000AC01C301B2010E94D7B12B013C01C35204
:10E05000DF4F288139814A815B81CD5DD040C70186
:10E06000B6010E94D9AD6B017C01CF51DF4F2881F1
:10E0700039814A815B81C15ED040C751DF4F6881E1
:10E0800079818A819B81C95ED0400E94D9AD9B0174
:10E09000AC01C701B6010E94D7B16B017C01209190
:10E0A000C90E3091CA0E4091CB0E5091CC0E0E94F9
:10E0B000D9AD4B015C012091CD0E3091CE0E409137
:10E0C000CF0E5091D00EC301B2010E94D9AD9B0179
:10E0D000AC01C501B4010E94D8B14B015C01209193
:10E0E000D10E3091D20E4091D30E5091D40EC9541E
:10E0F000DF4F688179818A819B81C75BD0400E9414
:10E10000D9AD9B01AC01C501B4010E94D8B14B014E
:10E110005C01CF52DF4F688179818A819B81C15D2B
:10E12000D0409058A70196010E94D9ADCF52DF4F41
:10E13000688379838A839B83C15DD040A301920168
:10E14000CB52DF4F688179818A819B81C55DD04048
:10E150000E94D9AD9B01AC01CF52DF4F688179811C
:10E160008A819B81C15DD0400E94D7B1CB52DF4FE5
:10E17000688379838A839B83C55DD040C954DF4F10
:10E18000288139814A815B81C75BD040C553DF4F0D
:10E19000688179818A819B81CB5CD0400E94D9AD16
:10E1A0009B01AC01CB52DF4F688179818A819B81D1
:10E1B000C55DD0400E94D7B19B01AC01C501B4013F
:10E1C0000E94D8B14B015C0120E030E0A9010E941F
:10E1D000FEB3181624F0B7FAB094B7F8B094A701BC
:10E1E0009601C701B6010E94D9AD6B017C01A30164
:10E1F0009201C301B2010E94D9AD9B01AC01C701DC
:10E20000B6010E94D8B16B017C01C954DF4F28814F
:10E2100039814A815B81C75BD040CA01B9010E9444
:10E22000D9AD9B01AC01C701B6010E94D8B10E94D3
:10E2300043B49B01AC01C501B4010E94B4B2AB016F
:10E24000BC018BE790E10E9499508AE0B1D58AE049
:10E25000AFD5E5E6F0E184918F010F5F1F4F882372
:10E2600019F0A6D5F801F7CF48E0C154DF4F688117
:10E2700079818A819B81CF5BD0400E94877BE0E6D9
:10E28000F0E184918F010F5F1F4F882319F090D523
:10E29000F801F7CF48E0CD53DF4F688179818A815B
:10E2A0009B81C35CD04090580E94877BEBE5F0E1F6
:10E2B00084918F010F5F1F4F882319F079D5F801E2
:10E2C000F7CFC151DF4F688179818A819B81CF5E11
:10E2D000D040905848E00E94877B8AE069D5C153BE
:10E2E000DF4F08811981CF5CD04003301105BCF0AD
:10E2F00002E410E1F8018491882321F00F5F1F4FA1
:10E3000057D5F8CF48E0C752DF4F688179818A81BD
:10E310009B81C95DD0400E94877B8AE049D5C2516C
:10E32000DF4F0881CE5ED0400111E9C1C554DF4FF7
:10E33000288139814A815B81CB5BD040CB56DF4F4E
:10E34000288339834A835B83C559D040CD53DF4F3F
:10E3500088819981AA81BB81C35CD040C756DF4FB9
:10E3600088839983AA83BB83C959D040C12CD12CFF
:10E3700060E8E62E6FE3F62EC356DF4FC882D982DF
:10E38000EA82FB82CD59D040CE018B569F4F0E942E
:10E390003692C757DF4FC882D982EA82FB82C958BA
:10E3A000D040C357DF4F188219821A821B82CD5882
:10E3B000D040C154DF4F088119812A813B81CF5B56
:10E3C000D040CF56DF4F088319832A833B83C1593E
:10E3D000D040CE0187579F4F0E943692CB56DF4FD9
:10E3E000288139814A815B81C559D040C954DF4FAA
:10E3F000288339834A835B83C75BD040C756DF4F8E
:10E40000488059806A807B80C959D040C356DF4F0D
:10E4100088809980AA80BB80CD59D040C757DF4FF4
:10E4200088819981AA81BB81C958D040C554DF4FEA
:10E4300088839983AA83BB83CB5BD040C357DF4FCC
:10E44000088119812A813B81CD58D040C154DF4FCA
:10E45000088319832A833B83CF5BD040CF56DF4F9D
:10E46000C880D980EA80FB80C159D040A7019601BD
:10E47000C301B2010E94D9ADCD53DF4F68837983C8
:10E480008A839B83C35CD040C154DF4F288139818C
:10E490004A815B81CF5BD040C501B4010E94D9ADF8
:10E4A0009B01AC01CD53DF4F688179818A819B81CB
:10E4B000C35CD0400E94D7B1C358DF4F68837983D3
:10E4C0008A839B83CD57D040C554DF4F2881398143
:10E4D0004A815B81CB5BD040C501B4010E94D9ADBC
:10E4E0004B015C01A7019601C954DF4F6881798116
:10E4F0008A819B81C75BD0400E94D9AD9B01AC0152
:10E50000C501B4010E94D7B1CF57DF4F688379832B
:10E510008A839B83C158D040C154DF4F2881398101
:10E520004A815B81CF5BD040C954DF4F68817981DC
:10E530008A819B81C75BD0400E94D9AD6B017C0171
:10E54000C554DF4F288139814A815B81CB5BD04044
:10E55000C301B2010E94D9AD9B01AC01C701B60154
:10E560000E94D7B1CB57DF4F688379838A839B831F
:10E57000C558D040CE0183589F4F0E943692C7574E
:10E58000DF4F088119812A813B81C958D040C35788
:10E59000DF4F488059806A807B80CD58D040CF566D
:10E5A000DF4F88809980AA80BB80C159D040C35872
:10E5B000DF4F88819981AA81BB81CD57D040C95452
:10E5C000DF4F88839983AA83BB83C75BD040CF5733
:10E5D000DF4F88819981AA81BB81C158D040C55441
:10E5E000DF4F88839983AA83BB83CB5BD040CB5713
:10E5F000DF4F88819981AA81BB81C558D040C15421
:10E60000DF4F88839983AA83BB83CF5BD040CB56EF
:10E61000DF4FC880D980EA80FB80C559D040C756FB
:10E62000DF4F488159816A817B81C959D040C356E7
:10E63000DF4F88819981AA81BB81CD59D040009359
:10E640004D0E10934E0E20934F0E3093500E40926D
:10E65000510E5092520E6092530E7092540E809250
:10E66000550E9092560EA092570EB092580EC95465
:10E67000DF4F088119812A813B81C75BD04000931D
:10E68000590E10935A0E20935B0E30935C0EC554B6
:10E69000DF4F088119812A813B81CB5BD0400093F9
:10E6A0005D0E10935E0E20935F0E3093600EC1548A
:10E6B000DF4F088119812A813B81CF5BD0400093D5
:10E6C000610E1093620E2093630E3093640EC0921D
:10E6D000650ED092660EE092670EF092680E40933F
:10E6E000690E50936A0E60936B0E70936C0E80935C
:10E6F0006D0E90936E0EA0936F0EB093700ECD5072
:10E70000DF4F1881C35FD040112309F454C2EFE7F3
:10E71000FFE084918F010F5F1F4F81113DC06E019B
:10E7200023EAC20ED11CC554DF4FD982C882CB5B0D
:10E73000D04002E0CB52DF4F0883C55DD040212C92
:10E7400010ECC154DF4F1883CF5BD04009E7CD53A5
:10E75000DF4F0883C35CD04014E4C553DF4F1883F8
:10E76000CB5CD0408E010B561F4FCF54DF4F198327
:10E770000883C15BD0400C501109CD54DF4F198381
:10E780000883C35BD0400C501109CB54DF4F198371
:10E790000883C55BD04038C00BD3F801BACF80E204
:10E7A00007D345E0C501B401B2D7C954DF4F088192
:10E7B0001981C75BD0400C5F1F4FC954DF4F1983CD
:10E7C0000883C75BD0400830110521F58AE0F0D2FC
:10E7D000C554DF4F08811981CB5BD040025011092D
:10E7E000C554DF4F19830883CB5BD040CB52DF4F3A
:10E7F0001881C55DD040113009F4F1C001E0CB5261
:10E80000DF4F0883C55DD040C954DF4F198218829D
:10E81000C75BD040C554DF4FE881F981CB5BD04066
:10E82000C954DF4F08811981C75BD040E00FF11F49
:10E83000008111817801EE0CFF1CEE0CFF1CEDE64F
:10E84000F0E0EC0FFD1FEE0DFF1D40805180628057
:10E850007380C752DF4F288139814A815B81C95D4E
:10E86000D040C301B2010E94D7B14B015C01E1E08D
:10E87000F0E0EC0FFD1FEE0DFF1D84AD95ADA6ADD4
:10E88000B7ADCB56DF4F88839983AA83BB83C55925
:10E89000D040F8013496EE0FFF1FEE0FFF1F21E06E
:10E8A00030E02C0F3D1FE20FF31F84AD95ADA6ADF8
:10E8B000B7ADC757DF4F88839983AA83BB83C958F5
:10E8C000D040C358DF4F188219821A821B82CD575D
:10E8D000D040CA54DF4F3881C65BD0403F93CB5401
:10E8E000DF4F4881C55BD0404F93CC54DF4F5881F8
:10E8F000C45BD0405F93CD54DF4F8881C35BD04071
:10E900008F93CE54DF4F9881C25BD0409F93CF54FA
:10E91000DF4FA881C15BD040AF93EDB7FEB7B4978E
:10E920000FB6F894FEBF0FBEEDBFADB7BEB71196E0
:10E93000EDE4FEE084E201900D928A95E1F70E94F9
:10E940005191C358DF4F288139814A815B81CD576E
:10E95000D040C301B2010E94D7B17B018C010FB638
:10E96000F894DEBF0FBECDBF9B01AC01622DC15438
:10E97000DF4F7881CF5BD040CD53DF4F8881C35CC0
:10E98000D040C553DF4F9881CB5CD0400E94FEB38E
:10E99000181684F42E2CC154DF4FF882CF5BD04080
:10E9A000CD53DF4F0883C35CD040C553DF4F18837E
:10E9B000CB5CD04020E030E0A901C501B4010E9449
:10E9C000FEB387FDECCEECE7FFE084918F010F5F93
:10E9D0001F4F882309F4E5CEEBD1F801F6CF8AE08A
:10E9E000E7D1C153DF4F08811981CF5CD04004309B
:10E9F000110509F0E0C0E3E5FFE084918F010F5FAE
:10EA00001F4F882319F0D4D1F801F7CF02E0C1538A
:10EA1000DF4F0883CF5CD0404E0115E9810E911C79
:10EA20005E0129E8A20EB11C7E013DE7E30EF11C58
:10EA300000E010E0F601E00FF11F808191813C01C0
:10EA4000660C771C660C771CE1E0F0E0EC0FFD1F14
:10EA5000E60DF71D44AD55AD66AD77ADD4014D93D0
:10EA60005D936D937C931397FC013496EE0FFF1F1B
:10EA7000EE0FFF1F21E030E02C0F3D1FE20FF31FD0
:10EA800084AD95ADA6ADB7ADF50180839183A2832A
:10EA9000B383D7011D921D921D921C921397FF9272
:10EAA000EF92BF92AF929F928F92EDB7FEB7B4975D
:10EAB0000FB6F894FEBF0FBEEDBFADB7BEB711964F
:10EAC000EDE4FEE084E201900D928A95E1F70E9468
:10EAD0005191EDE6F0E0EC0FFD1FE60DF71DD701BB
:10EAE0002D913D914D915C916081718182819381E5
:10EAF0000E94D7B1222DC154DF4F3881CF5BD04067
:10EB0000CD53DF4F4881C35CD040C553DF4F5881A0
:10EB1000CB5CD0400E94D7B12B013C010FB6F894DA
:10EB2000DEBF0FBECDBF20E030E0A9010E94FEB3E2
:10EB300087FD1FC0E0E5FFE084919F012F5F3F4FFD
:10EB40008823C9F0CB5FDE4F2883C550D140CA5F10
:10EB5000DE4F3883C650D1402BD1CB5FDE4F2881AA
:10EB6000C550D140CA5FDE4F3881C650D140F9014F
:10EB7000E3CF80E21DD145E0C301B201C8D50C5FEF
:10EB80001F4F0830110509F055CF8AE011D1F2E08E
:10EB9000CF1AD108C153DF4F0881CF5CD04001307C
:10EBA00039F011E0C153DF4F1883CF5CD04040CF24
:10EBB0008AE0FED008C0C153DF4F08811981CF5CC5
:10EBC000D040012B21F081E39FE00E9494A8C25124
:10EBD000DF4F1881CE5ED040111184C08CE0E6E298
:10EBE000FEE0DE01A358BF4F01900D928A95E1F738
:10EBF00081E08093620DCE0183589F4F0E94AD63E8
:10EC0000C355DF4F288139814A815B81CD5AD0407D
:10EC10006091260E7091270E8091280E9091290EFA
:10EC20000E94D7B16B017C012DEB37E346E855EB31
:10EC30000E94FEB387FD4BC02DEB37E346E855E35A
:10EC4000C701B6010E9474AD18160CF440C0C75538
:10EC5000DF4F288139814A815B81C95AD040609158
:10EC60002A0E70912B0E80912C0E90912D0E0E94E9
:10EC7000D7B16B017C012DEB37E346E855EB0E94E1
:10EC8000FEB387FD24C02DEB37E346E855E3C7010B
:10EC9000B6010E9474AD1816D4F0C953DF4F288115
:10ECA00039814A815B81C75CD04060912E0E7091A2
:10ECB0002F0E8091300E9091310E0E94D7B1CB571C
:10ECC000DF4F688379838A839B83C558D0408CE06B
:10ECD000FE01E358FF4FA6E2BEE001900D928A9537
:10ECE000E1F705C0CC50DF4F3882C45FD040CC5034
:10ECF000DF4F0881C45FD0400093620D0E940A314B
:10ED000081E08093E40C8091620D81110E94733444
:10ED10000E94074133C081E0CF52DF4F1881C15DAF
:10ED2000D0401827CF52DF4F1883C15DD04011115A
:10ED300017C01FEFC752DF4F1883C95DD0400FEFD8
:10ED4000C553DF4F0883CB5CD04011E021E030E0B9
:10ED5000CD53DF4F39832883C35CD0400C949F6927
:10ED600001E0C752DF4F0883C95DD04012E0C553B0
:10ED7000DF4F1883CB5CD04010E0E8CFCA5FDE4F96
:10ED80000FB6F894DEBF0FBECDBFDF91CF911F91BC
:10ED90000F91FF90EF90DF90CF90BF90AF909F903A
:10EDA0008F907F906F905F904F903F902F9008953D
:10EDB00091E09093C9049091C10095FD04C0909199
:10EDC000C00095FD40C02091C7042F5F2F710FB682
:10EDD00007FC34C09091C804291322C09091C00050
:10EDE00095FF1DC09091C8044091C704491791F048
:10EDF000E92FF0E0E955FB4F30819F5F9F71309321
:10EE0000C6009093C8043091C00030643093C000B5
:10EE1000491305C09091C1009F7D9093C100DACF46
:10EE2000E091C704F0E0E955FB4F80832093C704CD
:10EE30008091C10080628093C10008959091C804C0
:10EE40002913EECFFBCF8093C6008091C000806471
:10EE50008093C0000895CF93DF931F921F92CDB788
:10EE6000DEB7789484B5826084BD84B5816084BD4A
:10EE700085B5826085BD85B5816085BD80916E0058
:10EE8000816080936E001092810080918100826089
:10EE900080938100809181008160809381008091C6
:10EEA00080008160809380008091B10084608093B5
:10EEB000B1008091B00081608093B000809191009A
:10EEC0008260809391008091910081608093910095
:10EED000809190008160809390008091A100826079
:10EEE0008093A1008091A10081608093A100809116
:10EEF000A00081608093A0008091210182608093B6
:10EF00002101809121018160809321018091200164
:10EF100081608093200180917A00846080937A00E0
:10EF200080917A00826080937A0080917A0081607B
:10EF300080937A0080917A00806880937A001092A2
:10EF4000C10082E08093C0001092C50087E08093EA
:10EF5000C4008091C10080618093C1008091C10094
:10EF600088608093C1008091C10080688093C10057
:10EF70008091C1008F7D8093C1001092C904E0E6AA
:10EF8000F2E184918F010F5F1F4F882319F010DF8A
:10EF9000F801F7CFEAECFFE184918F010F5F1F4F7B
:10EFA000882319F005DFF801F7CF14B710FF0CC064
:10EFB000E7E5F2E184917F019FEFE91AF90A8823DE
:10EFC00019F0F6DEF701F6CF11FF0CC0E6E4F2E12E
:10EFD00084917F019FEFE91AF90A882319F0E8DE8E
:10EFE000F701F6CF12FF0CC0E4E3F2E184917F0158
:10EFF0009FEFE91AF90A882319F0DADEF701F6CF54
:10F0000013FF0CC0E3E2F2E184917F019FEFE91A64
:10F01000F90A882319F0CCDEF701F6CF15FF0BC0F3
:10F02000E2E1F2E184918F010F5F1F4F882319F015
:10F03000BFDEF801F7CF14BEEBE0F2E184918F015F
:10F040000F5F1F4F882319F0B3DEF801F7CF80E27E
:10F05000AFDEE4E0F2E184918F010F5F1F4F882360
:10F0600019F0A6DEF801F7CF8AE0A2DEEAECFFE1B4
:10F0700084918F010F5F1F4F882319F099DEF801EB
:10F08000F7CFE4EFF1E184918F010F5F1F4F8823E9
:10F0900019F08EDEF801F7CFE0EEF1E184918F01F7
:10F0A0000F5F1F4F882319F083DEF801F7CFE7EADF
:10F0B000F1E184918F010F5F1F4F882319F078DEF3
:10F0C000F801F7CFEAECFFE184918F010F5F1F4F4A
:10F0D000882319F06DDEF801F7CFE0E9F1E18491C2
:10F0E0008F010F5F1F4F882319F062DEF801F7CF01
:10F0F000EAECFFE184918F010F5F1F4F882319F025
:10F1000057DEF801F7CF2091D50E3091D60ECE0103
:10F1100001962115310519F48B5D9E4002C0821BBA
:10F12000930B9A83898369817A8181E891E10E94B6
:10F13000975160E875E08AE691E10E9497518AE074
:10F1400037DE81E08093FE048093FF048093000506
:10F1500080930105809302050E94919F8CE0E2EF6D
:10F16000F4E0A6E2BEE001900D928A95E1F70E94DC
:10F1700073346D9A809101018061809301018091C7
:10F1800001018860809301019D9A80910101806254
:10F190008093010188E00E94D9A8809101018860D4
:10F1A0008093010186E00E94D9A887ED80937A00C0
:10F1B00010927E0010927D0080917E00816080938D
:10F1C0007E0080917E00846080937E0080E888BD10
:10F1D00080916E00846080936E006AEF70E080E042
:10F1E00090E00E94223C85E090E09093CF048093D1
:10F1F000CE0460E080913302909134020E942B4B48
:10F2000020E030E040EA50E40E9474AD87FF0AC07D
:10F21000809133029091340240979093340280930E
:10F220003302E7CF81E391E0909336028093350279
:10F2300060E08091CC049091CD040E942B4B20E0A3
:10F2400030E848E953E40E94FEB3181654F4809164
:10F25000CC049091CD0440969093CD048093CC043F
:10F26000E7CF80913102909132020E94B24C20E0AF
:10F2700030E040EA50E40E9474AD87FF0AC08091FC
:10F280003102909132024097909332028093310282
:10F29000E8CF8091CA049091CB040E94B24C20E048
:10F2A00030E046E153E40E94FEB3181654F4809116
:10F2B000CA049091CB0440969093CB048093CA04E7
:10F2C000E8CF1092DC041092D8041092D904109266
:10F2D000DA041092DB041092D4041092D504109238
:10F2E000D6041092D7041092D0041092D104109238
:10F2F000D2041092D30482E390E00E943AB18631A6
:10F3000019F00E943C3808C040E150E063E370E02F
:10F310008EED94E00E942AB181E08093DD0426986E
:10F320002E9A25982D9A24982C9A3F98479A0A98B5
:10F33000129A0998119A8093EF048093EE048091B9
:10F340000A01886080930A0180910A01806180939C
:10F350000A0180910A01806280930A010E942FA312
:10F3600080912101887F816080932101999A989AE8
:10F37000809107018068809307019A9A8091070124
:10F380008064809307018091070180628093070168
:10F390008091070188608093070180910701806157
:10F3A000809307012CE0E22E23E0F22E10E0F7011B
:10F3B00061917F01812F0E94BDA21F5F1530B9F7B7
:10F3C00080910A01826080930A0180910A01816024
:10F3D00080930A0180910A01846080930A018091E0
:10F3E0000A01806480930A010F9A179A0E9A169A5E
:10F3F0000D9A159A0C9A149A389A4098179A8091F7
:10F40000F0048E7F8093F004399A4198169A809187
:10F41000F0048D7F8093F0043A9A4298159A809177
:10F42000F0048B7F8093F0043B9A4398149A809168
:10F4300080008C7F8093800080918100877E88602F
:10F4400080938100809180008F73809380008091F1
:10F450008100887F82608093810080E090E49093B7
:10F46000890080938800109285001092840080911A
:10F470006F00826080936F0081E08093EF04789446
:10F480000E94E6861092F1048091010188608093C9
:10F49000010198E288E10FB6F894A8958093600086
:10F4A0000FBE9093600080E6D82E90E0E92E90E0A9
:10F4B000F92E8091E606853030F40E94FD338111EB
:10F4C00002C00E94E4328091E606882309F439C024
:10F4D0000091E506D09E800111240C5F1A4F8091A7
:10F4E000030580FF17C0EAECFFE184915F019FEF05
:10F4F000A91AB90A811102C0580103C059DCF501EB
:10F50000F4CFF50181915F01882311F051DCF9CF2F
:10F510008AE04EDCC8010E945EA081E00E94CF100C
:10F520008091E606882369F081508093E6068091F9
:10F53000E5068F5F853018F48093E50602C01092CF
:10F54000E5068091250E882309F436C09091250E9A
:10F550008091E406981781F1EAECFFE184918F0134
:10F560000F5F1F4F882319F023DCF801F7CFE3E783
:10F57000F2E184918F010F5F1F4F882319F018DC8F
:10F58000F801F7CF8091250E80FD23C08091250ED4
:10F5900084FD1FC08091250E81FD25C08091250E20
:10F5A00085FD21C08091250E82FD27C08091250E0A
:10F5B00086FD23C08AE0FCDB8091250E8093E40663
:10F5C0000E94B594E114F10409F473CF0E94000085
:10F5D00070CF80E00E948063AB01BC018FE692E1B6
:10F5E0000E949950D7CF81E00E948063AB01BC019B
:10F5F0008BE692E10E949950D5CF82E00E94806311
:10F60000AB01BC0187E692E10E949950D3CF8F9263
:10F610009F92AF92BF92EF92FF921F93CF93DF938F
:10F62000CDB7DEB7A0970FB6F894DEBF0FBECDBF43
:10F63000611571058105910579F110E0842E912CF9
:10F64000A12CB12CEE24E394F12CEC0EFD1EE10E66
:10F65000F11C17FDFA94A50194010E9480B1F701F5
:10F660006083B901CA011F5F6115710581059105AC
:10F6700049F7115010F1E1E0F0E0EC0FFD1FE10F50
:10F68000F11D17FDFA9580818A3010F097E301C0D3
:10F6900090E3890F8DDBEDCF80E3A0960FB6F89451
:10F6A000DEBF0FBECDBFDF91CF911F91FF90EF90D6
:10F6B000BF90AF909F908F907BCBA0960FB6F894A1
:10F6C000DEBF0FBECDBFDF91CF911F91FF90EF90B6
:10F6D000BF90AF909F908F900895CF92DF92EF925E
:10F6E000FF926B017C0197FF0AC08DE261DBF09411
:10F6F000E094D094C094C11CD11CE11CF11C4AE0E0
:10F70000C701B601FF90EF90DF90CF9080CF8F922E
:10F710009F92AF92BF92CF92DF92EF92FF92CF93E0
:10F720006B017C01B42E20E030E0A9010E9474AD91
:10F7300087FF06C08DE23CDBF7FAF094F7F8F0940F
:10F74000C0E060E070E080E09FE3CB1541F02DEC7D
:10F750003CEC4CEC5DE30E94D9ADCF5FF6CF9B0152
:10F76000AC01C701B6010E94D8B16B017C010E94B7
:10F7700021B34B015C014AE04ADFCC2379F1C5019A
:10F78000B4010E9478AD9B01AC01C701B6010E9493
:10F79000D7B16B017C018EE20BDB20E030E040E270
:10F7A00051E4C701B6010E94D9AD4B015C010E9432
:10F7B0001CB36B01770FEE08FF08C701B6018DDFA0
:10F7C000C701B6010E947AAD9B01AC01C501B4012D
:10F7D0000E94D7B16B017C01C150F9F6CF91FF9027
:10F7E000EF90DF90CF90BF90AF909F908F90089553
:10F7F0008091A5049091A604891759F0E92FF0E0B3
:10F80000EB5DFB4F80819F5F9F779093A60490E014
:10F8100008958FEF9FEF0895CF93DF938F38924035
:10F82000A1F0E8E3F0E28491EF012196882319F03A
:10F83000BFDAFE01F8CFE2E8F2E18491EF01219610
:10F84000882329F0B5DAFE01F8CF80E001C081E01D
:10F85000DF91CF9108952F923F924F925F926F92D6
:10F860007F928F929F92AF92BF92CF92DF92EF9250
:10F87000FF920F931F93CF93DF93CDB7DEB7C5569B
:10F88000D1090FB6F894DEBF0FBECDBF2DB63EB680
:10F890006B961FAE1EAE6B9784E690E069969FAFA5
:10F8A0008EAF699701E09E01275A3F4F44E050E038
:10F8B000BE01655B7F4FCE01895A9F4F0E949E9F7C
:10F8C0009E01275A3F4F42E050E0BE016B5A7F4FE6
:10F8D000CE01895A9F4F0E949E9F43E050E0BE0197
:10F8E000655B7F4F81E193E00E94E1B4892B09F4CD
:10F8F00038C02F968FAD2F97882339F08FE32C9641
:10F900008FAF2C972D961FAE2D97EAECFFE18491D7
:10F910008F010F5F1F4F882319F04ADAF801F7CFE4
:10F92000E5E4F3E184918F010F5F1F4F882319F005
:10F930003FDAF801F7CFBE01655B7F4F8CE393E1BF
:10F940000E94B051EEE2F3E184918F010F5F1F4FEF
:10F95000882319F02DDAF801F7CF81E08093E706CC
:10F96000E2C42DB73EB7A4963FAF2EAFA4972B9617
:10F970001CAE1DAE1EAE1FAE2B976B961FAE1EAEFD
:10F980006B9701E09E01275A3F4F41E050E0BE01D6
:10F99000605A7F4FCE01895A9F4F0E949E9F80E1FF
:10F9A000E1E6F2E0DE01919601900D928A95E1F791
:10F9B00080E1E1E7F2E0DE01519601900D928A9537
:10F9C000E1F780E1E1E8F2E09E012F5F3F4F79012E
:10F9D000D90101900D928A95E1F7A1964FADA197BB
:10F9E00050E04D5F5F4F440F551F440F551F8DB7BB
:10F9F0009EB7841B950B0FB6F8949EBF0FBE8DBFAC
:10FA0000EDB7FEB731964F0100E0285A3F4FBF01D6
:10FA1000CE01895A9F4F0E949E9F9E01275A3F4FB9
:10FA200044E050E06BE77DE0CE01895A9F4F0E9491
:10FA30009E9FA1966FACA197712CF3E06F0E711C85
:10FA4000660C771C660C771C2DB73EB72619370954
:10FA50000FB6F8943EBF0FBE2DBF8DB79EB701966F
:10FA60005C01EDB7FEB7E619F7090FB6F894FEBFD3
:10FA70000FBEEDBF2DB73EB72F5F3F4F69019E010F
:10FA8000275A3F4FA301BC01CE01895A9F4F0E94C4
:10FA90009E9F9E01275A3F4FA301B601CE01895A6E
:10FAA0009F4F0E949E9F8091390D882309F4A3C027
:10FAB00000E09E01275A3F4F44E050E067E87DE0B8
:10FAC000CE01895A9F4F0E949E9F9E01275A3F4F09
:10FAD00044E050E063E87DE0CE01895A9F4F0E94E8
:10FAE0009E9F9E01275A3F4F44E050E06FE77DE024
:10FAF000CE01895A9F4F0E949E9F9E01275A3F4FD9
:10FB000044E050E067E77DE0CE01895A9F4F0E94B4
:10FB10009E9F9E01275A3F4F44E050E063E77DE0FF
:10FB2000CE01895A9F4F0E949E9F9E01275A3F4FA8
:10FB300040E150E063E67DE0CE01895A9F4F0E948C
:10FB40009E9F9E01275A3F4F44E050E0BE01695BF3
:10FB50007F4FCE01895A9F4F0E949E9F9E01275A38
:10FB60003F4F4CE050E062EF74E0CE01895A9F4F66
:10FB70000E949E9F9E01275A3F4F44E050E0BE01E5
:10FB8000695B7F4FCE01895A9F4F0E949E9F9E01C5
:10FB9000275A3F4F44E050E0BE01695B7F4FCE01E2
:10FBA000895A9F4F0E949E9F01E09E01275A3F4F16
:10FBB00041E050E0BE01615A7F4FCE01895A9F4F0C
:10FBC0000E949E9F9E01275A3F4F41E050E0BE0198
:10FBD000625A7F4FCE01895A9F4F0E949E9FA096E6
:10FBE0008FADA0976F96EFAC6F978E9D700111242B
:10FBF000C12CD12C5FC0A1962FADA19730E02E5F14
:10FC00003F4F8BE99DE0A6969FAF8EAFA697ABEADC
:10FC1000BDE06BE87DE080E090E040E050E024173C
:10FC2000350714F0840104C001E210E00C0F1D1F21
:10FC3000080F191FF8014080518062807380FB011A
:10FC40004192519261927192BF012417350714F0CD
:10FC5000850104C001E110E00C0F1D1F080F191FE2
:10FC6000F80140805180628073804D925D926D9268
:10FC70007D922417350714F0860101C08701080F13
:10FC8000191FF8014080518062807380A696EEAD06
:10FC9000FFADA6974192519261927192A696FFAFE5
:10FCA000EEAFA6974F5F5F4F04964430510509F0C1
:10FCB000B6CFFECECE14DF0491F000E09E01275AAD
:10FCC0003F4F44E050E0BE01695B7F4FCE01895A4F
:10FCD0009F4F0E949E9FFFEFCF1ADF0AEBCF6B96DC
:10FCE000EEACFFAC6B9769968EAD9FAD6997909324
:10FCF00038028093370200E09E01275A3F4F44E0CC
:10FD000050E066E37EE0CE01895A9F4F0E949E9F9D
:10FD10006B96FFAEEEAE6B979E01275A3F4F44E2C3
:10FD200050E06DE47EE0CE01895A9F4F0E949E9F75
:10FD300001E09E01275A3F4F41E050E0BE01635A67
:10FD40007F4FCE01895A9F4F0E949E9F9E01275A46
:10FD50003F4F41E050E0BE01645A7F4FCE01895AC7
:10FD60009F4F0E949E9F00E09E01275A3F4F44E014
:10FD700050E0BE01695C7F4FCE01895A9F4F0E94BF
:10FD80009E9F9E01275A3F4F44E050E0BE016F5CAA
:10FD90007F4FCE01895A9F4F0E949E9F6E968FADD6
:10FDA0006E976D96EFAC6D978E9D70011124C12CEE
:10FDB000D12C00E09E01275A3F4FCE14DF0471F092
:10FDC00044E050E0BE01695B7F4FCE01895A9F4FEE
:10FDD0000E949E9F2FEFC21AD20AEBCF41E050E063
:10FDE000BE016F597F4FCE01895A9F4F0E949E9F3F
:10FDF0009E01275A3F4F41E050E0BE01655A7F4FB8
:10FE0000CE01895A9F4F0E949E9F9E01275A3F4FC5
:10FE100044E050E0BE016D5B7F4FCE01895A9F4F99
:10FE20000E949E9F9E01275A3F4F44E050E0BE0132
:10FE3000615C7F4FCE01895A9F4F0E949E9F9E0119
:10FE4000275A3F4F44E050E0BE01655C7F4FCE0132
:10FE5000895A9F4F0E949E9F10E000E09E01275A02
:10FE60003F4F44E050E0BE01695B7F4FCE01895AAD
:10FE70009F4F0E949E9F111143C02B96CCACDDACCE
:10FE8000EEACFFAC2B9720E030E84BE355E4C70124
:10FE9000B6010E9474AD882399F18091390D8111CA
:10FEA00008C0C0925E0DD0925F0DE092600DF0929E
:10FEB000610D00E09E01275A3F4F44E050E06AE5A3
:10FEC0007DE0CE01895A9F4F0E949E9F9E01275A36
:10FED0003F4F44E050E066E57DE0CE01895A9F4FF8
:10FEE0000E949E9F9E01275A3F4F44E050E0BE0172
:10FEF000695B7F4FCE01895A9F4F0E949E9F14C01D
:10FF000084E0F82EFA94FF2079F000E09E01275A51
:10FF10003F4F44E050E0BE01695B7F4FCE01895AFC
:10FF20009F4F0E949E9FEECF1F5F153009F095CF27
:10FF300000E09E01275A3F4F42E050E0BE016D5A5B
:10FF40007F4FCE01895A9F4F0E949E9F9E01275A44
:10FF50003F4F44E050E0BE01695B7F4FCE01895ABC
:10FF60009F4F0E949E9F2B96CCACDDACEEACFFACBD
:10FF70002B9720E030E84BE355E4C701B6010E941F
:10FF800074AD882329F18091390D811108C0C09288
:10FF9000520DD092530DE092540DF092550D00E0A9
:10FFA0009E01275A3F4F44E050E06EE47DE0CE01D1
:10FFB000895A9F4F0E949E9F9E01275A3F4F44E0BF
:10FFC00050E06AE47DE0CE01895A9F4F0E949E9FD7
:10FFD00000E09E01275A3F4F42E050E0BE016F5AB9
:10FFE0007F4FCE01895A9F4F0E949E9F9E01275AA4
:10FFF0003F4F41E050E0BE016F597F4FCE01895A1B
:020000021000EC
:100000009F4F0E949E9F19E0115000E09E01275AC9
:100010003F4F112359F044E050E0BE01695B7F4F30
:10002000CE01895A9F4F0E949E9FEECF41E050E043
:100030006FEB7DE0CE01895A9F4F0E949E9F00E0AA
:100040009E01275A3F4F44E050E0BE01695B7F4F5D
:10005000CE01895A9F4F0E949E9F8091390D811138
:1000600010C011110EC02B968CAD9DADAEADBFADC5
:100070002B978093BB0D9093BC0DA093BD0DB093B7
:10008000BE0D1F5F1530D9F61CE0115079F000E06D
:100090009E01275A3F4F42E050E0BE01615B7F4F17
:1000A000CE01895A9F4F0E949E9FEFCF1CE01150B6
:1000B00000E09E01275A3F4F112359F044E050E0E1
:1000C000BE01695C7F4FCE01895A9F4F0E949E9F5F
:1000D000EECF46E050E0BE016F5C7F4FCE01895A03
:1000E0009F4F0E949E9F9E01275A3F4F44E050E041
:1000F00066E47DE0CE01895A9F4F0E949E9F13E0E7
:10010000115090F034E0139FB0011124665C724FDF
:1001100000E09E01275A3F4F44E050E0CE01895A4B
:100120009F4F0E949E9FECCF1CE1115079F000E0A0
:100130009E01275A3F4F44E050E0BE01695B7F4F6C
:10014000CE01895A9F4F0E949E9FEFCF14E011501D
:1001500079F000E09E01275A3F4F44E050E0BE0195
:10016000695B7F4FCE01895A9F4F0E949E9FEFCFC0
:100170001BE0115079F000E09E01275A3F4F44E008
:1001800050E0BE01695B7F4FCE01895A9F4F0E94AC
:100190009E9FEFCF69968EAD9FAD6997845691096A
:1001A0003BDB8093E706882301F1EAECFFE18491D1
:1001B0008F010F5F1F4F882321F00E94D876F8012E
:1001C000F6CF69966EAD7FAD69976456710986E288
:1001D00093E10E9497516FE872E08EE193E10E94F3
:1001E00097518AE00E94D8768BC06B962EAD3FADBA
:1001F0006B9767968EAD9FAD67972817390709F4FF
:1002000044C081E08093E706E8E3F0E284918F0147
:100210000F5F1F4F882321F00E94D876F801F6CF98
:10022000EEEFF2E184918F010F5F1F4F882321F0E1
:100230000E94D876F801F6CF67966EAD7FAD6797CE
:1002400080E090E04AE0E3D9E9EFF2E184918F01A8
:100250000F5F1F4F882321F00E94D876F801F6CF58
:100260006B966EAD7FAD6B9780E090E04AE0CFD9A2
:10027000E9EEF2E184918F010F5F1F4F882309F4AB
:100280003FC00E94D876F801F5CF8091390D8111D9
:1002900037C0EAECFFE184918F010F5F1F4F81119E
:1002A00003C001E113E004C00E94D876F801F3CF47
:1002B000F80181918F01882319F00E94D876F8CF38
:1002C00069966EAD7FAD6997645671098CEC92E1C9
:1002D0000E9497516B964EAD5FAD6B9760E070E0FA
:1002E0008FEB92E10E947C50ECEBF2E184918F0164
:1002F0000F5F1F4F882321F00E94D876F801F6CFB8
:100300008091390D811106C08091E706811102C0EC
:100310000E9441A3A4962EAD3FADA4970FB6F894CA
:100320003EBF0FBE2DBF8091390D811102C00E94CA
:10033000AA999091E70681E089270FB6F8943EBE0E
:100340000FBE2DBECB59DF4F0FB6F894DEBF0FBEE8
:10035000CDBFDF91CF911F910F91FF90EF90DF9074
:10036000CF90BF90AF909F908F907F906F905F9055
:100370004F903F902F9008958F929F92AF92BF928F
:10038000CF92DF92EF92FF920F931F93CF93DF9361
:10039000CDB7DEB7CA59D1090FB6F894DEBF0FBE8C
:1003A000CDBFCB57DF4F188219821A821B82C558E6
:1003B000D04085E492E5A2E5B0E0CF57DF4F8883D7
:1003C0009983AA83BB83C158D040CF56DF4F19828F
:1003D0001882C159D04084E690E0C157DF4F99831D
:1003E0008883CF58D0401092E7069E012F563F4F8A
:1003F00044E050E0BE016F577F4FCE0181579F4FC1
:100400000E94EB9FC157DF4F88819981CF58D04020
:100410000296C157DF4F99838883CF58D040CF567B
:10042000DF4F19821882C159D04081E0C656DF4F94
:100430008883CA59D0409E012F563F4F41E050E07B
:10044000BE0166567F4FCE0181579F4F0E94EB9FA2
:100450009E012F563F4F40E150E06BE87DE0CE011A
:1004600081579F4F0E94EB9F9E012F563F4F44E0C4
:1004700050E06BE77DE0CE0181579F4F0E94EB9FDC
:100480009E012F563F4F40E150E06BEA7DE0CE01E8
:1004900081579F4F0E94EB9F9E012F563F4F40E197
:1004A00050E06BE97DE0CE0181579F4F0E94EB9FAA
:1004B0009E012F563F4F44E050E067E87DE0CE01BB
:1004C00081579F4F0E94EB9F9E012F563F4F44E064
:1004D00050E063E87DE0CE0181579F4F0E94EB9F83
:1004E0009E012F563F4F44E050E06FE77DE0CE0184
:1004F00081579F4F0E94EB9F9E012F563F4F44E034
:1005000050E067E77DE0CE0181579F4F0E94EB9F4F
:100510009E012F563F4F44E050E063E77DE0CE015F
:1005200081579F4F0E94EB9F9E012F563F4F40E106
:1005300050E063E67DE0CE0181579F4F0E94EB9F24
:100540008AE097EDA3EABCE3CB57DF4F888399831A
:10055000AA83BB83C558D0409E012F563F4F44E02D
:1005600050E0BE016B577F4FCE0181579F4F0E94D5
:10057000EB9F9E012F563F4F4CE050E062EF74E03E
:10058000CE0181579F4F0E94EB9F80E090E0A0E258
:10059000B1E4C358DF4F88839983AA83BB83CD57C7
:1005A000D0409E012F563F4F44E050E0BE016358BB
:1005B0007F4FCE0181579F4F0E94EB9FCB57DF4F5C
:1005C000188219821A821B82C558D04083E0C75610
:1005D000DF4F8883C959D040C856DF4F8883C85938
:1005E000D0409E012F563F4F44E050E0BE016B5774
:1005F0007F4FCE0181579F4F0E94EB9F9E012F5648
:100600003F4F41E050E0BE0167567F4FCE0181571A
:100610009F4F0E94EB9F9E012F563F4F41E050E0BD
:10062000BE0168567F4FCE0181579F4F0E94EB9FBE
:100630001AE0115071F09E012F563F4F44E050E0F8
:10064000BE016B577F4FCE0181579F4F0E94EB9F9A
:10065000F0CFCF56DF4F08811981C159D040C15723
:10066000DF4F88819981CF58D04090933802809392
:1006700037029E012F563F4F44E050E066E37EE094
:10068000CE0181579F4F0E94EB9FCF56DF4F1983BA
:100690000883C159D0409E012F563F4F44E250E09D
:1006A0006DE47EE0CE0181579F4F0E94EB9F83E077
:1006B000C956DF4F8883C759D040CA56DF4F888359
:1006C000C659D040ED961CAE1DAE1EAE1FAEED97C6
:1006D000E9961CAE1DAE1EAE1FAEE997CB57DF4F9D
:1006E000188219821A821B82C558D0409E012F564B
:1006F0003F4F41E050E0BE0169567F4FCE01815728
:100700009F4F0E94EB9F9E012F563F4F41E050E0CC
:10071000BE016A567F4FCE0181579F4F0E94EB9FCB
:100720009E012F563F4F44E050E0BE016B587F4F73
:10073000CE0181579F4F0E94EB9F9E012F563F4F46
:1007400044E050E0BE0167587F4FCE0181579F4F74
:100750000E94EB9F0AE010E00150110971F09E0128
:100760002F563F4F44E050E0BE016B577F4FCE0104
:1007700081579F4F0E94EB9FEFCFCB56DF4F1882E0
:10078000C559D0408FEFCC56DF4F8883C459D04035
:100790009E012F563F4F41E050E0BE016B567F4F08
:1007A000CE0181579F4F0E94EB9F9E012F563F4FD6
:1007B00041E050E0BE016C567F4FCE0181579F4F04
:1007C0000E94EB9F88EC90E0E3969FAF8EAFE3979B
:1007D00080EF90E0E5969FAF8EAFE59786E490E0DE
:1007E000AF969FAF8EAFAF978EE690E0E1969FAF4A
:1007F0008EAFE197AB961FAE1EAEAB97AD961FAE18
:100800001EAEAD979E012F563F4F44E050E0BE0113
:100810006F587F4FCE0181579F4F0E94EB9F9E01E3
:100820002F563F4F44E050E0BE0163597F4FCE0149
:1008300081579F4F0E94EB9F9E012F563F4F44E0F0
:1008400050E0BE0167597F4FCE0181579F4F0E94F4
:10085000EB9F10E0C12C80E8D82E8BE3E82E85E4D6
:10086000F82E812C912C90E8A92E9FE3B92E11111E
:100870003AC09E012F563F4F44E050E06EE57DE0C8
:10088000CE0181579F4F0E94EB9F9E012F563F4FF5
:1008900044E050E06AE57DE0CE0181579F4F0E9421
:1008A000EB9F9E012F563F4F44E050E066E57DE010
:1008B000CE0181579F4F0E94EB9FCB57DF4F88821D
:1008C0009982AA82BB82C558D0409E012F563F4FC5
:1008D00044E050E0BE016B577F4FCE0181579F4FE0
:1008E0000E94EB9F2EC0CB57DF4FC882D982EA828D
:1008F000FB82C558D0409E012F563F4F44E050E048
:10090000BE016B577F4FCE0181579F4F0E94EB9FD7
:10091000CB57DF4F188219821A821B82C558D040EC
:1009200004E0015071F09E012F563F4F44E050E02B
:10093000BE016B577F4FCE0181579F4F0E94EB9FA7
:10094000F0CF1F5F153009F092CF84E190E0C357DC
:10095000DF4F99838883CD58D0409E012F563F4F5B
:1009600042E050E0BE0163577F4FCE0181579F4F59
:100970000E94EB9F9E012F563F4F44E050E062E5FE
:100980007DE0CE0181579F4F0E94EB9F9E012F5625
:100990003F4F44E050E06EE47DE0CE0181579F4F31
:1009A0000E94EB9F9E012F563F4F44E050E06AE4C7
:1009B0007DE0CE0181579F4F0E94EB9F80E290E047
:1009C000C557DF4F99838883CB58D0409E012F565F
:1009D0003F4F42E050E0BE0165577F4FCE01815747
:1009E0009F4F0E94EB9FCD56DF4F1882C359D040D6
:1009F00080E2E1E9F2E0DE019D9601900D928A9598
:100A0000E1F79E012F563F4F41E050E0BE016D5689
:100A10007F4FCE0181579F4F0E94EB9F9E012F5623
:100A20003F4F40E250E0BE01635D7F4FCE018157F2
:100A30009F4F0E94EB9F9E012F563F4F41E050E099
:100A40006FEB7DE0CE0181579F4F0E94EB9F10E03E
:100A5000111110C08091BB0D9091BC0DA091BD0DE6
:100A6000B091BE0DCB57DF4F88839983AA83BB8398
:100A7000C558D0409E012F563F4F44E050E0BE0184
:100A80006B577F4FCE0181579F4F0E94EB9F1F5F97
:100A90001530F1F6BE01635B7F4F86E1FB011192D9
:100AA0008A95E9F79E012F563F4F46E150E0CE016F
:100AB00081579F4F0E94EB9F8CE2E1EBF2E0DE0159
:100AC000119601900D928A95E1F79E012F563F4FA6
:100AD0004CE250E0BE016F5F7F4FCE0181579F4FC8
:100AE0000E94EB9FBE016D597F4F86E0FB01119282
:100AF0008A95E9F79E012F563F4F46E050E0CE0120
:100B000081579F4F0E94EB9F9E012F563F4F44E01D
:100B100050E066E47DE0CE0181579F4F0E94EB9F3D
:100B200013E0115088F0F4E01F9FB0011124665CBF
:100B3000724F9E012F563F4F44E050E0CE01815747
:100B40009F4F0E94EB9FEDCFCB57DF4F188219824A
:100B50001A821B82C558D0401CE1115071F09E01D1
:100B60002F563F4F44E050E0BE016B577F4FCE0100
:100B700081579F4F0E94EB9FF0CFCB57DF4F1882DA
:100B800019821A821B82C558D04014E0115071F0AE
:100B90009E012F563F4F44E050E0BE016B577F4F00
:100BA000CE0181579F4F0E94EB9FF0CFCB57DF4F75
:100BB000188219821A821B82C558D0401BE011503E
:100BC00071F09E012F563F4F44E050E0BE016B573D
:100BD0007F4FCE0181579F4F0E94EB9FF0CF8091B6
:100BE000E706811167C0C157DF4FE880F980CF5811
:100BF000D04084E6E81AF108CF56DF4F888199810A
:100C0000C159D040C757DF4F99838883C958D04016
:100C100084E690E0C157DF4F99838883CF58D04056
:100C20009E012F563F4F44E050E061E173E0CE015A
:100C300081579F4F0E94EB9F9E012F563F4F42E0EE
:100C400050E0BE0167577F4FCE0181579F4F0E94F2
:100C5000EB9FEAECFFE184918F010F5F1F4F882328
:100C600021F00E94D876F801F6CFB7018AEA92E126
:100C70000E949751C757DF4F48815981C958D040CA
:100C800060E070E08DE992E10E947C50EAE9F2E1D7
:100C900084918F010F5F1F4F882321F00E94D87627
:100CA000F801F6CFC7010E940C7C9091E706892BD2
:100CB0008093E7069091E70681E08927C656DF4FCB
:100CC0000FB6F894DEBF0FBECDBFDF91CF911F915D
:100CD0000F91FF90EF90DF90CF90BF90AF909F90DB
:100CE0008F90089580914B0E90914C0E891B8F70C0
:100CF00019F480E090E008959091480E992351F006
:100D0000833030F48FEF890F19F08093480EF1CFC4
:100D10001092480EE0914C0E88E5E89FF0011124F6
:100D2000E45FF84F808180FDE4CF80914C0E8F5FAF
:100D30008F708093490E90914C0E80914A0E9813BB
:100D400004C08091490E80934A0ECF0108950F93FD
:100D50000FB70F9300916E000F930B7F00936E00FF
:100D600000916F000D7F00936F000F930BB70F93EF
:100D70000CB70F921F922F933F934F935F936F93F4
:100D80007F938F939F93AF93BF93EF93FF93112420
:100D90005DD0FF91EF91BF91AF919F918F917F9126
:100DA0006F915F914F913F912F911F900F900CBFCA
:100DB0000F910BBF0F910260F89400936F000F9199
:100DC00000936E000F910FBF0F9118958091920CB8
:100DD00080FF07C080910B018270809309018FEF23
:100DE00007C080910B01809582708093090181E09A
:100DF00080938C0C8091920C81FF08C080910B0134
:100E000080958170809309018FEF06C080910B015E
:100E100081708093090181E080938D0C8091920C08
:100E200082FF07C080910B018470809309018FEFCE
:100E300007C080910B01809584708093090181E047
:100E400080938E0C00000000000008952F923F92C6
:100E50004F925F926F927F928F929F92AF92BF92CA
:100E6000CF92DF92EF92FF920F931F93CF93DF9376
:100E700000D000D0CDB7DEB7F8948FEF9FEF9093FE
:100E80008900809388002AE02E83212C312C7894CD
:100E90008091DC0C9091DD0CA091DE0CB091DF0C08
:100EA000892B8A2B8B2B09F0CDC18091C00D882313
:100EB000D1F01092C00D8091C60D9091C70D892B75
:100EC00091F01092D30C1092C70D1092C60D909114
:100ED0004B0E80914C0E981731F080914C0E8F5F25
:100EE0008F7080934C0E8091C60D9091C70D892B09
:100EF00009F4A8C14091D80C5091D90C6091DA0C3A
:100F00007091DB0C9091C60C0091D40C1091D50C13
:100F10002091D60C3091D70C041B150B260B370BE8
:100F2000892F90E0A0E0B0E0081719072A073B07D7
:100F300010F4D901C801E82F840F951FA61FB71F11
:100F40008093D80C9093D90CA093DA0CB093DB0C5F
:100F50002091840030918500225E3F4F4091AC0C7F
:100F60005091AD0C6091AE0C7091AF0C80919C0CC7
:100F700090919D0CA0919E0CB0919F0C840F951F99
:100F8000A61FB71F8093AC0C9093AD0CA093AE0C32
:100F9000B093AF0CB7FD1CC0409A4091D40D509156
:100FA000D50D6091D60D7091D70D80918C0C082EC7
:100FB000000C990BAA0BBB0B840F951FA61FB71F24
:100FC0008093D40D9093D50DA093D60DB093D70DEB
:100FD0004091B00C5091B10C6091B20C7091B30C77
:100FE0008091A00C9091A10CA091A20CB091A30CA7
:100FF000840F951FA61FB71F8093B00C9093B10C60
:10100000A093B20CB093B30CB7FD1CC0419A4091B1
:10101000D80D5091D90D6091DA0D7091DB0D809152
:101020008D0C082E000C990BAA0BBB0B840F951F7F
:10103000A61FB71F8093D80D9093D90DA093DA0DFA
:10104000B093DB0D4091B40C5091B50C6091B60C8F
:101050007091B70C8091A40C9091A50CA091A60C56
:10106000B091A70C840F951FA61FB71F8093B40CD7
:101070009093B50CA093B60CB093B70CB7FD1CC001
:10108000429A4091DC0D5091DD0D6091DE0D709122
:10109000DF0D80918E0C082E000C990BAA0BBB0B58
:1010A000840F951FA61FB71F8093DC0D9093DD0D55
:1010B000A093DE0DB093DF0D4091B80C5091B90CA8
:1010C0006091BA0C7091BB0C8091A80C9091A90C06
:1010D000A091AA0CB091AB0C840F951FA61FB71F4F
:1010E0008093B80C9093B90CA093BA0CB093BB0C3E
:1010F000B7FD3AC0C090E00DD090E10DE090E20D58
:10110000F090E30D40918F0C042E000C550B660BF4
:10111000770B4C0D5D1D6E1D7F1D4093E00D5093B0
:10112000E10D6093E20D7093E30D4091980C5091A6
:10113000990C60919A0C70919B0C841B950BA60BDB
:10114000B70B8093B80C9093B90CA093BA0CB093E2
:10115000BB0C9091920C8091C40C93FF02C0815003
:1011600001C08F5F8093C40C8091840090918500B2
:1011700082179307C8F38091AC0C9091AD0CA091AD
:10118000AE0CB091AF0CB7FD15C04091980C5091CA
:10119000990C60919A0C70919B0C841B950BA60B7B
:1011A000B70B8093AC0C9093AD0CA093AE0CB093A6
:1011B000AF0C40988091B00C9091B10CA091B20C02
:1011C000B091B30CB7FD15C04091980C5091990C9B
:1011D00060919A0C70919B0C841B950BA60BB70B1E
:1011E0008093B00C9093B10CA093B20CB093B30C5D
:1011F00041988091B40C9091B50CA091B60CB0912F
:10120000B70CB7FD15C04091980C5091990C6091A6
:101210009A0C70919B0C841B950BA60BB70B8093BB
:10122000B40C9093B50CA093B60CB093B70C429845
:10123000E15041F0809184009091850082179307DE
:10124000C8F38ACE8091420290914302A091440259
:10125000B0914502892B8A2B8B2B09F09AC0809183
:10126000C50C882309F455C0C090D80CD090D90C77
:10127000E090DA0CF090DB0C4091C00C5091C10C66
:101280006091C20C7091C30C8091C40C4C155D052B
:101290006E057F0588F42091900C3091910CE091BF
:1012A000950CF091960CE217F30730F4815080937F
:1012B000C40C2150310915C0C416D506E606F70640
:1012C000E8F42091900C3091910C4091930C509146
:1012D000940C2417350790F48F5F8093C40C2F5F14
:1012E0003F4F3093910C2093900C40913E025091CF
:1012F0003F0260914002709141020EC08FEF9FEF5C
:10130000DC0180933E0290933F02A0934002B09391
:1013100041024FEF5FEFBA018091C40C87FD03C01B
:1013200080910B0103C080910B01809580748093A4
:1013300009012091840030918500225E3F4F809109
:10134000C40C8823F1F0439A809184009091850029
:1013500082179307C8F38091C40C87FF02C08F5F88
:1013600001C081508093C40C43988091C40C8823A1
:1013700031F3809184009091850082179307C8F320
:10138000DCCF409342025093430260934402709337
:1013900045028091DC0C9091DD0CA091DE0CB091A7
:1013A000DF0C892B8A2B8B2B09F063C3A091C60D10
:1013B000B091C70D109739F1C090D80CD090D90CCE
:1013C000E090DA0CF090DB0C4091D40C5091D50CED
:1013D0006091D60C7091D70CC416D506E606F706B8
:1013E000C8F01092D30C1092C70D1092C60D9091B8
:1013F0004B0E80914C0E981731F080914C0E8F5F00
:101400008F7080934C0EA0ED8A2EA7E09A2EA12C0F
:10141000B12C81C14091CF0C5091D00C6091D10C76
:101420007091D20C4C155D056E057F0508F46EC0F9
:101430004091CB0C5091CC0C6091CD0C7091CE0CA6
:10144000D2960D911D912D913C91D597EE27419FFC
:10145000F12D529FC001629F900D619F800D911DE3
:10146000429FF00D811D9E1F519FF00D811D9E1FFB
:10147000609FF00D811D9E1F509FF10D8E1F9E1FBE
:10148000F6958E1F9E1F349F800D911D359F900DE8
:101490001124FD01EA5BFF4F00811181228133811C
:1014A000080F191F211D311D0093C70C1093C80C84
:1014B0002093C90C3093CA0C349780809180A2800D
:1014C000B38080169106A206B30640F48092C70C42
:1014D0009092C80CA092C90CB092CA0C8090C70C14
:1014E0009090C80CA090C90CB090CA0C8EE59BE1FE
:1014F00077247394FC010591159125913491081579
:1015000019052A053B0508F42EC338C32091C00CE9
:101510003091C10C4091C20C5091C30C29833A8385
:101520004B835C832C153D054E055F0508F068C0B4
:101530004091BC0C5091BD0C6091BE0C7091BF0CE1
:10154000D2960D911D912D913C91D597EE27419FFB
:10155000F12D529FC001629F900D619F800D911DE2
:10156000429FF00D811D9E1F519FF00D811D9E1FFA
:10157000609FF00D811D9E1F509FF10D8E1F9E1FBD
:10158000F6958E1F9E1F349F800D911D359F900DE7
:1015900011248C0120E030E04090C70C5090C80C22
:1015A0006090C90C7090CA0CFD01E65BFF4F0415FA
:1015B00015052605370580F480809180A280B380D0
:1015C000401A510A620A730A481459046A047B04D7
:1015D00038F42401350104C040805180628073805A
:1015E0008EE59BE131E03D83FC010591159125914C
:1015F0003491041515052605370508F43CC348C386
:101600008091C40C8823D9F0D8964D915C91D997DC
:1016100060E070E000913E0210913F022091400294
:1016200030914102041715072607370741F0109241
:1016300042021092430210924402109245024091DD
:101640003A0250913B0260913C0270913D0277FF5B
:101650005AC0AE5BBF4F8D919D910D90BC91A02D56
:101660002EE53BE141E0F901C590D590E590F4907D
:10167000C816D906EA06FB0658F4B695A7959795BD
:101680008795440F2C5F3F4F5BE12A37350759F7A9
:101690004093C60C80329105A105B10508F4E7C35B
:1016A0008097A109B1098115E8E09E07A105B10560
:1016B00008F4B8C324E0929FF00111249F01225A3C
:1016C000384EF901329645915491EE27859FB0012D
:1016D000849F610D7E1F06946E1F7E1F1124AB0137
:1016E00060E070E0F90185919491A0E0B0E0841B86
:1016F000950BA60BB70B80933A0290933B02A093F5
:101700003C02B0933D0280903A0290903B02A09040
:101710003C02B0903D028091C60D9091C70D892B7F
:1017200009F09FC1DFDA9093C70D8093C60D892B16
:1017300009F497C1E091C60DF091C70D808183FF38
:101740003EC085899689A789B08D8093D40D9093EA
:10175000D50DA093D60DB093D70D818D928DA38D0D
:10176000B48D8093D80D9093D90DA093DA0DB093DA
:10177000DB0D858D968DA78DB0A18093DC0D9093A8
:10178000DD0DA093DE0DB093DF0D81A192A1A3A189
:10179000B4A18093E00D9093E10DA093E20DB0937E
:1017A000E30D90914B0E80914C0E981709F4BACF2F
:1017B00080914C0E8F5F8F7080934C0EB3CFC58895
:1017C000D688E788F08C81E0C114D104E104F104EB
:1017D00009F480E0018D128D238D348D01151105E2
:1017E0002105310509F08260458D568D678D70A108
:1017F000411551056105710509F084608093D30C92
:101800001092BC0C1092BD0C1092BE0C1092BF0C2A
:101810001092CB0C1092CC0C1092CD0C1092CE0CDE
:1018200085A196A1A7A1B0A58093D40C9093D50CC7
:10183000A093D60CB093D70C882499245401881A0D
:10184000990AAA0ABB0A8092B80C9092B90CA0928D
:10185000BA0CB092BB0C8092B40C9092B50CA092D2
:10186000B60CB092B70C8092B00C9092B10CA092D2
:10187000B20CB092B30C8092AC0C9092AD0CA092D2
:10188000AE0CB092AF0CCC0CDD1CEE1CFF1CC09259
:101890009C0CD0929D0CE0929E0CF0929F0C000F3D
:1018A000111F221F331F0093A00C1093A10C209333
:1018B000A20C3093A30C440F551F661F771F409353
:1018C000A40C5093A50C6093A60C7093A70C41A197
:1018D00052A163A174A1440F551F661F771F409347
:1018E000A80C5093A90C6093AA0C7093AB0C880FB2
:1018F000991FAA1FBB1F8093980C9093990CA093DB
:101900009A0CB0939B0C1092D80C1092D90C109298
:10191000DA0C1092DB0C82A593A5A4A5B5A5809343
:10192000CF0C9093D00CA093D10CB093D20C86A581
:1019300097A5A0A9B1A98093C00C9093C10CA093C6
:10194000C20CB093C30C81A58093970C97A9909378
:10195000C50C992361F024AD35AD3093960C2093DE
:10196000950C22AD33AD3093940C2093930C96A933
:101970002091920C92130AC02091390230E0482F36
:10198000082E000C550B4217530729F09093920C28
:10199000809339021BDA0E94B6368FEF9FEFDC018D
:1019A00080933A0290933B02A0933C02B0933D0295
:1019B000E091C60DF091C70DEA5BFF4F80819181E8
:1019C000A281B3818093C70C9093C80CA093C90CDB
:1019D000B093CA0C2EE53BE141E0F901C590D590EA
:1019E000E590F490C816D906EA06FB0658F4B695B9
:1019F000A79597958795440F2C5F3F4FEBE12A37CA
:101A00003E0759F74093C60C80329105A105B105F8
:101A100008F455C28097A109B1098115E8E09E0735
:101A2000A105B10508F428C2F4E09F9F900111249C
:101A3000225A384EF901329645915491EE27859FEE
:101A4000B001849F610D7E1F06946E1F7E1F1124BE
:101A5000F90185909490A12CB12C861A970AA108BF
:101A6000B1088092DC0C9092DD0CA092DE0CB0925A
:101A7000DF0C0091DC0C1091DD0C2091DE0C30911C
:101A8000DF0C4091420250914302609144027091F8
:101A90004502F02EE12EF22FE32F40175107620787
:101AA000730720F4F42EE52EF62FE72F8F2D9E2DB1
:101AB000AF2FBE2F0097E1E0AE07B10520F08FEF0A
:101AC0009FEFA0E0B0E0081B190B2A0B3B0B009323
:101AD000DC0C1093DD0C2093DE0C3093DF0C4F3FB9
:101AE000FFEF5F076F077F0761F0481B590B6A0B19
:101AF0007B0B4093420250934302609344027093E5
:101B00004502F8942091840030918500205F3F4F7A
:101B10004E8141504E83442339F0280E391E22163F
:101B2000330608F4B4C901C019013092890020922B
:101B30008800789426960FB6F894DEBF0FBECDBF0E
:101B4000DF91CF911F910F91FF90EF90DF90CF9099
:101B5000BF90AF909F908F907F906F905F904F90CD
:101B60003F902F900895B694A79497948794770CFC
:101B70000496EBE18A379E0709F0BCCC7092C60C44
:101B800080E288169104A104B10408F41CC190E21B
:101B9000891A9108A108B1088114E8E09E06A10401
:101BA000B104F8F0F4E09F9EC0011124825A984ECF
:101BB000FC01329625913491F82DEE27F39F800198
:101BC000F29F010D1E1F06940E1F1E1F1124FC0103
:101BD00085909490A12CB12C801A910AA108B1088B
:101BE00023C0950184013695279517950795F8012F
:101BF000EC7F9F01225A3C4EF90185919491F901A5
:101C0000329605911491E82DE770E09F9001E19FD5
